:100000000C9442430C94C4430C94C4430C94C443D6
:100010000C94C4430C94C4430C94C4430C94C44344
:100020000C94C4430C94C4430C94C4430C94C44334
:100030000C94C4430C94E7470C94C4430C94C443FD
:100040000C94C4430C94C4430C94C4430C94C44314
:100050000C94C4430C94C4430C94C4430C94C44304
:100060000C94C4430C94C4430C94C4430C94C443F4
:100070000000000000000000000000000000000080
:100080000000000000000000000000000000000070
:100090000000000000000000000000000000000060
:1000A0000000FF00000000FFFFFF000000FFFFFF57
:1000B00000000000FF0000000000FF000000000042
:1000C000000000000000FF00000000000000000031
:1000D000FFFF00FFFF00FFFF00FFFF00FF0000FF2A
:1000E0000000000000000000000000000000000010
:1000F0000000000000000000000000000000000000
:1001000000000000000000FF00FF0000FFFFFFFFF5
:10011000FF0000FF00FF000000FF00FF0000FFFFE6
:10012000FFFFFF0000FF00FF0000000000000000D4
:1001300000FF0000000000FFFFFF0000FF000000C4
:10014000000000FFFF000000000000FF0000FFFFB4
:10015000FF0000000000FF000000000000000000A1
:10016000FFFF0000FF00FFFF0000FF00000000FF96
:1001700000000000FF00000000FF00000000FF0082
:1001800000FFFF00FF0000FFFF0000000000000074
:1001900000FF00000000FF00FF000000FF00FF0064
:1001A000000000FF00000000FF00FF00FF00FF0054
:1001B00000FF000000FFFF00FF0000000000000043
:1001C00000FFFF00000000FFFF00000000FF000034
:1001D000000000000000000000000000000000001F
:1001E000000000000000000000000000000000000F
:1001F0000000FF00000000FF0000000000FF000002
:10020000000000FF0000000000FF0000000000FFF1
:10021000000000000000FF000000000000000000DF
:1002200000FF000000000000FF0000000000FF00D1
:1002300000000000FF0000000000FF0000000000C0
:10024000FF00000000FF00000000000000000000B0
:1002500000000000000000FF00FF000000FFFFFFA3
:100260000000FFFFFFFFFF0000FFFFFF000000FF97
:1002700000FF00000000000000000000000000007F
:100280000000000000000000FF0000000000FF0070
:100290000000FFFFFFFFFF000000FF000000000064
:1002A000FF0000000000000000000000000000004F
:1002B000000000000000000000000000000000003E
:1002C000000000000000000000000000000000FF2F
:1002D000FF00000000FFFF00000000FF0000000022
:1002E000000000000000000000000000000000000E
:1002F0000000FFFFFFFFFF00000000000000000003
:1003000000000000000000000000000000000000ED
:1003100000000000000000000000000000000000DD
:10032000000000000000000000000000000000FFCE
:10033000FF00000000FFFF000000000000000000C0
:1003400000000000000000000000FF00000000FFAF
:1003500000000000FF00000000FF00000000FF00A0
:10036000000000000000000000000000000000008D
:10037000002F2F2F00002F0000002F002F00002F34
:100380002F002F002F002F002F2F00002F002F00F5
:1003900000002F00002F2F2F0000000000000000A1
:1003A00000002F000000002F2F00000000002F0091
:1003B000000000002F00000000002F0000000000DF
:1003C0002F000000002F2F2F000000000000000071
:1003D000002F2F2F00002F0000002F000000000032
:1003E0002F0000002F2F0000002F000000002F0022
:1003F000000000002F2F2F2F2F0000000000000012
:10040000002F2F2F00002F0000002F000000000001
:100410002F00002F2F2F0000000000002F002F00C2
:1004200000002F00002F2F2F000000000000000010
:100430000000002F000000002F2F0000002F002FD1
:1004400000002F00002F00002F2F2F2F2F00000063
:10045000002F00000000002F00000000000000003E
:100460002F2F2F2F2F002F00000000002F00000043
:1004700000002F2F2F2F0000000000002F002F0062
:1004800000002F00002F2F2F0000000000000000B0
:1004900000002F2F0000002F000000002F000000A0
:1004A00000002F2F2F2F00002F0000002F002F0003
:1004B00000002F00002F2F2F000000000000000080
:1004C0002F2F2F2F2F00000000002F000000002FE3
:1004D000000000002F000000002F00000000002F8F
:1004E00000000000002F00000000000000000000DD
:1004F000002F2F2F00002F0000002F002F000000E2
:100500002F00002F2F2F00002F0000002F002F00A2
:1005100000002F00002F2F2F00000000000000001F
:10052000002F2F2F00002F0000002F002F000000B1
:100530002F00002F2F2F2F00000000002F000000A1
:10054000002F0000002F2F0000000000000000001E
:1005500000000000000000000000000000FFFF009D
:10056000000000FFFF00000000000000000000FF8E
:10057000FF00000000FFFF0000000000000000007E
:1005800000000000000000000000000000FFFF006D
:10059000000000FFFF00000000000000000000FF5E
:1005A000FF00000000FFFF00000000FF000000004F
:1005B00000000000FF00000000FF00000000FF003E
:1005C000000000FF000000000000FF00000000002D
:1005D00000FF000000000000FF000000000000001D
:1005E000000000000000000000000000FFFFFFFF0F
:1005F000FF00000000000000000000000000FFFFFE
:10060000FFFFFF00000000000000000000000000ED
:1006100000FF000000000000FF000000000000FFDD
:10062000000000000000FF00000000FF00000000CC
:10063000FF00000000FF00000000000000000000BC
:1006400000FFFFFF0000FF000000FF0000000000AF
:10065000FF000000FFFF00000000FF00000000009E
:10066000000000000000FF0000000000000000008B
:1006700000FFFFFF0000FF000000FF00FF00FFFF82
:10068000FF00FF00FF00FF00FF00FFFFFF00FF0073
:100690000000000000FFFFFF00000000000000005D
:1006A00000FFFFFF0000FF000000FF00FF00000050
:1006B000FF00FF000000FF00FFFFFFFFFF00FF0043
:1006C0000000FF00FF000000FF000000000000002D
:1006D000FFFFFFFF0000FF000000FF00FF00000021
:1006E000FF00FFFFFFFF0000FF000000FF00FF0012
:1006F0000000FF00FFFFFFFF0000000000000000FF
:1007000000FFFFFF0000FF000000FF00FF000000EF
:100710000000FF0000000000FF0000000000FF00DC
:100720000000FF0000FFFFFF0000000000000000CD
:10073000FFFFFFFF0000FF000000FF00FF000000C0
:10074000FF00FF000000FF00FF000000FF00FF00AF
:100750000000FF00FFFFFFFF00000000000000009E
:10076000FFFFFFFFFF00FF0000000000FF00000090
:100770000000FFFFFFFF0000FF0000000000FF007F
:1007800000000000FFFFFFFFFF000000000000006E
:10079000FFFFFFFFFF00FF0000000000FF00000060
:1007A0000000FFFFFFFF0000FF0000000000FF004F
:1007B00000000000FF00000000000000000000003A
:1007C00000FFFFFF0000FF000000FF00FF0000002F
:1007D0000000FF00FFFFFF00FF000000FF00FF0020
:1007E0000000FF0000FFFFFFFF000000000000000E
:1007F000FF000000FF00FF000000FF00FF000000FE
:10080000FF00FFFFFFFFFF00FF000000FF00FF00F1
:100810000000FF00FF000000FF00000000000000DB
:1008200000FFFFFF00000000FF0000000000FF00CD
:1008300000000000FF0000000000FF0000000000BA
:10084000FF00000000FFFFFF0000000000000000AC
:1008500000000000FF0000000000FF00000000009A
:10086000FF0000000000FF00FF000000FF00FF008D
:100870000000FF0000FFFFFF00000000000000007C
:10088000FF000000FF00FF0000FF0000FF00FF006E
:100890000000FFFF00000000FF00FF000000FF005D
:1008A00000FF0000FF000000FF000000000000004B
:1008B000FF0000000000FF0000000000FF0000003B
:1008C0000000FF0000000000FF0000000000FF002B
:1008D00000000000FFFFFFFFFF000000000000001D
:1008E000FF000000FF00FFFF00FFFF00FF00FF0010
:1008F000FF00FF000000FF00FF000000FF00FF00FE
:100900000000FF00FF000000FF00000000000000EA
:10091000FF000000FF00FFFF0000FF00FF00FF00DE
:10092000FF00FF0000FFFF00FF000000FF00FF00CE
:100930000000FF00FF000000FF00000000000000BA
:1009400000FFFFFF0000FF000000FF00FF000000AD
:10095000FF00FF000000FF00FF000000FF00FF009D
:100960000000FF0000FFFFFF00000000000000008B
:10097000FFFFFFFF0000FF000000FF00FF0000007E
:10098000FF00FFFFFFFF0000FF0000000000FF006E
:1009900000000000FF000000000000000000000058
:1009A00000FFFFFF0000FF000000FF00FF0000004D
:1009B000FF00FF000000FF00FF00FF00FF00FF003E
:1009C00000FF000000FFFF00FF000000000000002B
:1009D000FFFFFFFF0000FF000000FF00FF0000001E
:1009E000FF00FFFFFFFF0000FF0000FF0000FF000F
:1009F0000000FF00FF000000FF00000000000000FA
:100A000000FFFFFF0000FF000000FF00FF000000EC
:100A1000000000FFFFFF000000000000FF00FF00DB
:100A20000000FF0000FFFFFF0000000000000000CA
:100A3000FFFFFFFFFF000000FF0000000000FF00BD
:100A400000000000FF0000000000FF0000000000A8
:100A5000FF0000000000FF00000000000000000098
:100A6000FF000000FF00FF000000FF00FF0000008B
:100A7000FF00FF000000FF00FF000000FF00FF007C
:100A80000000FF0000FFFFFF00000000000000006A
:100A9000FF000000FF00FF000000FF00FF0000005B
:100AA000FF00FF000000FF00FF000000FF0000FF4C
:100AB00000FF00000000FF00000000000000000038
:100AC000FF000000FF00FF000000FF00FF00FF002C
:100AD000FF00FF00FF00FF00FF00FF00FF00FF001E
:100AE000FF00FF0000FF00FF00000000000000000A
:100AF000FF000000FF00FF000000FF0000FF00FFFC
:100B000000000000FF00000000FF00FF0000FF00E9
:100B10000000FF00FF000000FF00000000000000D8
:100B2000FF000000FF00FF000000FF00FF000000CA
:100B3000FF0000FF00FF00000000FF0000000000B9
:100B4000FF0000000000FF000000000000000000A7
:100B5000FFFFFFFF0000000000FF00000000FF009B
:100B6000000000FF00000000FF0000000000FF0088
:100B700000000000FFFFFFFF000000000000000079
:100B80000000FFFF000000FF0000000000FF000069
:100B90000000FFFF0000000000FF0000000000FF59
:100BA000000000000000FFFF000000000000000047
:100BB0000000FFFF000000FF0000FF00FF00FFFF3C
:100BC00000FFFF00FF0000FFFF00FFFF00FF00FF2E
:100BD0000000FF000000FFFF000000000000000018
:100BE00000FFFF000000000000FF0000000000FF09
:100BF0000000000000FFFF00000000FF00000000F8
:100C000000FF000000FFFF000000000000000000E7
:100C10000000F114FF0000EE05FF0000EE010500EA
:100C200000FF0008640000DC02FF0008280000F656
:100C300007FF0008280000F607FF000000100C0066
:100C4000000000000000150C000000000200001A67
:100C50000C00000000030000220C00000000000057
:100C6000002A0C00000000020000320C000000000E
:100C7000FFFFFFFFFFFFFFFFFFFFFFFFFFFFFFFF84
:100C8000FFFFFFFFFFFFFFFFFFFFFFFFFFFFFFFF74
:100C9000FFFFFFFFFFFFFFFFFFFFFFFFFFFFFFFF64
:100CA0000000000000000000000000000000000044
:100CB0000000000000000000000000000000000034
:100CC0000000000000000000000000000000000024
:100CD0000000000000000000000000000000000014
:100CE0000000000000000000000000000000000004
:100CF00000000000000000000000000000000000F4
:100D000000000000000000000000000000000000E3
:100D100000000000000000000000000000000000D3
:100D200000000000000000000000000000000000C3
:100D300000000000000000000000000000000000B3
:100D400000000000000000000000000000000000A3
:100D50000000000000000000000000000000000093
:100D60005B5B5B5B5B5B5B5B5B5B5B5B5B090000DB
:100D7000095B5B5B5200095B5BADFF00095B5B5B82
:100D80005B5B5B5B5B5B5B5B5B5B5B5B5B5B5B5BB3
:100D90005B5B5B5B5B5B5B5B5B5B5B5B5B090000AB
:100DA000095B5B5B5200095B5BADFF00095B5B5B52
:100DB0005B5B5B5B5B5B5B5B5B5B5B5B5B5B5B5B83
:100DC0005B5B5B5B5B5B5B5B5B5B5B5B5B0900007B
:100DD000095B5B5B5200095B5BADFF00095B5B5B22
:100DE0005B5B5B5B5B5B5B5B5B5B5B5B5B5B5B5B53
:100DF0005B5B5B5B5B5B5B5B5B5B5B5B5B0900004B
:100E0000095B5B5B5200095B5BADFF00095B5B5BF1
:100E10005B5B5B5B5B5B5B5B5B5B5B5B5B5B5B5B22
:100E20000000001D0A001D1D1C000000000A1D5BC3
:100E30005C1C1D1D1C000A1D1D0A001C1D1D000937
:100E40005B1D0A005A5C1D1D5C5A1D0A001C1D1DFD
:100E5000000A1D000A1D1D0A00000A1D000A1D5B74
:100E600009001D1D1C000A1D1D0A001C1D1D1C5C07
:100E70005B1D0A005B09001C1D1D1D1D1C5B09007C
:100E8000000A1D1D1D1C1D5C52000A1D1D5C5B1D02
:100E90000A0000095B1C1D1C1D0A001D0A001D1D07
:100EA0001C0000001D0A001C5C52000A1D0000000E
:100EB0005B5C1D1D1D1C1D1D1C5B0900525C1C0084
:100EC0000A1D000A1D5B5C1C1D0A001D0A001C1D7A
:100ED0001C000A1D000A1D0000001D0A001D0A005A
:100EE000000000FFFFFF00A4FF5BADFFFFAE1DFF92
:100EF000AD5B52ADFF1D5C5B5B5B5B5A5C1D5A5C7E
:100F00001D5B5B5B5B5B5B1C1D1C5B5B5B5B5B5B2B
:100F1000FFA4000000001DAEFF000000FFFFFFFF68
:100F20005B001CAEFFFFFFFF52ADFFFFFFFF5A5CEF
:100F30001D52ADFF5B5A5BFFFFFF5A5C1D52ADFFB8
:100F40005B0900525B5B5B5B5200095B5B09005213
:100F50005B5B5B5B5200095B5B5B5B5B09000009F1
:100F60005B5B5B5B0000005B090000000000095B4D
:100F70005B5B5B5A5C1D5A5C1D5B5C1D5B5B5B5B7A
:100F80005B5B5B5B5B5B5B5B525B5B5B09005B5B67
:100F90005B5B09001C5C520000005B090000000064
:100FA00000000000095B000000000A1D0000005264
:100FB0005B5B00000014AE0000095BFF0000000A4C
:100FC0001D5B5B5B5B5C1D1D1D1D650A0000000059
:100FD00000A4000000005B090000000052ADFF000B
:100FE000000000AD5200000000000000A4005B5BA8
:100FF0005B5B09001D1D1D1CAE0000000000095BAD
:101000005B09000000001D1D1D1D1D1D00095B5B0F
:101010005B5B000A65FF000000000052AD000000AD
:10102000001C5C5A000000000A1D000000000A1DA0
:1010300000000000A4001D1D1D1D5C5B5B5B5B00D0
:10104000A4000000FF5B09000000FF0000005B5BE4
:10105000520000005B09000000001D0A00000000B3
:1010600000A4FFFFFFFF00095BFFFFFF00095B5BC0
:101070005B52000000000000FFFFFF005BFFFFFF6E
:10108000FF00095B5B5B5200095B00000000000091
:10109000005BFFFFFFFF00095BFFFFFF00095B5BD9
:1010A0005B5B000000000000FFFFFF005BFFFFFF35
:1010B000FF00095B5B5B5200095B00000000000061
:1010C00000A4FFFFFFFF00095BFFFFFF00095B5B60
:1010D0005B52000000000000FFFFFF005BFFFFFF0E
:1010E000FF00095B5B5B5200095B00000000000031
:1010F000005BFFFFFFFF00095BFFFFFF00095B5B79
:101100005B5B000000000000FFFFFF005BFFFFFFD4
:10111000FF00095B5B5B5200095B00000000000000
:101120000000000000000000005B09000000005209
:101130005B5B00095B00095B00095B00095B000069
:1011400000525B5B00000000095B000000525B5B2B
:1011500000000000000000095B0000005B5B520023
:1011600000005B09005B09005B09005B09005B5B39
:10117000520000005B09000000005B5B52000000B1
:1011800000095B005B0000A40000095B0000000098
:10119000A40000000000095B00000014AE00000085
:1011A000001D0A000000001D0A0000A40000A400A9
:1011B000005B005B09005B090000A40000A40000C4
:1011C00000005B090000000000AE14000000000AEF
:1011D0001D000000000A1D00000000A40000A40083
:1011E00000000000005200000000020D0000000995
:1011F000A4FF00000004A6FF00000909090900027D
:101200000D0D0D0D0900000000000D020000000092
:10121000FFA4000000000A0000000000FFFFFF0024
:101220000000FFA409000000090952FFA4000D0DF1
:101230000C0A000000000000A4FF00000000000AEB
:10124000090B0D0D0D0D0D0B09090909000052FFC9
:10125000FFFF00020DFFFFFF000000090909000069
:10126000000C0D0D00000000020D00000000020D3A
:101270000D0D0D04A6FF09090909090AFFFFFFFF6B
:10128000A400FFFFFF52000009ADFF0000000D0B9E
:10129000090000000A00000000000D02000000002C
:1012A00000000000005200000000020D00000009D4
:1012B000A4FF0000000D0B0900000A0C0D0D000238
:1012C0000D0000005200000000000C0D0D0D0D0D72
:1012D000FFA4000000000A0000000000FFFFFF0064
:1012E00000000909090000000D0D0DFFA400000019
:1012F0000009000000000000A4FF0D0D0D0D0B09FA
:101300005209090909090466FFFFFFFF000052FFA7
:10131000FFFF00020D0A0909000000090B0D000083
:10132000000D020000000000020D00000000020D90
:1013300009090909ADFFFFFFFFFFA409FFFFFFFF38
:10134000A40009090909000004A6FF00000000002C
:10135000090000000A00000000000D02000000006B
:1013600000000000005200000000020D0000000913
:1013700009090000000C0D0D00000900000000022A
:101380000D000000510B0D0D0D0D0D0B0909090984
:10139000FFA4000000000A000000000009ADFF00EB
:1013A00000000D0B09000000000000FFA400000079
:1013B000000900000D0D0D04A6FF09090909090A1D
:1013C00009A4FFFFFFFF0466FFFFFFFF00000909FC
:1013D000090900020D0D0D0D0000000900000000BC
:1013E000000D020000000000020D00000000020DD0
:1013F000FFFFFFFFFFFFFFFFFFFFA409090952FFE7
:10140000A4000D0D0C0A000000A4FF000000000065
:10141000090000000A00000000000D0200000000AA
:1014200000000000005200000000020D0000000952
:101430000B0D0000000D020000000900000000027A
:101440000D0D0D0D5209090909090466FFFFFFFF83
:10145000FFA4000000000A000000000004A6FF0036
:101460000000000009000000000000FFA4000D0DB6
:101470000C0A000009090909ADFFFFFFFFFFA409DD
:1014800009A4FFFFFFFF0D0B0909090900000A0C61
:101490000D0D00020D00000000000009000000001A
:1014A000000C0D0D00000000020D00000000020DF8
:1014B000FFFFFFFFFFFF09090909090A0D0D0DFFD5
:1014C000A40000000009000000A4FF0000000D0BB4
:1014D000090000000A00000000000D0200000000EA
:1014E00000000000005200000000020D0000000992
:1014F00000000000000D020000000A0C0D0D0002AB
:101500000D0A090909A4FFFFFFFF0466FFFFFFFFA3
:10151000FFA4000000000A000000000000A4FF007B
:1015200000000000090000000D0D0DFFA4000909D6
:1015300009090000FFFFFFFFFFFFFFFFFFFFA409F6
:101540005209090909090C0D0D0D0D0D00000900C6
:10155000000000020D000000000000090B0D00005B
:10156000000D0B0900000000020D00000000020D3C
:1015700009090909ADFF0D0D0D0D0B09000000FF54
:10158000A40000000009000004A6FF0000000909F3
:10159000090000000A00000000000D020000000029
:1015A00000000000005200000000020D00000009D1
:1015B00000000000000C0D0D0000090909090002DF
:1015C0000DFFFFFF09A4FFFFFFFF0D0B090909092C
:1015D000FFA4000000000A000000000000A4FF00BB
:1015E00000000D0B09000000090952FFA400FFFFD5
:1015F000FF520000FFFFFFFFFFFF09090909090A69
:10160000510B0D0D0D0D0D02000000000000090032
:10161000000000020D0D0D0D000000090909000079
:101620000004A6FF00000000020D00000000020DF3
:101630000D0D0D04A6FF00000000000A000000FFD1
:10164000A4000D0D0C0A000009ADFF000000FFA46E
:10165000090000000A00000000000D020000000068
:1016600000000000005200000000020D0000000910
:101670000B0D0000000D0B09000052FFFFFF0002E0
:101680000DFFFFFF5209090909090C0D0D0D0D0D84
:10169000FFA4000000000A000000000004A6FF00F4
:1016A0000000090909000000FFFFFFFFA400FFFF81
:1016B000FF52000009090909ADFF0D0D0D0D0B09C1
:1016C0005200000000000D020000000000000A0CA3
:1016D0000D0D00020D0A090900000009A4FF000019
:1016E0000004A6FF00000000020D00000000020D33
:1016F00000000000A4FF00000000000A0D0D0DFF17
:10170000A400090909090000FFFFFF000000FFA471
:10171000090000000A00000000000D0200000000A7
:1017200000000000005200000000020D000000094F
:10173000090900000004A6FF000052FFFFFF00029D
:101740000D0A0909510B0D0D0D0D0D0200000000D1
:10175000FFA4000000000A000000000009ADFF0027
:101760000000FFA409000000FFFFFFFFA40009091B
:10177000090900000D0D0D04A6FF0000000000097E
:101780005200000000000C0D0D0D0D0D00000909A8
:10179000090900020DFFFFFF00000009A4FF00007F
:1017A000000D0B0900000000020D00000000020DFA
:1017B00000000000A4FF0D0D0D0D0B09090952FFDB
:1017C000A400FFFFFF520000FFFFFF000000090917
:1017D000090000000A00000000000D0200000000E7
:1017E0000000000000000000000009520000000995
:1017F0005209000952000052000952000052000034
:1018000000095209000000000952000000000952BE
:101810000000000000005209000000000952090009
:101820000000095209000000095209000000095295
:1018300009000000520900000000520900000000E9
:1018400000000000A4FF000000FFAD090000000040
:10185000A4FF00000000095200000004A6FF0002DF
:101860000D00000000020D000000FFFFFF0000005F
:10187000FFA400000000520900000000FFA40000C7
:101880000000520900000000FFA6040D0200000045
:101890000000A4FF00000000A4FF00000000000002
:1018A00000000000000000000000095200000009D4
:1018B0005209000952000052000952000052000073
:1018C00000095209000000000952000000000952FE
:1018D0000000000000005209000000000952090049
:1018E00000000952090000000952090000000952D5
:1018F0000900000052090000000052090000000029
:1019000000000000A4FF000000FFAD09000000007F
:10191000A4FF00000000095200000004A6FF00021E
:101920000D00000000020D000000FFFFFF0000009E
:10193000FFA400000000520900000000FFA4000006
:101940000000520900000000FFA6040D0200000084
:101950000000A4FF00000000A4FF00000000000041
:101960000000000000000000000009520000000913
:1019700052090009520000520009520000520000B2
:10198000000952090000000009520000000009523D
:101990000000000000005209000000000952090088
:1019A0000000095209000000095209000000095214
:1019B0000900000052090000000052090000000068
:1019C00000000000A4FF000000FFAD0900000000BF
:1019D000A4FF00000000095200000004A6FF000060
:1019E000000D02000000000D020000A4FFFFA40093
:1019F000FFA400000000520900000000FFA4000046
:101A00000000520900000000FFA6040000000002D0
:101A10000D04A6FF00000000A4FF0000000000006D
:101A200000000000000000000000000000000000B6
:101A30000952000000095209000952000052000931
:101A40005200005200000009520900000000095233
:101A5000000000000000000000000000520900002B
:101A60000000095209000000095209000000095253
:101A7000090000000952090000005209000000009E
:101A800000000000A4FF000000FFAD0900000000FE
:101A9000A4FF00000000095200000004A6FF00009F
:101AA000000D02000000000D020000A4FFFFA400D2
:101AB000FFA400000000520900000000FFA4000085
:101AC0000000520900000000FFA4000000000C0DFF
:101AD0000D0D020000020DFFA400000000FFA40095
:101AE00000000000000000000000000000000000F6
:101AF0000952000000095209000952000052000971
:101B00005200005200000009520900000000095272
:101B1000000000000000000000000000520900006A
:101B20000000095209000000095209000000095292
:101B300009000000095209000000520900000000DD
:101B400000000000A4FF000000FFAD09000000003D
:101B5000A4FF00000000095200000000A4FF0000E4
:101B60000000020D00000000020D000000FFFFFF5A
:101B7000FFA400000000520900000000FFA40000C4
:101B80000000520900000000FFA4000000000D0248
:101B90000000000004A6FF00000000A4FF000000F9
:101BA0000000000000000000000000000000000035
:101BB00009520000000952090009520000520009B0
:101BC00052000052000000095209000000000952B2
:101BD00000000000000000000000000052090000AA
:101BE00000000952090000000952090000000952D2
:101BF000090000000952090000005209000000001D
:101C000000000000A4FF000000FFAD09000000007C
:101C1000A4FF00000000095200000000A4FF000023
:101C2000000C0D0D0000000C0D0D00000000A4FFC5
:101C3000FFA400000000520900000000FFA4000003
:101C40000000520900000000FFA4000000000D0287
:101C5000000000000D0200000000FFA400000000D2
:101C60000000000000000000000009520000000910
:101C700052090009520000520009520000520000AF
:101C8000000952090000000009520000000009523A
:101C90000000000000005209000000000952090085
:101CA0000000095209000000095209000000095211
:101CB0000900000052090000000052090000000065
:101CC00000000000A4FF000000FFAD0900000000BC
:101CD000A4FF00000000095200000000A4FF000063
:101CE000000C0D0D0000000C0D0D000000FFFFFFAB
:101CF000FFA400000000520900000000FFA4000043
:101D00000000520900000000FFA4000000000D02C6
:101D1000000000000D0200000000FFFFFF000000B7
:101D2000000000000000000000000952000000094F
:101D300052090009520000520009520000520000EE
:101D40000009520900000000095200000000095279
:101D500000000000000052090000000009520900C4
:101D60000000095209000000095209000000095250
:101D700009000000520900000000520900000000A4
:101D800000000000A4FF000000FFAD0900000000FB
:101D9000A4FF00000000095200000004A6FF00009C
:101DA000000D02000000000D020000A4FFFFA400CF
:101DB000FFA400000000520900000000FFA4000082
:101DC0000000520900000000FFA4000000000C0DFC
:101DD0000D0D020000020DFFA400000000FFA40092
:101DE000000000000000000000000952000000098F
:101DF00052090000000952090000000952090000C0
:101E000000095209000000000952000000000952B8
:101E10000000000000005209000000000952090003
:101E200000005200005209005200005209000952FD
:101E300009000000520900000000520900000000E3
:101E400000000000A4FF0000000009520000000094
:101E5000A4FF00000000095200020D04A6FFFFA429
:101E600000000000FFA400000000000000000000CF
:101E7000FFA40000000009ADFF000000FFA4000067
:101E80000000520900000000FFA60400000000004E
:101E9000000D02000000000D0200000000FFFFFF27
:101EA00000000000000000000000095200000009CE
:101EB00052090000000952090000000952090000FF
:101EC00000095209000000000952000000000952F8
:101ED0000000000000005209000000000952090043
:101EE000000052000052090052000052090009523D
:101EF0000900000052090000000052090000000023
:101F000000000000A4FF00000000095200000000D3
:101F1000A4FF00000000095200020D04A6FFFFA468
:101F200000000000FFA4000000000000000000000E
:101F3000FFA40000000009ADFF000000FFA40000A6
:101F40000000520900000000FFA60400000000008D
:101F5000000D02000000000D0200000000FFFFFF66
:101F6000000000000000000000000952000000090D
:101F7000520900000009520900000009520900003E
:101F80000009520900000000095200000000095237
:101F90000000000000005209000000000952090082
:101FA000000052000052090052000052090009527C
:101FB0000900000052090000000052090000000062
:101FC00000000000A4FF0000000009520000000013
:101FD000A4FF00000000095200000004A6FFFFA6B5
:101FE000040D0D0CFFA40000000000000000000024
:101FF000FFA40000000009ADFF000000FFA40000E6
:102000000000520900000000FFA6040000000002CA
:102010000D00000000020D00000000A4FFFFA4005E
:1020200000000000000000000000000000000000B0
:10203000095200000009520900000009520900007D
:10204000000952090000000952090000000009526D
:102050000000000000000000000000005209000025
:10206000000009520900000052000052090052000D
:102070000052090009520900000052090000000046
:1020800000000000A4FF0000000009520000000052
:10209000A4FF00000000095200000000A4FF00029D
:1020A0000D0D0D0C00A4FF0D020000A4FF000000A8
:1020B000FFA40000000009ADFF000000FFA4000025
:1020C0000000520900000000FFA60400000000020A
:1020D0000D00000000020D00000000A4FFFFA4009E
:1020E00000000000000000000000000000000000F0
:1020F00009520000000952090000000952090000BD
:1021000000095209000000095209000000000952AC
:102110000000000000000000000000005209000064
:10212000000009520900000052000052090052004C
:102130000052090009520900000052090000000085
:1021400000000000A4FF0000000009520000000091
:10215000A4FF00000000095200000000A4FF0000DE
:102160000000020D000000FFA604000000FFA40014
:10217000FFA40000000009ADFF000000FFA4000064
:102180000000520900000000FFA4000000000D0242
:10219000000000000D0200000000FFFFFF00000033
:1021A000000000000000000000000000000000002F
:1021B00009520000000952090000000952090000FC
:1021C00000095209000000095209000000000952EC
:1021D00000000000000000000000000052090000A4
:1021E000000009520900000052000052090052008C
:1021F00000520900095209000000520900000000C5
:1022000000000000A4FF00000000095200000000D0
:10221000A4FF00000000095200000000A4FF00001D
:102220000000020D00000000020D00000000A4FFED
:10223000FFA40000000009ADFF000000FFA40000A3
:102240000000520900000000FFA4000000000D0D76
:102250000C0000000D0D0C000000FFA400000000A9
:10226000000000000000000000000952000000090A
:10227000520900000009520900000009520900003B
:102280000009520900000000095200000000095234
:10229000000000000000520900000000095209007F
:1022A0000000520000520900520000520900095279
:1022B000090000005209000000005209000000005F
:1022C00000000000A4FF0000000009520000000010
:1022D000A4FF00000000095200000000A4FF00005D
:1022E0000000020D00000000020D000000FFFFFFD3
:1022F000FFA40000000009ADFF000000FFA40000E3
:102300000000520900000000FFA4000000000D0DB5
:102310000C0000000D0D0C000000FFFFFF0000008E
:102320000000000000000000000009520000000949
:10233000520900000009520900000009520900007A
:102340000009520900000000095200000000095273
:1023500000000000000052090000000009520900BE
:1023600000005200005209005200005209000952B8
:10237000090000005209000000005209000000009E
:1023800000000000A4FF000000000952000000004F
:10239000A4FF00000000095200000000A4FF00029A
:1023A0000D0D0D0C00A4FF0D020000A4FF000000A5
:1023B000FFA40000000009ADFF000000FFA4000022
:1023C0000000520900000000FFA604000000000207
:1023D0000D00000000020D00000000A4FFFFA4009B
:1023E0000000000000000000000009520000000989
:1023F00052090000000952090000000952090000BA
:1024000000095209000000000952000000000952B2
:1024100000000000000052090000000009520900FD
:1024200000005200005209005200005209000952F7
:1024300009000000520900000000520900000000DD
:1024400000000000A4FF000000000952000000008E
:10245000A4FF00000000095200000000A4FF0002D9
:102460000D0D0D0C00A4FF0D020000A4FF000000E4
:10247000FFA40000000009ADFF000000FFA4000061
:102480000000520900000000FFA604000000000246
:102490000D00000000020D00000000A4FFFFA400DA
:1024A00000000000000000000052090000000009C8
:1024B0005209000952000052000952000052000067
:1024C00000095209000000000952000000095209E9
:1024D000000000000000000952000000095209003D
:1024E0000000520000520900520000520900095237
:1024F0000900000052090000000009520900000014
:10250000000952005BFF00A4FF0000520000000021
:10251000A4FF00000000095200000004A6FF000014
:10252000000D02000000000D020000A4FFFFA40047
:10253000FF5B00520900520000FFA400FFA400004E
:102540000000520900000000FFA604000000000285
:102550000D00000000020D00000000A4FFFFA40019
:10256000000000000000000000000000000000006B
:10257000000000000000000000000000000000005B
:1025800000FFA40000A4FF00000000000000A4FF62
:10259000000000000000000000000000000000003B
:1025A000000000000000000000A4FF000000000088
:1025B00000000000FFA400000000000000FFA400D5
:1025C000000000000000000000FFA40000A4FF00C5
:1025D000000000000000A4FF000000000000000058
:1025E00000000000000000000000000000000000EB
:1025F000FFA40000000000000000000000A4FF0095
:102600000000FFA400000000000000000000000027
:1026100000000000000000000000000000000000BA
:10262000000000000000FFA400FFA4000000000064
:102630000000000000FFA40000A4FF000000000054
:1026400000000000FFA400000000000000000000E7
:10265000FFA400000000000000FFA4000000000034
:102660000000FFA400FFA40000000000000000A480
:10267000FF00000000000000A4FF000000000000B8
:10268000000000000000FFA40000000000000000A7
:10269000000000A4FF00000000000000A4FFFFA451
:1026A00000000000000000FFA40000000000000087
:1026B000000000000000000000FFA4000000000077
:1026C0000000FFA40000A4FF0000000000000000C4
:1026D00000FFA40000000000000000000000000057
:1026E00000000000020D00A4FF00A4FF0000000D88
:1026F0000200000000FFA400000000000909000023
:10270000000000000D0200090900FFA40000000005
:102710000D020000000000000000000000020D009B
:10272000A4FF09A4FF0000000000000D020000004B
:1027300000FFA40000090900020D00000000A4FF32
:102740000D0200000000FFA40009090000000000C5
:10275000000000A4FF0009090000000D02000000B5
:1027600000FFA40000A4FF00020D00000000A4FF71
:1027700000000000090900000000A4FF0009090989
:102780000900000000FFA4000D0B0900000000007C
:102790000000A4FF090900000000FFA400000000E1
:1027A00000000000020D00000000A4FF0000000D6A
:1027B0000200000000FFA40000020D00090900A4AF
:1027C000FF0000000D020009A4FFFFA60D0009098B
:1027D0000D0200000000FFA40000000000020D0038
:1027E000000009A4FF0000000000000D0200FFA48B
:1027F00000FFA4000D0B0900020D09090009A4FF48
:102800000D020000A4FFFFA40009090000020D0D45
:10281000020000A4FF0009090000000DA6FF00004F
:1028200000FFA40000000000020D00000000A4FF53
:1028300000020D0D0B0909090000A4FF00A4FF0907
:102840000900090900FFA4000009090000000DA605
:10285000FF000000090900000000FFA400000000C4
:102860000000000000000000005209000000000904
:1028700052090009520000520009520000520000A3
:102880000009520900000000095200000009520925
:102890000000000000000009520000000952090079
:1028A0000000520000520900520000520900095273
:1028B0000900000052090000000009520900000050
:1028C000000952005BFF00A4FF000052000000005E
:1028D000A4FF00000000095200000004A6FF000051
:1028E000000D02000000000D020000A4FFFFA40084
:1028F000FF5B00520900520000FFA400FFA400008B
:102900000000520900000000FFA6040000000002C1
:102910000D00000000020D00000000A4FFFFA40055
:102920000000000000000000005209000000000943
:1029300052090009520000520009520000520000E2
:102940000009520900000000095200000009520964
:1029500000000000000000095200000009520900B8
:1029600000005200005209005200005209000952B2
:10297000090000005209000000000952090000008F
:10298000000952005BFF00A4FF000052000000009D
:10299000A4FF00000000095200000004A6FF000090
:1029A000000D02000000000D020000A4FFFFA400C3
:1029B000FF5B00520900520000FFA400FFA40000CA
:1029C0000000520900000000FFA604000000000201
:1029D0000D00000000020D00000000A4FFFFA40095
:1029E0000000000000000000005209000000000983
:1029F0005209000952000052000952000052000022
:102A000000095209000000000952000000095209A3
:102A100000000000000000095200000009520900F7
:102A200000005200005209005200005209000952F1
:102A300009000000520900000000095209000000CE
:102A4000000952005BFF00A4FF00005200000000DC
:102A5000A4FF00000000095200000004A6FF0000CF
:102A6000000D02000000000D020000A4FFFFA40002
:102A7000FF5B00520900520000FFA400FFA4000009
:102A80000000520900000000FFA604000000000240
:102A90000D00000000020D00000000A4FFFFA400D4
:102AA00000000000000000000052090000000009C2
:102AB0005209000952000052000952000052000061
:102AC00000095209000000000952000000095209E3
:102AD0000000000000000009520000000952090037
:102AE0000000520000520900520000520900095231
:102AF000090000005209000000000952090000000E
:102B0000000952005BFF00A4FF000052000000001B
:102B1000A4FF00000000095200000004A6FF00000E
:102B2000000D02000000000D020000A4FFFFA40041
:102B3000FF5B00520900520000FFA400FFA4000048
:102B40000000520900000000FFA60400000000027F
:102B50000D00000000020D00000000A4FFFFA40013
:102B60000000000000000000005209000000000901
:102B700052090009520000520009520000520000A0
:102B80000009520900000000095200000009520922
:102B90000000000000000009520000000952090076
:102BA0000000520000520900520000520900095270
:102BB000090000005209000000000952090000004D
:102BC000000952005BFF000000FFAD09000000009B
:102BD000A4FF00000000095200000004A6FF00004E
:102BE000000D020000A4FFFFA40000000000000090
:102BF000FF5B00520900520000FFA400FFA4000088
:102C00000000520900000000FFA6040000000002BE
:102C10000D00000000020D00000000A4FFFFA40052
:102C20000000000000000000005209000000000940
:102C300052090009520000520009520000520000DF
:102C40000009520900000000095200000009520961
:102C500000000000000000095200000009520900B5
:102C600000005200005209005200005209000952AF
:102C7000090000005209000000000952090000008C
:102C8000000952005BFF000000FFAD0900000000DA
:102C9000A4FF00000000095200000004A6FF00008D
:102CA000000D020000A4FFFFA400000000000000CF
:102CB000FF5B00520900520000FFA400FFA40000C7
:102CC0000000520900000000FFA6040000000002FE
:102CD0000D00000000020D00000000A4FFFFA40092
:102CE0000000000000000000005209000000000980
:102CF000520900095200005200095200005200001F
:102D000000095209000000000952000000095209A0
:102D100000000000000000095200000009520900F4
:102D200000005200005209005200005209000952EE
:102D300009000000520900000000095209000000CB
:102D4000000952005BFF00A4FF00005200000000D9
:102D5000A4FF00000000095200000004A6FF0000CC
:102D6000000D02000000000D020000A4FFFFA400FF
:102D7000FF5B00520900520000FFA400FFA4000006
:102D80000000520900000000FFA60400000000023D
:102D90000D00000000020D00000000A4FFFFA400D1
:102DA00000000000000000000052090000000009BF
:102DB000520900095200005200095200005200005E
:102DC00000095209000000000952000000095209E0
:102DD0000000000000000009520000000952090034
:102DE000000052000052090052000052090009522E
:102DF000090000005209000000000952090000000B
:102E0000000952005BFF00A4FF0000520000000018
:102E1000A4FF00000000095200000004A6FF00000B
:102E2000000D02000000000D020000A4FFFFA4003E
:102E3000FF5B00520900520000FFA400FFA4000045
:102E40000000520900000000FFA60400000000027C
:102E50000D00000000020D00000000A4FFFFA40010
:102E600000000000000000000052090000000009FE
:102E7000520900095200005200095200005200009D
:102E8000000952090000000009520000000952091F
:102E90000000000000000009520000000952090073
:102EA000000052000052090052000052090009526D
:102EB000090000005209000000000952090000004A
:102EC000000952005BFF000000FFAD090000000098
:102ED000A4FF00000000095200000004A6FF00004B
:102EE000000D020000A4FFFFA4000000000000008D
:102EF000FF5B00520900520000FFA400FFA4000085
:102F00000000520900000000FFA6040000000002BB
:102F10000D00000000020D00000000A4FFFFA4004F
:102F2000000000000000000000520900000000093D
:102F300052090009520000520009520000520000DC
:102F4000000952090000000009520000000952095E
:102F500000000000000000095200000009520900B2
:102F600000005200005209005200005209000952AC
:102F70000900000052090000000009520900000089
:102F8000000952005BFF000000FFAD0900000000D7
:102F9000A4FF00000000095200000004A6FF00008A
:102FA000000D020000A4FFFFA400000000000000CC
:102FB000FF5B00520900520000FFA400FFA40000C4
:102FC0000000520900000000FFA6040000000002FB
:102FD0000D00000000020D00000000A4FFFFA4008F
:102FE000000000000000000000520900000000097D
:102FF000520900095200005200095200005200001C
:10300000000952090000000009520000000952099D
:1030100000000000000000095200000009520900F1
:1030200000005200005209005200005209000952EB
:1030300009000000520900000000095209000000C8
:10304000000952005BFF00A4FF00005200000000D6
:10305000A4FF00000000095200000004A6FF0000C9
:10306000000D02000000000D020000A4FFFFA400FC
:10307000FF5B00520900520000FFA400FFA4000003
:103080000000520900000000FFA60400000000023A
:103090000D00000000020D00000000A4FFFFA400CE
:1030A00000000000000000000052090000000009BC
:1030B000520900095200005200095200005200005B
:1030C00000095209000000000952000000095209DD
:1030D0000000000000000009520000000952090031
:1030E000000052000052090052000052090009522B
:1030F0000900000052090000000009520900000008
:10310000000952005BFF00A4FF0000520000000015
:10311000A4FF00000000095200000004A6FF000008
:10312000000D02000000000D020000A4FFFFA4003B
:10313000FF5B00520900520000FFA400FFA4000042
:103140000000520900000000FFA604000000000279
:103150000D00000000020D00000000A4FFFFA4000D
:10316000FFA400000000520900000000FFFFFF0064
:103170000000FFAD09000000090952FFA4000D0D79
:103180000C52080000000000A4FF000000000852DC
:1031900000000000095200000000020D00000009BC
:1031A000ADFF00000004A6FF000952095209000209
:1031B0000D0D0D0C5200000000000D02000000007B
:1031C0000D0D0D04A6FF09090909490AFFFFFFFFBC
:1031D000A400FFFFFF52000009ADFF0000000D0B2F
:1031E000490000005209000000000D02000000002C
:1031F000520B0D0D0D0C0D0B51095209000052FF21
:10320000FFFF00020DFFFFFF000000095209000050
:10321000000C0D0C00000000020D00000000020D6B
:10322000FFA400000000520900000000FFFFFF00A3
:103230000000FFAD09000000090952FFA4000D0DB8
:103240000C52080000000000A4FF0000000008521B
:1032500000000000095200000000020D00000009FB
:10326000ADFF00000004A6FF000952095209000248
:103270000D0D0D0C5200000000000D0200000000BA
:103280000D0D0D04A6FF09090909490AFFFFFFFFFB
:10329000A400FFFFFF52000009ADFF0000000D0B6E
:1032A000490000005209000000000D02000000006B
:1032B000520B0D0D0D0C0D0B51095209000052FF60
:1032C000FFFF00020DFFFFFF000000095209000090
:1032D000000C0D0C00000000020D00000000020DAB
:1032E00000A4FF00000000A4FF0000000000520046
:1032F0000000000052000000000052FFA400000285
:103300000D52080000000000A4FF00000000085259
:103310000000005209000000005209000000000DEA
:1033200002000000000D02000009525209000002D4
:103330000D0D02005200000000000D020000000010
:1033400000020D04A6FF00005209490A005BFFFFBE
:10335000A400005BFF52000000A4FF000000000872
:103360005200000000085200000000020D000000A2
:10337000520B0D0D02000D0B51520900000052FFBF
:10338000A40000020DFFA40000000052090000008C
:10339000000D02000000005209000000000D0200B4
:1033A000000000FFA400000000520900000000FF20
:1033B000A4000000005209000000005209000000B3
:1033C000000D020000000000A4FF000000000852F1
:1033D00000095200000000020D0000000009520028
:1033E000000000020D000000000952000000000271
:1033F0000D0000005200000000000D02000000005F
:1034000000000000A4FF000000000852000000526D
:1034100009000000000D0200000000520900000039
:10342000000D02000000005209000000000D020023
:103430005200000000000D020000000000095200D0
:10344000000000020D000000000952000000000210
:103450000D00000000095200000000020D000000F5
:1034600000A4FF00000000A4FF00000000005200C4
:103470000000000052000000000052FFA400000203
:103480000D52080000000000A4FF000000000852D8
:103490000000005209000000005209000000000D69
:1034A00002000000000D0200000952520900000253
:1034B0000D0D02005200000000000D02000000008F
:1034C00000020D04A6FF00005209490A005BFFFF3D
:1034D000A400005BFF52000000A4FF0000000008F1
:1034E0005200000000085200000000020D00000021
:1034F000520B0D0D02000D0B51520900000052FF3E
:10350000A40000020DFFA40000000052090000000A
:10351000000D02000000005209000000000D020032
:10352000FFA400000000520900000000FFFFFF00A0
:103530000000FFAD09000000090952FFA4000D0DB5
:103540000C52080000000000A4FF00000000085218
:1035500000000000095200000000020D00000009F8
:10356000ADFF00000004A6FF000952095209000245
:103570000D0D0D0C5200000000000D0200000000B7
:103580000D0D0D04A6FF09090909490AFFFFFFFFF8
:10359000A400FFFFFF52000009ADFF0000000D0B6B
:1035A000490000005209000000000D020000000068
:1035B000520B0D0D0D0C0D0B51095209000052FF5D
:1035C000FFFF00020DFFFFFF00000009520900008D
:1035D000000C0D0C00000000020D00000000020DA8
:1035E000FFA400000000520900000000FFFFFF00E0
:1035F0000000FFAD09000000090952FFA4000D0DF5
:103600000C52080000000000A4FF00000000085257
:1036100000000000095200000000020D0000000937
:10362000ADFF00000004A6FF000952095209000284
:103630000D0D0D0C5200000000000D0200000000F6
:103640000D0D0D04A6FF09090909490AFFFFFFFF37
:10365000A400FFFFFF52000009ADFF0000000D0BAA
:10366000490000005209000000000D0200000000A7
:10367000520B0D0D0D0C0D0B51095209000052FF9C
:10368000FFFF00020DFFFFFF0000000952090000CC
:10369000000C0D0C00000000020D00000000020DE7
:1036A00052090909090952090909090952000000CA
:1036B00000005200000000005200000909095200F9
:1036C0000009090952000009ADFF52000009ADFFD1
:1036D00009090909095209090909095200000000EC
:1036E00000520000000000520909090000520909B7
:1036F00009000052FFAD09000052FFAD0900005261
:1037000052000009ADFF52000009ADFF5200000950
:103710000909520000090909520000000000520086
:10372000000000005209090909095209090909099B
:10373000FFAD09000052FFAD090000520909090060
:103740000052090909000052000000000052000068
:103750000000005209090909095209090909095219
:1037600000000000000000000000000000005209FE
:103770000909000052090909000052FFFFFF00007B
:1037800052FFFFFF000052FFAD09000052FFAD09DC
:1037900000000000000000000000000009090952BC
:1037A0000000090909520000FFFFFF520000FFFF5F
:1037B000FF52000009ADFF52000009ADFF520000AA
:1037C000000052FFAD09000052FFAD09000052FF9A
:1037D000FFFF000052FFFFFF00005209090900002F
:1037E000520909090000000000000000000000006C
:1037F00009ADFF52000009ADFF520000FFFFFF526C
:103800000000FFFFFF5200000909095200000909EA
:10381000095200000000000000000000000000004D
:1038200052090909090952090909090909ADFFFFE6
:10383000FFFF09ADFFFFFFFF09ADFF52090909AD09
:10384000FF52090909ADFF52000009ADFF52000007
:10385000090909090952090909090952FFFFFFFF6E
:10386000AD09FFFFFFFFAD09090952FFAD090909C5
:1038700052FFAD09000052FFAD09000052FFAD0933
:1038800009ADFF52000009ADFF52000009ADFF5223
:10389000090909ADFF52090909ADFFFFFFFF09AD95
:1038A000FFFFFFFF5209090909095209090909091E
:1038B000000052FFAD09000052FFAD09090952FF97
:1038C000AD09090952FFAD09FFFFFFFFAD09FFFF79
:1038D000FFFFAD0909090909095209090909095236
:1038E000FFFFFFFFFFFFFFFFFFFFFFFFFFAD090926
:1038F0000909FFAD09090909FFAD09000000FFAD85
:1039000009000000FFAD09000052FFAD09000052A0
:10391000FFFFFFFFFFFFFFFFFFFFFFFF090909098F
:10392000ADFF09090909ADFF00000009ADFF000066
:103930000009ADFF52000009ADFF52000009ADFFC4
:10394000FFAD09000052FFAD09000052FFAD0900B4
:103950000000FFAD09000000FFAD09090909FFAD36
:1039600009090909FFFFFFFFFFFFFFFFFFFFFFFF3F
:1039700052000009ADFF52000009ADFF0000000930
:10398000ADFF00000009ADFF09090909ADFF0909F4
:103990000909ADFFFFFFFFFFFFFFFFFFFFFFFFFF75
:1039A00052090909090952090909090952000000C7
:1039B00000005200000000005200000909095200F6
:1039C0000009090952000009ADFF52000009ADFFCE
:1039D00009090909095209090909095200000000E9
:1039E00000520000000000520909090000520909B4
:1039F00009000052FFAD09000052FFAD090000525E
:103A000052000009ADFF52000009ADFF520000094D
:103A10000909520000090909520000000000520083
:103A20000000000052090909090952090909090998
:103A3000FFAD09000052FFAD09000052090909005D
:103A40000052090909000052000000000052000065
:103A50000000005209090909095209090909095216
:103A600000000000000000000000000000005209FB
:103A70000909000052090909000052FFFFFF000078
:103A800052FFFFFF000052FFAD09000052FFAD09D9
:103A900000000000000000000000000009090952B9
:103AA0000000090909520000FFFFFF520000FFFF5C
:103AB000FF52000009ADFF52000009ADFF520000A7
:103AC000000052FFAD09000052FFAD09000052FF97
:103AD000FFFF000052FFFFFF00005209090900002C
:103AE0005209090900000000000000000000000069
:103AF00009ADFF52000009ADFF520000FFFFFF5269
:103B00000000FFFFFF5200000909095200000909E7
:103B1000095200000000000000000000000000004A
:103B200052090909090952090909090909ADFFFFE3
:103B3000FFFF09ADFFFFFFFF09ADFF52090909AD06
:103B4000FF52090909ADFF52000009ADFF52000004
:103B5000090909090952090909090952FFFFFFFF6B
:103B6000AD09FFFFFFFFAD09090952FFAD090909C2
:103B700052FFAD09000052FFAD09000052FFAD0930
:103B800009ADFF52000009ADFF52000009ADFF5220
:103B9000090909ADFF52090909ADFFFFFFFF09AD92
:103BA000FFFFFFFF5209090909095209090909091B
:103BB000000052FFAD09000052FFAD09090952FF94
:103BC000AD09090952FFAD09FFFFFFFFAD09FFFF76
:103BD000FFFFAD0909090909095209090909095233
:103BE000FFFFFFFFFFFFFFFFFFFFFFFFFFAD090923
:103BF0000909FFAD09090909FFAD09000000FFAD82
:103C000009000000FFAD09000052FFAD090000529D
:103C1000FFFFFFFFFFFFFFFFFFFFFFFF090909098C
:103C2000ADFF09090909ADFF00000009ADFF000063
:103C30000009ADFF52000009ADFF52000009ADFFC1
:103C4000FFAD09000052FFAD09000052FFAD0900B1
:103C50000000FFAD09000000FFAD09090909FFAD33
:103C600009090909FFFFFFFFFFFFFFFFFFFFFFFF3C
:103C700052000009ADFF52000009ADFF000000092D
:103C8000ADFF00000009ADFF09090909ADFF0909F1
:103C90000909ADFFFFFFFFFFFFFFFFFFFFFFFFFF72
:103CA000FFFFFFFFFFFFFFFF0909FFFFFFFF0909FC
:103CB0000909FFFF00000000FFFFFFFF0000FFFFFA
:103CC000FFFF0000090909090000000000000000D2
:103CD000FFFFFFFFFFFFFFFFFFFF09090909FFFFCC
:103CE00009090000FFFF0000FFFFFFFFFFFFFFFFCC
:103CF000FFFFFFFFFFFF09090909FFFF00000000A8
:103D0000FFFFFFFFFFFFFFFF0909FFFFFFFF09099B
:103D10000909FFFF00000000FFFFFFFF0000FFFF99
:103D2000FFFF000009090909000000000000000071
:103D3000FFFFFFFFFFFFFFFFFFFF09090909FFFF6B
:103D400009090000FFFF0000FFFFFFFFFFFFFFFF6B
:103D5000FFFFFFFFFFFF09090909FFFF0000000047
:103D6000FFFFFFFF0000FFFFFFFF00000909090937
:103D700000000000000000000000FFFFFFFF000047
:103D8000FFFFFFFF0000FFFF09090000FFFF000029
:103D9000FFFFFFFFFFFFFFFFFFFFFFFFFFFF09091F
:103DA0000909FFFF00000000FFFFFFFFFFFFFFFF0B
:103DB000FFFF09090909FFFF09090000FFFF0000D3
:103DC000FFFFFFFF0000FFFFFFFF000009090909D7
:103DD00000000000000000000000FFFFFFFF0000E7
:103DE000FFFFFFFF0000FFFF09090000FFFF0000C9
:103DF000FFFFFFFFFFFFFFFFFFFFFFFFFFFF0909BF
:103E00000909FFFF00000000FFFFFFFFFFFFFFFFAA
:103E1000FFFF09090909FFFF09090000FFFF000072
:103E20000000FFFFFFFF0000FFFFFFFF0000FFFF9C
:103E300009090000FFFF0000FFFFFFFFFFFFFFFF7A
:103E4000FFFFFFFF09090909FFFF00000000FFFF56
:103E5000FFFF0000FFFFFFFF000009090909000044
:103E60000909000000000000FFFFFFFFFFFF090934
:103E7000FFFFFFFF09090909FFFF00000000FFFF26
:103E80000000FFFFFFFF0000FFFFFFFF0000FFFF3C
:103E900009090000FFFF0000FFFFFFFFFFFFFFFF1A
:103EA000FFFFFFFF09090909FFFF00000000FFFFF6
:103EB000FFFF0000FFFFFFFF0000090909090000E4
:103EC0000909000000000000FFFFFFFFFFFF0909D4
:103ED000FFFFFFFF09090909FFFF00000000FFFFC6
:103EE000FFFFFFFF0000FFFFFFFF0000FFFF0909CA
:103EF0000000FFFF000000000000FFFFFFFF0000C8
:103F00000909FFFF0000090909090000000000007D
:103F1000FFFFFFFFFFFF0909FFFFFFFF0909FFFF89
:103F200009090000FFFF0000FFFF0000FFFFFFFF87
:103F300000000909FFFF00000909FFFF0000000061
:103F4000FFFFFFFF0000FFFFFFFF0000FFFF090969
:103F50000000FFFF000000000000FFFFFFFF000067
:103F60000909FFFF0000090909090000000000001D
:103F7000FFFFFFFFFFFF0909FFFFFFFF0909FFFF29
:103F800009090000FFFF0000FFFF0000FFFFFFFF27
:103F900000000909FFFF00000909FFFF0000000001
:103FA000FFFFFFFFFFFFFFFF0909FFFFFFFF0909F9
:103FB0000909FFFF00000000FFFFFFFF0000FFFFF7
:103FC000FFFF0000090909090000000000000000CF
:103FD000FFFFFFFFFFFFFFFFFFFF09090909FFFFC9
:103FE00009090000FFFF0000FFFFFFFFFFFFFFFFC9
:103FF000FFFFFFFFFFFF09090909FFFF00000000A5
:10400000FFFFFFFFFFFFFFFF0909FFFFFFFF090998
:104010000909FFFF00000000FFFFFFFF0000FFFF96
:10402000FFFF00000909090900000000000000006E
:10403000FFFFFFFFFFFFFFFFFFFF09090909FFFF68
:1040400009090000FFFF0000FFFFFFFFFFFFFFFF68
:10405000FFFFFFFFFFFF09090909FFFF0000000044
:10406000FFFFFFFF0000FFFFFFFF00000909090934
:1040700000000000000000000000FFFFFFFF000044
:10408000FFFFFFFF0000FFFF09090000FFFF000026
:10409000FFFFFFFFFFFFFFFFFFFFFFFFFFFF09091C
:1040A0000909FFFF00000000FFFFFFFFFFFFFFFF08
:1040B000FFFF09090909FFFF09090000FFFF0000D0
:1040C000FFFFFFFF0000FFFFFFFF000009090909D4
:1040D00000000000000000000000FFFFFFFF0000E4
:1040E000FFFFFFFF0000FFFF09090000FFFF0000C6
:1040F000FFFFFFFFFFFFFFFFFFFFFFFFFFFF0909BC
:104100000909FFFF00000000FFFFFFFFFFFFFFFFA7
:10411000FFFF09090909FFFF09090000FFFF00006F
:104120000000FFFFFFFF0000FFFFFFFF0000FFFF99
:1041300009090000FFFF0000FFFFFFFFFFFFFFFF77
:10414000FFFFFFFF09090909FFFF00000000FFFF53
:10415000FFFF0000FFFFFFFF000009090909000041
:104160000909000000000000FFFFFFFFFFFF090931
:10417000FFFFFFFF09090909FFFF00000000FFFF23
:104180000000FFFFFFFF0000FFFFFFFF0000FFFF39
:1041900009090000FFFF0000FFFFFFFFFFFFFFFF17
:1041A000FFFFFFFF09090909FFFF00000000FFFFF3
:1041B000FFFF0000FFFFFFFF0000090909090000E1
:1041C0000909000000000000FFFFFFFFFFFF0909D1
:1041D000FFFFFFFF09090909FFFF00000000FFFFC3
:1041E000FFFFFFFF0000FFFFFFFF0000FFFF0909C7
:1041F0000000FFFF000000000000FFFFFFFF0000C5
:104200000909FFFF0000090909090000000000007A
:10421000FFFFFFFFFFFF0909FFFFFFFF0909FFFF86
:1042200009090000FFFF0000FFFF0000FFFFFFFF84
:1042300000000909FFFF00000909FFFF000000005E
:10424000FFFFFFFF0000FFFFFFFF0000FFFF090966
:104250000000FFFF000000000000FFFFFFFF000064
:104260000909FFFF0000090909090000000000001A
:10427000FFFFFFFFFFFF0909FFFFFFFF0909FFFF26
:1042800009090000FFFF0000FFFF0000FFFFFFFF24
:1042900000000909FFFF00000909FFFF00000000FE
:1042A0003838383838383838383838384A21383893
:1042B0003838000152383838000152383838000197
:1042C000523838384A213838383838383838383859
:1042D0004A21383838383838383838383838383863
:1042E000383838383838214A38383838294A383850
:1042F0003838214A38383838383838383838383843
:104300003838383838384A21383838380001523887
:1043100038380001523838380001523838384A21CC
:10432000383838383838383838383838383838380D
:1043300038383838383838383838214A38383852E8
:104340000100383838520100383838520100383806
:104350003838214A383838383838383838383838E2
:1043600038383838294A38383838383838383838CA
:1043700038384A21383838380001523838384A211C
:1043800038383838383838383838383838383838AD
:104390000001523838384A213838383838383838F7
:1043A000214A38383852010038214A520000383842
:1043B0003852010038383838214A383838383838D7
:1043C0003838383838383838383838384A2938386A
:1043D00038380001523838384A29383838383838AF
:1043E0003838383838383838383838383838294A4A
:1043F000383838383838383838383838383838383D
:10440000214A38383852010038383838214A38388B
:10441000383838384A213838383800015238383876
:1044200038383852010038383838294A383838385E
:1044300038383838383838384A29383838383838F9
:1044400038383838383838383838383838383838EC
:104450000000004A29380001523838384A213838DB
:10446000383838383838214A383838520100383826
:104470003838214A383838383838383838383838C1
:1044800038383838383838383838383838383838AC
:10449000383838383838383838383838383838389C
:1044A0003838383838383838294A383838520100DE
:1044B000383838383838383838383838383838387C
:1044C00038383838383838383838383838384A2171
:1044D000383838380001523838380000004A293856
:1044E00038383838294A3838383838383838383849
:1044F00038384A21383838380001523838384A219B
:10450000383838383838383838383838383838382B
:104510000001523838384A21383838383838383875
:10452000383838383838383838383838214A383810
:1045300038383838383838383838383838383838FB
:10454000383838383838383838383838114A113827
:104550003838000152383838114A1138383838386C
:104560003838383838383838383838383838294AC8
:1045700038383838383838383838383838383838BB
:10458000214A38383852010038383838214A38380A
:10459000383838384A2138383838000152383838F5
:1045A0003838383838383838383838384A21383890
:1045B0003838000152383838000152383838000194
:1045C000523838384A213838383838383838383856
:1045D0004A21383838383838383838383838383860
:1045E000383838383838214A38383838294A38384D
:1045F0003838214A38383838383838383838383840
:104600003838383838384A21383838380001523884
:1046100038380001523838380001523838384A21C9
:10462000383838383838383838383838383838380A
:1046300038383838383838383838214A38383852E5
:104640000100383838520100383838520100383803
:104650003838214A383838383838383838383838DF
:1046600038383838294A38383838383838383838C7
:1046700038384A21383838380001523838384A2119
:1046800038383838383838383838383838383838AA
:104690000001523838384A213838383838383838F4
:1046A000214A38383852010038214A52000038383F
:1046B0003852010038383838214A383838383838D4
:1046C0003838383838383838383838384A29383867
:1046D00038380001523838384A29383838383838AC
:1046E0003838383838383838383838383838294A47
:1046F000383838383838383838383838383838383A
:10470000214A38383852010038383838214A383888
:10471000383838384A213838383800015238383873
:1047200038383852010038383838294A383838385B
:1047300038383838383838384A29383838383838F6
:1047400038383838383838383838383838383838E9
:104750000000004A29380001523838384A213838D8
:10476000383838383838214A383838520100383823
:104770003838214A383838383838383838383838BE
:1047800038383838383838383838383838383838A9
:104790003838383838383838383838383838383899
:1047A0003838383838383838294A383838520100DB
:1047B0003838383838383838383838383838383879
:1047C00038383838383838383838383838384A216E
:1047D000383838380001523838380000004A293853
:1047E00038383838294A3838383838383838383846
:1047F00038384A21383838380001523838384A2198
:104800003838383838383838383838383838383828
:104810000001523838384A21383838383838383872
:10482000383838383838383838383838214A38380D
:1048300038383838383838383838383838383838F8
:10484000383838383838383838383838114A113824
:104850003838000152383838114A11383838383869
:104860003838383838383838383838383838294AC5
:1048700038383838383838383838383838383838B8
:10488000214A38383852010038383838214A383807
:10489000383838384A2138383838000152383838F2
:1048A000000000FFFFFF00A4FF5BADFFFFAE1DFF98
:1048B000AD5B52ADFF1D5C5B5B5B5B5A5C1D5A5C84
:1048C0001D5B5B5B5B5B5B1C1D1C5B5B5B5B5B5B32
:1048D000FFA4000000001DAEFF000000FFFFFFFF6F
:1048E0005B001CAEFFFFFFFF52ADFFFFFFFF5A5CF6
:1048F0001D52ADFF5B5A5BFFFFFF5A5C1D52ADFFBF
:104900005B0900525B5B5B5B5200095B5B09005219
:104910005B5B5B5B5200095B5B5B5B5B09000009F7
:104920005B5B5B5B0000005B090000000000095B53
:104930005B5B5B5A5C1D5A5C1D5B5C1D5B5B5B5B80
:104940005B5B5B5B5B5B5B5B525B5B5B09005B5B6D
:104950005B5B09001C5C520000005B09000000006A
:1049600000000000005200000000020D00000009DD
:10497000A4FF00000004A6FF0000090909090002C5
:104980000D0D0D0D0900000000000D0200000000DB
:10499000FFA4000000000A0000000000FFFFFF006D
:1049A0000000FFA409000000090952FFA4000D0D3A
:1049B0000C0A000000000000A4FF00000000000A34
:1049C000090B0D0D0D0D0D0B09090909000052FF12
:1049D000FFFF00020DFFFFFF0000000909090000B2
:1049E000000C0D0D00000000020D00000000020D83
:1049F0000D0D0D04A6FF09090909090AFFFFFFFFB4
:104A0000A400FFFFFF52000009ADFF0000000D0BE6
:104A1000090000000A00000000000D020000000074
:104A20000000000000000000000000000000000086
:104A30000000000000000000000000000000000076
:104A400000FFA40000A4FF00000000000000A4FF7D
:104A50000000000000000000000000000000000056
:104A6000000000000000000000A4FF0000000000A3
:104A700000000000FFA400000000000000FFA400F0
:104A8000000000000000000000FFA40000A4FF00E0
:104A9000000000000000A4FF000000000000000073
:104AA0000000000000000000000000000000000006
:104AB000FFA40000000000000000000000A4FF00B0
:104AC0000000FFA400000000000000000000000043
:104AD00000000000000000000000000000000000D6
:104AE00000000000000000000000000000A4FF0023
:104AF000000000000000A4FF00A4FF00020D00025F
:104B00000D090900000909000000FFA60D000909B0
:104B1000000000000000000000000000FFA400FFF3
:104B2000A40000090900000000020DFFA40000001D
:104B3000000D0200090B0D09090000000009090021
:104B4000000000000000FFA60D090900000909008F
:104B500009090000000D0B09FFA4000D0200000070
:104B60000000A4FF00A4FF000000000000000000FF
:104B70000D0D0D0000000D0200FFA40000020D004D
:104B800000000D02000D02000D0200FFA400FFA4B2
:104B90000000000000000000000000000000000015
:104BA0000000000000000000000000000000000005
:104BB000000000000000000000000000A4FF00A4AE
:104BC000FF0D020000020D00000000A4FF00020D16
:104BD00000000000000000000000000000000000D5
:104BE000000000A4FF00000000020D000000000013
:104BF00000FFA4000DA6FF0D02000000000D020042
:104C000000000000000000A4FF0D020000020D00E3
:104C1000020D000000FFA60D000000FFA400000030
:104C20000000000000000000000000000000000084
:104C30000DA6FF0000000D020000000000020D00A4
:104C400000000D0200FFA400FFA40000000000000F
:104C50000000000000000000000000000000000054
:104C60000000000000000000000000000000000044
:104C70000000000000000000000000000000000034
:104C800000FFA40000A4FF00000000000000A4FF3B
:104C90000000000000000000000000000000000014
:104CA000000000000000000000A4FF000000000061
:104CB00000000000FFA400000000000000FFA400AE
:104CC000000000000000000000FFA40000A4FF009E
:104CD000000000000000A4FF000000000000000031
:104CE00000000000000000000000000000000000C4
:104CF000FFA40000000000000000000000A4FF006E
:104D00000000FFA400000000000000000000000000
:104D10000000000000000000000000000000000093
:104D20000000000000000000000000000000000083
:104D30000000000000000000000000000000000073
:104D400000FFA40000A4FF00000000000000A4FF7A
:104D50000000000000000000000000000000000053
:104D6000000000000000000000A4FF0000000000A0
:104D700000000000FFA400000000000000FFA400ED
:104D8000000000000000000000FFA40000A4FF00DD
:104D9000000000000000A4FF000000000000000070
:104DA0000000000000000000000000000000000003
:104DB000FFA40000000000000000000000A4FF00AD
:104DC0000000FFA400000000000000000000000040
:104DD00000000000000000000000000000000000D3
:104DE000000000000000FFA400FFA400000000007D
:104DF0000000000000FFA40000A4FF00000000006D
:104E000000000000FFA400000000000000000000FF
:104E1000FFA400000000000000FFA400000000004C
:104E20000000FFA400FFA40000000000000000A498
:104E3000FF00000000000000A4FF000000000000D0
:104E4000000000000000FFA40000000000000000BF
:104E5000000000A4FF00000000000000A4FFFFA469
:104E600000000000000000FFA4000000000000009F
:104E7000000000000000000000FFA400000000008F
:104E80000000FFA40000A4FF0000000000000000DC
:104E900000FFA4000000000000000000000000006F
:104EA00000000000020D00A4FF00A4FF0000000DA0
:104EB0000200000000FFA40000000000090900003B
:104EC000000000000D0200090900FFA4000000001E
:104ED0000D020000000000000000000000020D00B4
:104EE000A4FF09A4FF0000000000000D0200000064
:104EF00000FFA40000090900020D00000000A4FF4B
:104F00000D0200000000FFA40009090000000000DD
:104F1000000000A4FF0009090000000D02000000CD
:104F200000FFA40000A4FF00020D00000000A4FF89
:104F300000000000090900000000A4FF00090909A1
:104F40000900000000FFA4000D0B09000000000094
:104F50000000A4FF090900000000FFA400000000F9
:104F600000000000020D00000000A4FF0000000D82
:104F70000200000000FFA40000020D00090900A4C7
:104F8000FF0000000D020009A4FFFFA60D000909A3
:104F90000D0200000000FFA40000000000020D0050
:104FA000000009A4FF0000000000000D0200FFA4A3
:104FB00000FFA4000D0B0900020D09090009A4FF60
:104FC0000D020000A4FFFFA40009090000020D0D5E
:104FD000020000A4FF0009090000000DA6FF000068
:104FE00000FFA40000000000020D00000000A4FF6C
:104FF00000020D0D0B0909090000A4FF00A4FF0920
:105000000900090900FFA4000009090000000DA61D
:10501000FF000000090900000000FFA400000000DC
:105020005B5B5B5B5B5B5B5B5B5B5B5B5B000000E1
:1050300000005B00000000005B00000000005B005F
:10504000000000005B00000000005B0000000000AA
:105050005B5B5B5B5B5B5B5B5B5B5B5B000000000C
:10506000005B00000000005B00000000005B00002F
:105070000000005B00000000005B00000000005B1F
:105080005B00000000005B00000000005B0000000F
:1050900000005B00000000005B00000000005B00FF
:1050A000000000005B5B5B5B5B5B5B5B5B5B5B5BBC
:1050B00000000000005B00000000005B000000003A
:1050C000005B00000000005B00000000005B0000CF
:1050D0000000005B5B5B5B5B5B5B5B5B5B5B5B5B31
:1050E0005B5B5B5B5B5B5B5B5B5B5B5B5B00000021
:1050F00000005B00000000005B00000000005B009F
:10510000000000005B00000000005B0000000000E9
:105110005B5B5B5B5B5B5B5B5B5B5B5B000000004B
:10512000005B00000000005B00000000005B00006E
:105130000000005B00000000005B00000000005B5E
:105140005B00000000005B00000000005B0000004E
:1051500000005B00000000005B00000000005B003E
:10516000000000005B5B5B5B5B5B5B5B5B5B5B5BFB
:1051700000000000005B00000000005B0000000079
:10518000005B00000000005B00000000005B00000E
:105190000000005B5B5B5B5B5B5B5B5B5B5B5B5B70
:1051A0005B5B5B5B5B5B5B5B5B5B5B5B5B00000060
:1051B00000005B00000000005B00000000005B00DE
:1051C000000000005B00000000005B000000000029
:1051D0005B5B5B5B5B5B5B5B5B5B5B5B000000008B
:1051E000005B00000000005B00000000005B0000AE
:1051F0000000005B00000000005B00000000005B9E
:105200005B00000000005B00000000005B0000008D
:1052100000005B00000000005B00000000005B007D
:10522000000000005B5B5B5B5B5B5B5B5B5B5B5B3A
:1052300000000000005B00000000005B00000000B8
:10524000005B00000000005B00000000005B00004D
:105250000000005B5B5B5B5B5B5B5B5B5B5B5B5BAF
:105260005B5B5B5B5B5B5B5B5B5B5B5B5B0000009F
:1052700000005B00000000005B00000000005B001D
:10528000000000005B00000000005B000000000068
:105290005B5B5B5B5B5B5B5B5B5B5B5B00000000CA
:1052A000005B00000000005B00000000005B0000ED
:1052B0000000005B00000000005B00000000005BDD
:1052C0005B00000000005B00000000005B000000CD
:1052D00000005B00000000005B00000000005B00BD
:1052E000000000005B5B5B5B5B5B5B5B5B5B5B5B7A
:1052F00000000000005B00000000005B00000000F8
:10530000005B00000000005B00000000005B00008C
:105310000000005B5B5B5B5B5B5B5B5B5B5B5B5BEE
:105320005B5B5B5B5B5B5B5B5B5B5B5B5B090000D5
:10533000095B5B5B5200095B5BADFF00095B5B5B7C
:105340005B5B5B5B5B5B5B5B5B5B5B5B5B5B5B5BAD
:105350005B5B5B5B5B5B5B5B5B5B5B5B5B090000A5
:10536000095B5B5B5200095B5BADFF00095B5B5B4C
:105370005B5B5B5B5B5B5B5B5B5B5B5B5B5B5B5B7D
:105380005B5B5B5B5B5B5B5B5B5B5B5B5B09000075
:10539000095B5B5B5200095B5BADFF00095B5B5B1C
:1053A0005B5B5B5B5B5B5B5B5B5B5B5B5B5B5B5B4D
:1053B0005B5B5B5B5B5B5B5B5B5B5B5B5B09000045
:1053C000095B5B5B5200095B5BADFF00095B5B5BEC
:1053D0005B5B5B5B5B5B5B5B5B5B5B5B5B5B5B5B1D
:1053E0005B5B5B5B5B5B5B5B5B5B5B5B5B09000015
:1053F000095B5B5B5200095B5BADFF00095B5B5BBC
:105400005B5B5B5B5B5B5B5B5B5B5B5B5B5B5B5BEC
:105410005B5B5B5B5B5B5B5B5B5B5B5B5B090000E4
:10542000095B5B5B5200095B5BADFF00095B5B5B8B
:105430005B5B5B5B5B5B5B5B5B5B5B5B5B5B5B5BBC
:105440005B5B5B5B5B5B5B5B5B5B5B5B5B090000B4
:10545000095B5B5B5200095B5BADFF00095B5B5B5B
:105460005B5B5B5B5B5B5B5B5B5B5B5B5B5B5B5B8C
:105470005B5B5B5B5B5B5B5B5B5B5B5B5B09000084
:10548000095B5B5B5200095B5BADFF00095B5B5B2B
:105490005B5B5B5B5B5B5B5B5B5B5B5B5B5B5B5B5C
:1054A0005B5B5B5B5B5B5B5B5B5B5B5B5B09000054
:1054B000095B5B5B5200095B5BADFF00095B5B5BFB
:1054C0005B5B5B5B5B5B5B5B5B5B5B5B5B5B5B5B2C
:1054D0005B5B5B5B5B5B5B5B5B5B5B5B5B09000024
:1054E000095B5B5B5200095B5BADFF00095B5B5BCB
:1054F0005B5B5B5B5B5B5B5B5B5B5B5B5B5B5B5BFC
:105500005B5B5B5B5B5B5B5B5B5B5B5B5B090000F3
:10551000095B5B5B5200095B5BADFF00095B5B5B9A
:105520005B5B5B5B5B5B5B5B5B5B5B5B5B5B5B5BCB
:105530005B5B5B5B5B5B5B5B5B5B5B5B5B090000C3
:10554000095B5B5B5200095B5BADFF00095B5B5B6A
:105550005B5B5B5B5B5B5B5B5B5B5B5B5B5B5B5B9B
:105560005B5B5B5B5B5B5B5B5B5B5B5B5B09000093
:10557000095B5B5B5200095B5BADFF00095B5B5B3A
:105580005B5B5B5B5B5B5B5B5B5B5B5B5B5B5B5B6B
:105590005B5B5B5B5B5B5B5B5B5B5B5B5B09000063
:1055A000095B5B5B5200095B5BADFF00095B5B5B0A
:1055B0005B5B5B5B5B5B5B5B5B5B5B5B5B5B5B5B3B
:1055C0005B5B5B5B5B5B5B5B5B5B5B5B5B09000033
:1055D000095B5B5B5200095B5BADFF00095B5B5BDA
:1055E0005B5B5B5B5B5B5B5B5B5B5B5B5B5B5B5B0B
:1055F0005B5B5B5B5B5B5B5B5B5B5B5B5B09000003
:10560000095B5B5B5200095B5BADFF00095B5B5BA9
:105610005B5B5B5B5B5B5B5B5B5B5B5B5B5B5B5BDA
:10562000000000A6530066A65E0000000013A6D48A
:105630009D6666A65E0013A7A613005EA666004AD6
:10564000D5A61300D49D66669DD4A613005EA666FB
:105650000053A60013A6A653000053A60013A6D518
:105660004A0066A65E0013A6A713005EA666669DA6
:10567000D4A61300D54A005EA6666666A6D54A0083
:105680000013A76666A6669E940013A7669DD4A61F
:105690001300004AD5A6665EA61300A6130066A6F0
:1056A0005E000000A61300669E940053A600000052
:1056B000D49D6666A65E6666A6D54A00949E660080
:1056C00013A60013A6D49D66A61300A653005EA6DB
:1056D0005E0013A60013A6000000A61300A6530048
:1056E000000000FFFFFF00A4FFD4EEFFFFF766FFFE
:1056F000EED4D4EEFFA69DD4D5D4D4D49D66D49D4B
:1057000066D5D4D4D5D4D5A666A6D5D4D4D4D4D48D
:10571000FFA40000000066F7FF000000FFFFFFFF8E
:105720005B005EB7FFFFFFFF94EEFFFFFFFFD49D1E
:105730006694EEFFD5D4D5FFFFFFD49D6694EEFFAF
:10574000D54A0094D5D494D594004AD5D54A00942E
:10575000D5D494D594004AD594D5D4D54A00004ADE
:10576000D5D4D4D4000000D44A00000000004AD5AB
:10577000D4D4D4D49D66D49D66D49D66D4D4D4D4D8
:10578000D494D4D4D4D4D49494D5D4D54A00D4D4F5
:10579000D4D54A00669E94000000D54A000000005F
:1057A000000000A6530066A65E0000000013A6D409
:1057B0009D6666A65E0013A7A613005EA666004A55
:1057C000D5A61300D49D66669DD4A613005EA6667A
:1057D0000053A60013A6A653000053A60013A6D597
:1057E0004A0066A65E0013A6A713005EA666669D25
:1057F000D4A61300D54A005EA6666666A6D54A0002
:105800000013A76666A6669E940013A7669DD4A69D
:105810001300004AD5A6665EA61300A6130066A66E
:105820005E000000A61300669E940053A6000000D0
:10583000D49D6666A65E6666A6D54A00949E6600FE
:1058400013A60013A6D49D66A61300A653005EA659
:105850005E0013A60013A6000000A61300A65300C6
:10586000000000FFFFFF00A4FFD4EEFFFFF766FF7C
:10587000EED4D4EEFFA69DD4D5D4D4D49D66D49DC9
:1058800066D5D4D4D5D4D5A666A6D5D4D4D4D4D40C
:10589000FFA40000000066F7FF000000FFFFFFFF0D
:1058A0005B005EB7FFFFFFFF94EEFFFFFFFFD49D9D
:1058B0006694EEFFD5D4D5FFFFFFD49D6694EEFF2E
:1058C000D54A0094D5D494D594004AD5D54A0094AD
:1058D000D5D494D594004AD594D5D4D54A00004A5D
:1058E000D5D4D4D4000000D44A00000000004AD52A
:1058F000D4D4D4D49D66D49D66D49D66D4D4D4D457
:10590000D494D4D4D4D4D49494D5D4D54A00D4D473
:10591000D4D54A00669E94000000D54A00000000DD
:105920000000001309001313130000000009131DE9
:105930001C13131313000913130900131313000A84
:105940001D1309001D1C13131C1D13090013131331
:105950000009130009131309000009130009131D9E
:105960000A00131313000913130900131313131C54
:105970001D1309001D0A001313131313131D0A002E
:10598000000913131313131C1C000913131C1D13FC
:105990000900000A1D131313130900130900131340
:1059A00013000000130900131C1C00091300000061
:1059B0001D1C131313131313131D0A001C1C1300B7
:1059C00009130009131D1C131309001309001313F5
:1059D0001300091300091300000013090013090044
:1059E000000000FFFFFF00A4FF1DAEFFFFAD13FF8F
:1059F000AE1D1DAEFF13141D1D1D1D1D1C135D14BA
:105A0000131C1D1D1D1D1C1313131D1D1D1D1D1DF0
:105A1000FFA40000000013ADFF000000FFFFFFFF28
:105A20005B00136DFFFFFFFF1CAEFFFFFFFF1D1CA0
:105A3000131CAEFF1C1D1DFFFFFF1D1C131CAEFF22
:105A40001D0A001C1D1D1D1D1C000A1D1D0A001C19
:105A50001D1D1D1D1C000A1D1C1D1D1D0A00000A08
:105A60001D1D1D1D0000001D0A00000000000A1D74
:105A70001D1D1D1D1C131D1C131D1C131D1D1D1D77
:105A80001D1D1D1D1D1D1D1D1C1D1D1D0A001D1D77
:105A90001D1D0A00131C1C0000001D0A0000000050
:105AA000000000D44A0094D594000000004AD51D9F
:105AB0005DD494D594004AD5D54A0094D5D4000A33
:105AC0001DD54A001D5DD4D45D1DD44A0094D5D4A3
:105AD000004AD4004AD4D44A00004AD5004AD51D11
:105AE0000A00D4D594004AD5D54A0094D5D4D45DC3
:105AF0001DD54A001D0A0094D594D4D4941D0A00E3
:105B0000004AD5D4D494D45D1C004AD5D45D1DD5AB
:105B10004A00000A1D94D594D44A00D44A0094D572
:105B200094000000D44A00D45D1C004AD400000058
:105B30001D5DD4D4D594D4D4941D0A001C5DD4002A
:105B40004AD5004AD51D5DD4D44A00D44A0094D524
:105B500094004AD5004AD4000000D44A00D44A0038
:105B6000000000FFFFFF00A4FF1DAEFFFFEED4FF0B
:105B7000AE1D1DAEFFD5541D1D1D1D1D5DD41D5434
:105B8000D41D1D1D1D1D1D94D4941D1D1D1D1D1DE9
:105B9000FFA400000000D4EEFF000000FFFFFFFFA5
:105BA0005B0094EEFFFFFFFF1CAEFFFFFFFF1D5DDC
:105BB000D41CAEFF1D1D1DFFFFFF1D5DD41CAEFFDD
:105BC0001D0A001C1D1D1C1D1C000A1D1D0A001C99
:105BD0001D1D1D1D1C000A1D1C1D1D1D0A00000A87
:105BE0001D1D1D1D0000001D0A00000000000A1DF3
:105BF0001D1D1D1D5DD41D5DD41D5DD41D1D1D1DF0
:105C00001D1D1D1D1D1D1D1D1C1D1D1D0A001D1DF5
:105C10001D1D0A00D45D1C0000001D0A00000000CC
:105C2000000000E45200DCE4DC0000000052E41458
:105C30009CDCDCE4DC004AE4E44A00DCE4E4000A46
:105C400055E44A00149CE4E49C14E45200DCE4E4CF
:105C50000052E40052E4E452000052E4004AE455E9
:105C60000A00E4E4DC004AE4E44A00DCE4DCDC9C16
:105C700014E45200550A00DCE4E4E4E4DC550A00D4
:105C8000004AE4E4E4DCDC9C14004AE4E49C14E410
:105C90004A00000A55DCE4DCE45200E45200DCE493
:105CA000DC000000E45200DC9C140052E400000020
:105CB000149CE4E4E4DCE4E4DC550A00149CDC001D
:105CC0004AE4004AE4149CDCE45200E45200DCE4C0
:105CD000DC004AE40052E4000000E45200E4520018
:105CE000000000FFFFFF00A4FF14AEFFFFF6DCFF83
:105CF000AE1414AEFFE49C14551454149CE4559C4B
:105D0000E4541454551454DCE4DC551454545454E1
:105D1000FFA400000000DCF6FF000000FFFFFFFF13
:105D20005B00DCF6FFFFFFFF14AEFFFFFFFF149CDC
:105D3000E414AEFF541455FFFFFF149CE414AEFFAF
:105D4000550A00145454545414000A55550A0014AA
:105D50005454545414000A55145454550A00000A5B
:105D600055545454000000540A00000000000A5525
:105D7000545454149CE4149CE4149CE4545454541B
:105D80001455545454541455145454550A0054542E
:105D900054550A00DC9C14000000550A0000000065
:105DA000000000130900131313000000000913A6DC
:105DB0005D12131313000913130900131313005377
:105DC000A6130900A61D13131CA613090013131311
:105DD000000913000913130900000913000913A691
:105DE0005300131313000913130900131313125D47
:105DF000A6130900A71300131313131313A61300FC
:105E0000000913131313125DA6000913131DA61323
:105E100009000013A6131313130900130900131329
:105E200013000000130900125DA600091300000012
:105E3000A65D13131313131313A61300A65D12000C
:105E40000913000913A65D121309001309001313A7
:105E500013000913000913000000130900130900BF
:105E6000000000FFFFFF00A4FFD4EEFFFFAE1DFF08
:105E7000EED4D4EEFF1D54D4D5D4D4D45D1DD55466
:105E80001D94D4D4D5D4941D1D1DD5D4D4D4D4D42C
:105E9000FFA4000000001DAEFF000000FFFFFFFF99
:105EA0005B001CAEFFFFFFFF94EEFFFFFFFFD45D22
:105EB0001D94EEFF94D4D5FFFFFFD45D1D94EEFF3B
:105EC000D54A0094D5D4D4D594004AD5DD4A00945F
:105ED000D5D4D4D594004AD594D5D4D54A00004A17
:105EE000D5D4D4D4000000D44A00000000004AD524
:105EF000D4D4D4D4541DD45D1DD4541DD4D4D4D4FE
:105F0000D4D5D4D4D4D4D4D594D5D4D54A00D4D4EB
:105F1000D4D54A001C5DD4000000D54A0000000022
:105F2000000000E45200DCE4DC0000000052E46603
:105F3000A5DBDCE4DC004AE4E44A00DCE4E4001332
:105F4000A6E44A0066A5DCDCA566E45200DCE4E4D5
:105F50000052E40052E4E452000052E4004AE4A695
:105F60001300E4E4DC004AE4E44A00DCE4DCDBA502
:105F700066E45200A71300DCE4E4E4E4E4A61300C2
:105F8000004AE4E4E4E4DBE566004AE4DCA566E418
:105F90004A000013A6E4E4DCE45200E45200DCE42E
:105FA000DC000000E45200DBE5660052E400000083
:105FB00066A5DCE4E4DCE4E4E4A6130066E5DB00CB
:105FC0004AE4004AE466A5DBE45200E45200DCE463
:105FD000DC004AE40052E4000000E45200E4520015
:105FE000000000FFFFFF005BFF66B7FFFFEEDCFF76
:105FF000B76666B7FFE4A566A6666666A5E466A50D
:10600000E4A66666A666A6E4E4E4A6666666666638
:10601000FFA400000000DCF6FF000000FFFFFFFF10
:106020005B00DCEEFFFFFFFF5EB7FFFFFFFF66A533
:10603000E45EB7FFA666A6FFFFFF66A5E45EB7FFB6
:10604000A70B005EA666A6665E0013A7A70B005E00
:10605000A666A6665E0013A7A66666A71300000BD9
:10606000A7666666000000A613000000000013A7E4
:1060700066666666A5E466A5E466A5E46666666689
:1060800066666666666666665EA666A713006666F0
:1060900066A71300DBE566000000A7130000000000
:1060A000000000A45200A4A4A40000000052A566B1
:1060B000A5A4A4A4A40052A4A45200A4A4A40013C0
:1060C000A6A5520066A5A4A4A566A45200A4A4A4F3
:1060D0000052A40052ADA452000052AD0052A5A639
:1060E0000B00A4A4A40052ADA45200A4A4A4A4A58F
:1060F00066A55200A71300A4A4A4A4A4A4A60B0000
:106100000052A4A4A4A4A4A55E0052A4A4A566A5BC
:1061100052000013A6A4A4A4A45200A45200A4A454
:10612000A4000000A45200A4A55E0052A400000038
:1061300066A5A4A4A4A4A4A4A4A60B005EA5A40080
:1061400052AD0052A566A5A4A45200A45200A4A476
:10615000A40052AD0052A4000000A45200A45200BA
:106160000000006B736B001974666D6B6B23136B0F
:106170006D66A66D6B135DA6A66666A61C13A61CAF
:106180001366A666A66666131313A666666666663B
:1061900074190000000013236B0000006B736B7414
:1061A00011001323736B736B666D736B736BA61C9B
:1061B00013666D6B66A6666B736BA61C13666D6BC0
:1061C000A613005EA666A6665E0013A7A713005E70
:1061D000A66666A65E0013A75EA666A71300001358
:1061E000A7666666000000A653000000000013A723
:1061F000666666A61C13A61C13A61D136666666655
:1062000066A66666666666A65EA666A713006666EE
:1062100066A71300125DA6000000A713000000008F
:10622000000000540A00145414000000000A55E451
:106230009C14145414000A55550A00145454005266
:10624000E4550A00E49C14149CE4540A00145454C9
:10625000000A54000A54540A00000A55000A55E482
:106260005200545414000A55550A00145554149CF5
:10627000E4550A00E44A00145454541454E45200FF
:10628000000A55541454149CDC000A55149CE4551F
:106290000A00004AE4545414540A00540A001454E6
:1062A00014000000540A00149CDC000A5400000092
:1062B000E49C14545414541454E45200DC9C140010
:1062C0000A55000A55E49C14540A00540A00145557
:1062D00014000A55000A54000000540A00540A0031
:1062E000000000FFFFFF00A4FFDCF6FFFFAE14FF7D
:1062F000F6DCDCF6FF559CE4E4DCE4E49C14E49C6E
:1063000014DCE4E4E4E4DC541454E4DCE4E4E4E425
:10631000FFA40000000014AEFF000000FFFFFFFF1D
:106320005B0014AEFFFFFFFFDCF6FFFFFFFFE49C06
:1063300014DCF6FFDCDCE4FFFFFFE49C14DCF6FF7A
:10634000E44A00DCE4E4DCE4DC004AE4E44A00DCA7
:10635000E4E4E4E4DC004AE4DCE4E4E44A0000527F
:10636000E4E4E4E4000000E452000000000052E431
:10637000E4E4E4E49C14E49C14E49C14E4E4E4E425
:10638000DCE4E4E4E4E4DCE4DCE4E4E44A00E4E463
:10639000E4E45200149CDC000000E4520000000021
:1063A0000000008A49008A8A8A0000000041D2F673
:1063B000E4898A8A8A0041D29241008A8A8A005BF3
:1063C000F6D24100B6A48A8A9CF68A41008A8A8A5B
:1063D00000498A00418A8A49000041920041D2F670
:1063E0005B008A8A8A004192D241008A8A9289E4BB
:1063F000F6D24100F652008A8A8A8A8A92F65B00B7
:106400000041D28A8A9289E4AD0041D28AA4F6D2B0
:106410004000005BF6928A8A8A41008A41008A8A9B
:106420008A0000008A410089E4AD00498A0000002A
:10643000F6A48A8A8A8A8A8A92F65B00ADE4890089
:1064400041920041D2F6E4898A41008A41008A9251
:106450008A00419200418A0000008A41008A490076
:10646000000000FFFFFF00A4FFF6FFFFFFE58AFF2B
:10647000FFF6F6FFFF8A9CF6F6F6F6F69C8AF69C87
:106480008AEDF6F6F6F6ED928A92F6F6F6F6F6F65E
:10649000FFA4000000008AE5FF000000FFFFFFFFEF
:1064A0005B008AE5FFFFFFFFADFFFFFFFFFFF69CEC
:1064B0008AADFFFFEDF6F6FFFFFFF69C8AADFFFF0A
:1064C000F65200ADF6F6ADF6AD0052F6F65200AD5E
:1064D000F6F6EDF6AD0052F6ADF6F6F65200005BBC
:1064E000F6F6F6F6000000F65B00000000005BF632
:1064F000F6F6F6F69C8AF69C8AF6A48AF6F6F6F686
:10650000F6EDF6F6F6F6F6EDADF6F6F65200F6F620
:10651000F6F65B0089E4AD000000F65B00000000C9
:106520000000001D0A001C1D1C000000000A1DD4F4
:106530005D1C1C1D1C000A1D1D0A001C1D1D004A9F
:10654000D51D0A00D45D1D1D5DD41D0A001C1D1D36
:10655000000A1D000A1D1D0A00000A1D000A1DD5A3
:106560004A001D1D1C000A1D1D0A001C1D1C1C5D6F
:10657000D41D0A00D54A001C1D1D1D1D1DD54A0035
:10658000000A1D1D1D1D1C5DD4000A1D1C5DD41DAF
:106590000A00004AD51D1D1C1D0A001D0A001C1DF5
:1065A0001C0000001D0A001C5DD4000A1D00000034
:1065B000D45D1D1D1D1C1D1D1DD54A00D45D1C0074
:1065C0000A1D000A1DD45D1C1D0A001D0A001C1DA9
:1065D0001C000A1D000A1D0000001D0A001D0A0003
:1065E0000000006B736B0011741D246B749A8A6B2E
:1065F000241D1D246B92531D1D1D1D1D538A1D53EB
:106600008A1C1D1D1D1D1C928A921D1D1D1D1D1DF8
:106610007419000000008A9B6B0000006B736B74A0
:1066200011008A9B736B736B1D24736B736B1D530B
:106630008A1D24731C1D1D6B736B1D538A1D2473CF
:10664000650A001C1D1D1D1D1C000A1D650A001C7D
:106650001D1D1D1D1C000A1D1D1D1D1D0A00000AFB
:106660001D1D1D1D0000001D0A00000000000A1D68
:106670001D1D1D1D5C5B1D5C5B1D5C5B1D1D1D1DD3
:106680001D1D1D1D1D1D1D1D1C1D1D1D0A001D1D6B
:106690001D1D0A00525C1C0000001D0A00000000C5
:1066A0000000008A4900928A8A0000000041921D81
:1066B0005389928A8A0041D29241008A8A8A000ACA
:1066C0001D9241001D53CACA531D8A41008A8A8AFD
:1066D00000498A00418A8A49000041D20041921D46
:1066E0000A008A8A8A0041D2D241008A8A8A895362
:1066F0001D9241001D0A008A8A928A8A921D0A0010
:106700000041D28A8A9289531C0041D28A531D9239
:106710004100000A1D928A8A8A41008A4100928AB9
:106720008A0000008A410089531C00498A00000049
:106730001D53CA8A8A8A8A8A921D0A001C538900BC
:1067400041D20041921D53898A41008A41008A92B8
:106750008A0041D200418A0000008A41008A490033
:10676000000000FFFFFF00A4FF66F7FFFFAD13FF6F
:10677000F76666F7FF131CA6A66666A61C13A61C82
:106780001366A666A66666131313A6666666666635
:10679000FFA40000000013ADFF000000FFFFFFFF9B
:1067A0005B00136DFFFFFFFF5EF7FFFFFFFFA61CFF
:1067B000135EF7FF6666A6FFFFFFA61C135EF7FFDA
:1067C000A613005EA66666A65E0013A7A613005E6B
:1067D000A66666A65E0013A75EA666A71300001352
:1067E000A7666666000000A613000000000013A75D
:1067F00066666666A5A466A5A466A5A466666666C2
:1068000066A66666666666A65EA666A70B006666F0
:1068100066A70B00A4A55E000000A71300000000FF
:1068200001140A0F0A0B0C0D0E0C0C0C0C0C966EBE
:1068300046281E080B09D420001014003C32090021
:106840004201091E024209101E02250304042612F9
:10685000FF0214143203000157580A0C090D0A965E
:106860006E4646460A04090000001014083C32092E
:1068700002420108260242010F26024208031404C4
:106880004210031404421803140442200314044069
:106890000105260240010B26024001122602401487
:1068A000031404251215041216FF03000F00003212
:1068B000363437181718171596645A5046090809C0
:1068C0000400021014006432090025030404271494
:1068D000FF04140514006E70737724242424247894
:1068E00064503C320408090000100000001400004D
:1068F0000025010304261681080A040400300A0B4F
:1069000081100A04040030120B81180A04040030BC
:106910001A0B81200A04040030220BFF11141E0000
:106920000A0B0C0D0E06060606060A0A0A0A0A0ECD
:106930000209000000140000FE0900008700022880
:106940001607870002140C00320A0C100A04010A10
:106950000525030504120CFF0514325A000000003F
:1069600000040506070896785A3C1E090A0900002B
:106970000000000000000000250103042716800825
:106980000A03030080100A03030080180A030300AF
:1069900080200A03030014090C080A0A14110C08C9
:1069A000120A14190C081A0A14210C08220A800869
:1069B000100303008010100303008018100303006D
:1069C000802010030300140912080A101411120881
:1069D0001210141912081A10142112082210FF069E
:1069E00014283C0014151617040607080896786446
:1069F0005A500E0A09000010000000320000008208
:106A000001030A04008201060A04008201090A0443
:106A10000082010C0A0400410A030D041403050856
:106A2000040514030808040814030B08040B1403DA
:106A30000E08040E821D030A0400821D060A0400CB
:106A4000821D090A0400821D0C0A0400411D030D69
:106A50000414240508230514240808230814240B0F
:106A600008230B14240E08230E250314042614FFF8
:106A7000074B0A140207080A090F14191919787824
:106A8000787878090A0D00000010080064280200D8
:106A90004201070C02421C050B027A131502021474
:106AA000040614040E14041614220414220C1422D6
:106AB00016251403042707FF08140A14010304050C
:106AC000060A0F141414786E645A50020E0900005E
:106AD000001008005A320200140406142204142282
:106AE0000C0400052514034201070C0242010F0C9F
:106AF00002421C050B02421C0D0B02430E11080240
:106B0000140C10000E12141312410E0F0802FF1283
:106B1000140A000A0B0C0D0E10101010100F0F0F9E
:106B20000F0F060F090000000000000000000087A2
:106B30000002281607870002140C01500103090304
:106B400048020308035401050803500106070350D7
:106B50001203090554120508055012060705250100
:106B600004041204FF0914050A64898CFB334B4B9F
:106B700050555A9696828278080409000010140035
:106B800000F078000082050A0D0D00010C0A821940
:106B90000A0D0D00011F0A421112090240111309CA
:106BA0000225070C04080CFF0A14193C0000000021
:106BB000000C0C0C0C0C9682786E64060809000020
:106BC0000000000000000000250D030427165405F6
:106BD000041103541504110580050B110308C201AB
:106BE000041511000D04C207060D0D000D06C209A3
:106BF000080909000D08C20B0A0505000D0A8203E9
:106C000006030F080004065404100404FF0B14329A
:106C1000000004669764060606060678789696F0E5
:106C20000B080900000010080064500200420A032B
:106C300009044214030904421E0309044209160907
:106C400000420C0F110242050B0902420F0B090210
:106C500042190B0902421C130B01140403140E0306
:106C600014180314220314041614231525141404F1
:106C70002611FF0C141400003C023B6613130E1087
:106C800015B4AAA0A0A00C0A090000001014003C32
:106C9000320900420A051204420E0512044212058E
:106CA000120442160512044202060B0242020A0BAB
:106CB0000242020E0F024202120B02811E04040461
:106CC00000082005811E0904040008200A811E0E08
:106CD00004040008200F250314042716FF040A00EB
:106CE0000A0B0C0D0E0E0E0E0E0E141414141406B8
:106CF00008090000000000000000000087000228D2
:106D00001607870002140C0054010C1202880F09A8
:106D1000040408250803041207FF0D8C0508000170
:106D200002030432373C4650A09B96918C06080D16
:106D300000001000000028000000251203040A03D0
:106D40003A14034205121E027005131E0250051468
:106D50001E02C105151E02FF0E140A1400000000D9
:106D6000001E23282A2D96918C87820C080900008A
:106D70001000000000000000810A0A0D0D00700BD9
:106D80000B0C03C10C0A030DC1100A030DC1140A38
:106D9000030D5016080C024816070C02C117060313
:106DA00004C11B060304C11F0603042503030427B3
:106DB00014FF0F080A14011D1E1F200F1414191EA2
:106DC000787878788C080E0900000010080064506C
:106DD00002004202040A03420F0D0A01410C0E0395
:106DE00002430C0F0302041416251403FF10140AA7
:106DF000140178817E7B0C0F0F0F0C969696969659
:106E0000090A0900001000000032000000250103FB
:106E1000042704810813040400080A14C2070A06A0
:106E20000843070A0602811013040400081214C262
:106E30000F0A0608430F0A0602811813040400080B
:106E40001A14812013040400082214FF14031E00E6
:106E500000000000000606060606141414141406AA
:106E60000809000000000000000000008700022860
:106E70001607870002140C01D00B030302800B07D6
:106E8000030600430B060302430B0A0302500807E4
:106E9000030325030304090AFFFFFFFFFFFFFFFFB2
:106EA000FFFFFFFFFFFFFFFFFFFFFFFFFFFFFFFFF2
:106EB000FFFFFFFFFFFFFFFFFFFFFFFFFFFFFFFFE2
:106EC000FFFFFFFFFFFFFFFFFFE5E4E5E5E5E5E589
:106ED000E4E4D2EDFFE5E4E4D3DCE5E5E5E40952E2
:106EE000DBE5E4E5E5E5E5D3EDFFE5E4E4D3DCE56A
:106EF000E5E5E4094ADBE4E5E4D3DCEDFFFFFFD39D
:106F0000DBEDFFFFFFD3DCEDFFFFFFD3DCEDFFFF89
:106F1000FFD3DCEDFFFFFFD3DCEDFFFFFFD3DCEDA4
:106F2000FFFFFFD3DCEDFFFFFFFFFFFFFFFFFFFFD2
:106F3000FFFFFFFFFFFFFFFFFFFFFFFFFFFFFFFF61
:106F4000FFFFFFFFFFFFFFFFFFFFFFFFFFFFFFFF51
:106F5000FFFFFFFFFFFFFFFFFFE5E4E5E5E5E5FFDE
:106F6000F6E4D2EDFFFFFFFFD3DCE5FFFFFFFFED0F
:106F7000D2FFFFFFFFFFFFFFFFFFFFFFFFFFFFFF4E
:106F8000FFFFFFFFFFFFFFFFFFFFFFFFFFFFFFFF11
:106F9000FFFFFFFFFFFFFFFFFFFFFFFFFFFFFFFF01
:106FA000FFFFFFFFFFFFFFFFFFFFFFFFFFFFFFFFF1
:106FB000FFFFFFFFFFFFFFFFFFFFFFFFFFFFFFFFE1
:106FC000FFFFFFFFFFFFFFFFFFFFFFFFFFFFFFFFD1
:106FD000FFFFFFFFFFFFFFFFFFFFFFF6E4FFFFFFE5
:106FE000E5E4E4FFEDD2E4E5E4C7C7C7C7C7C7C718
:106FF000C7C7C7C7C7C7C7C7C7C7C7C7C7C7C7C721
:10700000C7C7C7C7C7C7C7C7C7C7C7C7C7C7C7C710
:10701000C7C7C7C7C7C7C7C7C72811010101010133
:107020000101010101010101010101010101010150
:107030000101010101010101010101010101010140
:107040000101010102020202020202020202020224
:107050000202020202020202020202020202020210
:107060000202020202020202020201010203010103
:1070700004050202020202020202020202020202EB
:1070800002020202020202020202020202020202E0
:1070900002020101020306020203020301010602C9
:1070A00003060203020306020202030104050203AF
:1070B00001010102030101050202010102030101B4
:1070C0000107020306020602030602030203060288
:1070D000020203060203020306020202030602037F
:1070E0000202010102030101010502030602060278
:1070F000030602030203060202020306020302035E
:10710000010102020301010702020101020301025F
:10711000020302030602060203060203020306023A
:107120000202030602030203060202020301010532
:10713000020201010203010101070203010106022B
:10714000030101010203010101020301010702031E
:107150000101010203010203020201010202020213
:1071600002020202020202020202020202020202FF
:1071700002020202020202020202020202020202EF
:1071800002020101020202020202030101010502E0
:1071900002020202020202020202020202020202CF
:1071A00002020202020202020202010102020202C1
:1071B00002020301020203020203010502030101AC
:1071C000010203010202030202020202020202029F
:1071D0000202010102020202020203010202030290
:1071E000030102030203010202020301020203027D
:1071F0000202020202020202020201010202020271
:107200000202030102020302030101010203010160
:107210000102030101010102020202020202020252
:10722000020201010202020202020301020203023F
:10723000030102030202020301020301020203022C
:107240000202020202020202020201010202020220
:10725000020203010101070203010203020301010B
:1072600001020301020203020202020202020202FE
:1072700002020101020202020202020202020202F0
:1072800002020202020202020202020202020202DE
:1072900002020202020202020202010101010101D4
:1072A00001010101010101010101010101010101CE
:1072B00001010101010101010101010101010101BE
:1072C0000100C00000B0077F00077F009029640024
:1072D000B2077F0092356400B3077F1390306400DB
:1072E0009239641390356400923C641390386400C2
:1072F00092416413902764009237641390326400C3
:10730000923A641490336400923C6413903A64009F
:107310009243641390256400923D641390256400A9
:10732000923F64139031640092416414902564008C
:107330009248640044641390336400923F64139055
:10734000466400924A64139034640092406413903F
:107350004464009248641490296400923564139048
:107360002964009241641390296400923064139060
:107370002964009237641390276400923364139059
:10738000276400924364149027640092376413903A
:10739000276400923364139029640092356413903B
:1073A000296400924164139029640092306414901F
:1073B0002964009237641390316400923D64139005
:1073C000316400924D6413903164009241641390D3
:1073D000316400923D641490276400923F641390DE
:1073E000276400923F641390276400922E641390E8
:1073F00027640092356413902F6400923B641390CD
:107400002F6400924B6414902F6400923F64139099
:107410002F6400923B6413902464009230641390B4
:107420003C6400924064139024640092326414908F
:107430003C64009241641390226400923A64139079
:10744000226400923A641390296400924664139077
:10745000296400923A641490296400924164139064
:10746000296400924164139029640092416413904E
:107470002964009241641390356400924164139032
:107480003564009241641490296400924164139021
:107490002964009241641390276400924164139020
:1074A0002764009241641390276400924164149011
:1074B00027640092416413903364009241641390F6
:1074C00033640092416413902764009241641390E6
:1074D00027640092416414902964009241641390DF
:1074E00045640092416413902964009241641390B2
:1074F0004664009241641390356400924164139095
:107500004564009241641490296400924164139090
:107510004664009241641390276400924164139082
:107520004564009241641390276400924164149072
:107530004664009241641390336400923F64139058
:10754000436400923F641390276400923F64139059
:10755000446400923F641490296400924164139043
:10756000296400924D641390296400924164139041
:10757000486400924B641390356400924164139008
:10758000356400924A641490296400924164139017
:107590004464009248641390276400923F641390FF
:1075A000276400924B641390276400923F64149008
:1075B000276400924B641390336400923F641390ED
:1075C0003364009246641390276400923F641390E2
:1075D000276400924B6414902964009241641390D4
:1075E00045640092416413902964009241641390B1
:1075F0004664009241641390356400924164139094
:1076000045640092416414902A640092416413908E
:107610004664009241641390276400924164139081
:107620004564009241641390276400924164149071
:107630004664009241641390336400923F64139057
:10764000436400923F641390276400923F64139058
:10765000446400923F641490416400924564139026
:107660003C6400923F641390396400923C64139030
:1076700035640092396413903F6400924364139020
:107680003A6400923F641490376400923A64139015
:107690002764009233641390486400924564139009
:1076A0004564009241641390416400923C641490DC
:1076B0003C640092396413903A64009243641390DE
:1076C000376400923F641390336400923A641390DD
:1076D00027640092336414B0077F0090296400B2DD
:1076E000077F0092296400B2077F0092356400B3DF
:1076F000077F139030640092306400396413903532
:107700006400923564003C641390386400923864DD
:10771000004164139027640092276400376413903B
:10772000326400923264003A6414903364009233FD
:1077300064003C6413903A6400923A64004364131A
:1077400090256400922564003D64139025640092A6
:107750002564003F641390316400923164004164F9
:1077600014902564009225640048640044641390DA
:10777000336400923364003F641390466400924681
:1077800064004A64139034640092346400406413CB
:107790009044640092446400486414902964009208
:1077A00029640035641390296400922964004164BF
:1077B00013902964009229640030641390296400B6
:1077C0009229640037641390276400922764003381
:1077D0006413902764009227640043641490276424
:1077E0000092276400376413902764009227640096
:1077F000336413902964009229640035641390293E
:107800006400922964004164139029640092296401
:107810000030641490296400922964003764139046
:10782000316400923164003D641390316400923100
:1078300064004D641390316400923164004164131C
:1078400090316400923164003D641490276400928A
:107850002764003F641390276400922764003F640C
:107860001390276400922764002E6413902764000D
:1078700092276400356413902F6400922F64003BBC
:107880006413902F6400922F64004B6414902F6453
:1078900000922F64003F6413902F6400922F6400C5
:1078A0003B64139024640092246400306413903C81
:1078B0006400923C64004064139024640092246449
:1078C00000326414903C6400923C64004164139064
:1078D000226400922264003A64139022640092228F
:1078E00064003A641390296400922964004664138A
:1078F00090296400922964003A64149029640092EB
:107900002964004164139029640092296400416451
:107910001390296400922964004164139029640043
:1079200092296400416413903564009235640041EB
:1079300064139035640092356400416414902964A6
:107940000092296400416413902964009229640024
:1079500041641390276400922764004164139027C8
:1079600064009227640041641390276400922764A6
:1079700000416414902764009227640041641390CE
:107980003364009233640041641390336400923393
:1079900064004164139027640092276400416413DB
:1079A0009027640092276400416414902964009237
:1079B0002964004164139045640092456400416469
:1079C0001390296400922964004164139046640076
:1079D000924664004164139035640092356400411E
:1079E00064139045640092456400416414902964D6
:1079F000009229640041641390466400924664003A
:107A000041641390276400922764004164139045F9
:107A100064009245640041641390276400922764D7
:107A200000416414904664009246640041641390DF
:107A3000336400923364003F6413904364009243C4
:107A400064003F641390276400922764003F64132E
:107A500090446400924464003F641490296400924E
:107A600029640041641390296400922964004D64E4
:107A700013902964009229640041641390486400C3
:107A8000924864004B641390356400923564004161
:107A9000641390356400923564004A64149029643C
:107AA000009229640041641390446400924464008D
:107AB00048641390276400922764003F6413902762
:107AC0006400922764004B6413902764009227643B
:107AD000003F641490276400922764004B64139065
:107AE000336400923364003F641390336400923334
:107AF000640046641390276400922764003F641377
:107B000090276400922764004B64149029640092CB
:107B10002964004164139045640092456400416407
:107B20001390296400922964004164139046640014
:107B300092466400416413903564009235640041BC
:107B400064139045640092456400416414902A6473
:107B500000922A64004164139046640092466400D7
:107B60004164139027640092276400416413904598
:107B70006400924564004164139027640092276476
:107B8000004164149046640092466400416413907E
:107B9000336400923364003F641390436400924363
:107BA00064003F641390276400922764003F6413CD
:107BB00090446400924464003F64149041640092D5
:107BC000416400456413903C6400923C64003F644F
:107BD0001390396400923964003C6413903564005A
:107BE00092356400396413903F6400923F6400430F
:107BF0006413903A6400923A64003F6414903764CE
:107C000000923764003A641390276400922764005E
:107C100033641390486400924864004564139045AF
:107C20006400924564004164139041640092416491
:107C3000003C6414903C6400923C640039641390EE
:107C40003A6400923A6400436413903764009237B8
:107C500064003F641390336400923364003A641309
:107C60009027640092276400336414FF2F00000201
:107C700005065C5C3F0107070707070707070303C3
:107C80000303040404043F3F3F3F3F3F3F3F3F3F68
:107C90003F3F335B35363F3F3F3F3F3F3F3F08630A
:107CA000084307630743373809093F3F3F3F000058
:107CB0000100010001000000FFFFFFFFFFFFFFFFC9
:107CC000FFFF00000100010001000000FFFF0A03A8
:107CD00003050A1E0A324449414D4F4E44533A00AF
:107CE00054494D453A004C4556454C3A004C49568E
:107CF00045533A0053434F52453A00434156453AA3
:107D00000050524553532053544152540047414D63
:107D100045204F564552002054494D45205550208E
:107D200000E66CF46CD26D5A714671F76C066D15F5
:107D30006D2E71236D316D00000001000200030003
:107D40000400050100010101020103010401050213
:107D50000002010202020302040205030003010300
:107D600002030303040305040004010402040304E2
:107D700004040505000501050205030504050506C3
:107D800000060106020603060406050700070107B0
:107D90000207030704070508000801080208030892
:107DA0000408050900090109020903090409050A73
:107DB000000A010A020A030A040A050B000B010B60
:107DC000020B030B040B050C000C010C020C030C42
:107DD000040C050D000D010D020D030D040D050E23
:107DE000000E010E020E030E040E050F000F010F10
:107DF000020F030F040F05100010011002100310F2
:107E000004100511001101110211031104110512D2
:107E100000120112021203120412051300130113BF
:107E200002130313041305140014011402140314A1
:107E30000414051500150115021503150415051682
:107E4000001601160216031604160517001701176F
:107E50000217031704170518001801180218031851
:107E60000418051900190119021903190419051A32
:107E7000001A011A021A031A041A051B001B011B1F
:107E8000021B031B041B051C001C011C021C031C01
:107E9000041C051D001D011D021D031D041D051EE2
:107EA000001E011E021E031E041E051F001F011FCF
:107EB000021F031F041F0500000000000000000057
:107EC00000000000000000000000000000000000B2
:107ED00000000000000000000000000000000000A2
:107EE0000000000000000000000000000000000092
:107EF0000000000000000000000000000000000082
:107F0000000000000000000000004900000049528D
:107F100052000052525C2D000000000000000000E2
:107F2000000000000000000040000000494A52002C
:107F30004952525B1C52531C25241B2425251B0A25
:107F40000A2D1C12120A0A00000000000000004066
:107F50004949494949525B5B5B525B1C1C13122423
:107F60001C1209090912090909090A0A0A0A0A0A56
:107F700013120A0A12130A00000000000092525263
:107F800052525213121309001C0A1212401B6509A7
:107F90000A0009241B120000251C1C010025241CBA
:107FA0001C0024252424240000000000005249491C
:107FB0004000001B1352494900641C1C5B4A481CCA
:107FC000651C2552491C1C652464491C1C652564DC
:107FD000491C1C6D2E5C49000000000000000000E0
:107FE00000004900000000535200000053522500D9
:107FF000004A52252500005B251300005B53000A50
:108000001C095B1C657F374052522E2E1C525C2E81
:10801000251B1324251C1C12002525120000121BF1
:108020000000132E37001B37372E2E37372E2E2EFB
:108030002E2E2E6E6E6E1C131312000913120000EA
:108040001213130012251C13132E371C131313368F
:108050001C131B1B1B25131C1C1B1B1B1C1C1C1C6F
:108060001C1C1C1C1C1C13131212131300131313BF
:108070001C000913131C010037131C13002E2E1CA7
:108080001C001C772E2500137F251C010A37241C99
:108090001C0A2E25250900132E242525252E2525ED
:1080A00025252525252D2E251B2E2E251C13252582
:1080B0001C1C1C1C011C1C1300011C0A0001657700
:1080C0005C016E7F6E521B25256D1C524925251CB7
:1080D0001353001C1C1C524A001B135B5B0000095D
:1080E000525C0000005B5C000000001B0000000010
:1080F00000000000000000135B7F776E6E13657751
:10810000766E6E1B65777676761B5BBF76B67609E4
:10811000136DBFB7B6001B125C76BF0000121B12B6
:108120005B00000000090A6E6E6E77241C6E6E778D
:10813000251C1C6E776E1C1C1C76761C1C2425B717
:1081400065646D6D1B766D6D5B09125B5C5B125B2C
:10815000641213131B12121C1C1C1C1C241C1C2438
:108160002525242425251B00002513000064BF00BD
:10817000096EBFBF6D6EBF6D5B12135B12131209E8
:10818000000901000000002E1C0900096E01000911
:10819000767F7F12777F7F6412BF775B121B095B4C
:1081A000121B0900001B0900000000000000000075
:1081B000000000000000007F7F5313130064121BB7
:1081C0000100001B12000000000000000000000081
:1081D000000000000000000000000000000000009F
:1081E0000000000000000000000000000026000069
:1081F0000026002F0000002F00370000003700FF8E
:10820000000000FF00BF000000BF00370000370083
:1082100000002626000000000000000000262626A0
:10822000262600000000002F00000000370000009C
:1082300000FF00000000BF00000000370000000049
:1082400000262626262600000000000000262626FE
:108250002626002F0000000000370000000000FF6D
:10826000FFFFFF0000BF000000000037000000001B
:1082700000262626262600000000000000262626CE
:108280002600002F0000002F00370000003700FFFD
:10829000FFFFFF0000BF000000BF003700000037F5
:1082A0000026262626000000000000000000002610
:1082B000262600002F00002F00370000003700FFA7
:1082C000000000FF00BF000000BF003700003700C3
:1082D0000026262600000000000000000026000006
:1082E0000026002F0000002F00003700370000009C
:1082F00000FF00000000BF00BF0000370000003793
:108300000026000000260000000000000000000021
:10831000000000000000000000000000000000005D
:10832000000000000000000000009B000000529BC5
:10833000A400005B9B6D77000000000000000000BF
:1083400000000000000000005B000000E4F6FF09F0
:108350009BEDF6FFBFA4ADBFBFBFBF767F7FB7B7B2
:10836000BF7F766EB7B7BF00000000000000005B63
:10837000B6F6F6F6FFFFFFFFBFFFFFFFBFBFAEFF82
:10838000FFFFB7AD65FFFFB7B6AD65FFFFBFB7AE87
:108390006EFFFFBFB7B765000000000000F6F6ED06
:1083A000EDADA4B66D6D5C526E6565655265765C2B
:1083B0005C52536E246552526E25255B52772D25F3
:1083C00025526E6E2D2525000000000000A49B9B09
:1083D0004900006564A49B92006D2525649349655E
:1083E0006E652E9B5224256D25655225246D2D65C5
:1083F0005225256E2E64520000000000000000008F
:1084000000004A000000005B9B0000005B5B2D0049
:1084100000525B2E2E00015B2D1C01005C5B014AAB
:10842000654A5B1C6E7F77495B9B77776D5B6577F1
:108430006E65656D2D25255C522E25130949641C3A
:1084400009095C7F7F091C7F7F777F777F77777F44
:108450007F7776777F7F6E656E6EA4B6FF655BA4CF
:10846000B7BFFF526DBFBFBFFF7FBFBFBFBFFFBF63
:10847000BFB7BFFFFF7FB7BFBFFFFF6EB7BFBFFF75
:10848000FF77BFBFBFFFFFFFFFBFBFB75BFFFFBFF0
:10849000BFA464FFFFBFADA47FFFFFBFA4BF7FFFEA
:1084A000BFADBFBFBFFFB6BFBFBF77F7BFBFBF770F
:1084B00077FFBFBFBF64526D7F6E2E2D2D7F766E0E
:1084C0006E6E2E777777762E1C7F776E251C25773C
:1084D0006525251C096E6E1C0949255B494A6E7F7E
:1084E000645377BF775B5C256E6E255B4A25651C00
:1084F0001B5B002524245B53001C1B5B5C00000AF3
:108500005B640000006464000000005C0000000088
:10851000000000000000005B5C7FBF77765C6D7F31
:10852000B777775C6D7FBF77775C64BFBFBFBF0AEB
:108530005C6EBFBFBF0065646DBFBF00005B6D6454
:108540006D00000000125B7777777F6E6E77777F24
:10855000766D7677BF776D6E76BF7F6D6E767FBFF7
:108560007676BFBF76BFBFBFB664ADADB6B6ADBFA2
:10857000FF646DADB6AD6477BFBFBFFFFF77BFBF10
:10858000BFFFFF7FBFBFBFFFF6BFB7ADF6FFFFA4C2
:10859000ADFFFFFFFFFFFFFFFFFFFFFFFFFFF6A4A1
:1085A000005B5200000000BFBFAD5B64BFB6ADAD65
:1085B000BFFFBFFFFFFFFFBF64FFFFBFB6765BFFDC
:1085C000BFBF5B0000FF5C00000000000000000077
:1085D00000000000000000BFBF645C5C006E5C65D2
:1085E0004900006D5B00000000000000000000007A
:1085F000000000000000000000000000000000007B
:10860000000000000000000600040000000100025D
:108610000003000400050006000700080009000A26
:10862000000B000C000D000E000F001000000011E8
:1086300000120013001400150016000600030000CD
:10864000001700180019001A001B001C001D001E56
:10865000001F002000210022002300240025002606
:1086600000000000020800085504085A0000F80045
:108670000990000A1E32050000FF0000006386001A
:108680000000000011241FBECFEFD0E1DEBFCDBF40
:1086900014BE88E10FB6F8948093600010926000D9
:1086A0000FBE11E0A0E0B1E0EEEDF8EE02C00590E3
:1086B0000D92AA30B107D9F710E1A0E2B1E001C0F4
:1086C0001D92A935B107E1F7F894E1E2FAE080E004
:1086D00090E020E802C02193019632E08C309307AD
:1086E000D4F381E29AE090932E0C80932D0C10929B
:1086F0002F0CE2E3FCE080E090E003C010820196E2
:108700003A9684309105D4F3909358108093571083
:1087100091E09093520C9093530C9093510C1092C3
:10872000810015BC8FEF87B984B980E88AB98CE0E5
:1087300081B983EF82B91092000A86E08093010A22
:10874000109285001092840083E0809389008DE868
:108750008093880089E08093810082E080936F009D
:1087600082E484BD17BC95BD83E88093B00010926D
:10877000B3009093B10081E185B978940E945D7354
:108780000E940D6A0C946D740C94000026483048C9
:108790003E484947EEEDC8950000EA95E1F7000034
:1087A00000000000000000000000C0E4D1E000EE86
:1087B000A02E662776E03BD434E23A95F1F70E948A
:1087C00011443FE03A95F1F70000AA94A9F00000A7
:1087D000639500000000683029F0C895C895C895D9
:1087E0000000E9CF6627002430E5C30FD01D00004C
:1087F000000000000000DFCFC895C895C895C89557
:10880000C8950000000013D411E00091030A01276D
:108810000093030A00FF1093020AE2E0E09336009F
:1088200008958F939F93DE01679FC00100004D91D3
:108830005D91480F591FFA01059108B94D910591B5
:1088400008B95D91059108B900C0059108B900C04B
:10885000059108B9480F591F059108B90000FA01A0
:10886000059108B94D91059108B95D91059108B937
:1088700000C0059108B900C0059108B9480F591FFB
:10888000059108B90000FA01059108B94D910591CB
:1088900008B95D91059108B900C0059108B900C0FB
:1088A000059108B9480F591F059108B90000FA0150
:1088B000059108B94D91059108B95D91059108B9E7
:1088C00000C0059108B900C0059108B9480F591FAB
:1088D000059108B90000FA01059108B94D9105917B
:1088E00008B95D91059108B900C0059108B900C0AB
:1088F000059108B9480F591F059108B90000FA0100
:10890000059108B94D91059108B95D91059108B996
:1089100000C0059108B900C0059108B9480F591F5A
:10892000059108B90000FA01059108B94D9105912A
:1089300008B95D91059108B900C0059108B900C05A
:10894000059108B9480F591F059108B90000FA01AF
:10895000059108B94D91059108B95D91059108B946
:1089600000C0059108B900C0059108B9480F591F0A
:10897000059108B90000FA01059108B94D910591DA
:1089800008B95D91059108B900C0059108B900C00A
:10899000059108B9480F591F059108B90000FA015F
:1089A000059108B94D91059108B95D91059108B9F6
:1089B00000C0059108B900C0059108B9480F591FBA
:1089C000059108B90000FA01059108B94D9105918A
:1089D00008B95D91059108B900C0059108B900C0BA
:1089E000059108B9480F591F059108B90000FA010F
:1089F000059108B94D91059108B95D91059108B9A6
:108A000000C0059108B900C0059108B9480F591F69
:108A1000059108B90000FA01059108B94D91059139
:108A200008B95D91059108B900C0059108B900C069
:108A3000059108B9480F591F059108B90000FA01BE
:108A4000059108B94D91059108B95D91059108B955
:108A500000C0059108B900C0059108B9480F591F19
:108A6000059108B90000FA01059108B94D910591E9
:108A700008B95D91059108B900C0059108B900C019
:108A8000059108B9480F591F059108B90000FA016E
:108A9000059108B94D91059108B95D91059108B905
:108AA00000C0059108B900C0059108B9480F591FC9
:108AB000059108B90000FA01059108B94D91059199
:108AC00008B95D91059108B900C0059108B900C0C9
:108AD000059108B9480F591F059108B90000FA011E
:108AE000059108B94D91059108B95D91059108B9B5
:108AF00000C0059108B900C0059108B9480F591F79
:108B0000059108B90000FA01059108B94D91059148
:108B100008B95D91059108B900C0059108B900C078
:108B2000059108B9480F591F059108B90000FA01CD
:108B3000059108B94D91059108B95D91059108B964
:108B400000C0059108B900C0059108B9480F591F28
:108B5000059108B90000FA01059108B94D910591F8
:108B600008B95D91059108B900C0059108B900C028
:108B7000059108B9480F591F059108B90000FA017D
:108B8000059108B94D91059108B95D91059108B914
:108B900000C0059108B900C0059108B9480F591FD8
:108BA000059108B90000FA01059108B94D910591A8
:108BB00008B95D91059108B900C0059108B900C0D8
:108BC000059108B9480F591F059108B90000FA012D
:108BD000059108B94D91059108B95D91059108B9C4
:108BE00000C0059108B900C0059108B9480F591F88
:108BF000059108B90000FA01059108B94D91059158
:108C000008B95D91059108B900C0059108B900C087
:108C1000059108B9480F591F059108B90000FA01DC
:108C2000059108B94D91059108B95D91059108B973
:108C300000C0059108B900C0059108B9480F591F37
:108C4000059108B90000FA01059108B94D91059107
:108C500008B95D91059108B900C0059108B900C037
:108C6000059108B9480F591F059108B90000FA018C
:108C7000059108B94D91059108B95D91059108B923
:108C800000C0059108B900C0059108B9480F591FE7
:108C9000059108B90000FA01059108B94D910591B7
:108CA00008B95D91059108B900C0059108B900C0E7
:108CB000059108B9480F591F059108B90000FA013C
:108CC000059108B94D91059108B95D91059108B9D3
:108CD00000C0059108B900C0059108B9480F591F97
:108CE000059108B90000FA01059108B94D91059167
:108CF00008B95D91059108B900C0059108B900C097
:108D0000059108B9480F591F059108B90000FA01EB
:108D1000059108B94D91059108B95D91059108B982
:108D200000C0059108B900C0059108B9480F591F46
:108D3000059108B90000FA01059108B94D91059116
:108D400008B95D91059108B900C0059108B900C046
:108D5000059108B9480F591F059108B90000FA019B
:108D6000059108B94D91059108B95D91059108B932
:108D700000C0059108B900C0059108B9480F591FF6
:108D8000059108B90000FA01059108B94D910591C6
:108D900008B95D91059108B900C0059108B900C0F6
:108DA000059108B9480F591F059108B90000FA014B
:108DB000059108B94D91059108B95D91059108B9E2
:108DC00000C0059108B900C0059108B9480F591FA6
:108DD000059108B90000FA01059108B94D91059176
:108DE00008B95D91059108B900C0059108B900C0A6
:108DF000059108B9480F591F059108B90000FA01FB
:108E0000059108B94D91059108B95D91059108B991
:108E100000C0059108B900C0059108B9480F591F55
:108E2000059108B90000FA01059108B94D91059125
:108E300008B95D91059108B900C0059108B900C055
:108E4000059108B9480F591F059108B90000FA01AA
:108E5000059108B94D91059108B95D91059108B941
:108E600000C0059108B900C0059108B9480F591F05
:108E7000059108B90000FA0100000027000008B9B8
:108E800008E00A95F1F70000000000009F918F9123
:108E9000089528980E94A74AE7E1EA95F1F7289AF1
:108EA00010D1E0E0F6E0F3D0E0FF4ED0E0FF02C0EA
:108EB0000E94C7490895129A0C945E470C9460472B
:108EC000129844275527662777278CE00C9468472B
:108ED0000C946A470C946C470C946E470C94704742
:108EE0000C947247440F551F00994160660F771F1D
:108EF00001996160139A0C947D470C947F471398F5
:108F00000C9482470C9484470C9486470C948847B1
:108F10008A9541F740955095609570955F707F7088
:108F200040930A0A50930B0A60930C0A70930D0A3F
:108F30009BE04830590711F40E945173683079075B
:108F400011F40E9451730895EF93E091010AE93EF4
:108F5000E0F5E930D0F12F923F924F925F926F92FD
:108F60007F928F929F92AF92BF92CF92DF92EF92B9
:108F7000FF920F931F932F933F934F935F936F93A2
:108F80007F938F939F93AF93BF93CF93DF930E9471
:108F9000CA43DF91CF91BF91AF919F918F917F9104
:108FA0006F915F914F913F912F911F910F91FF9082
:108FB000EF90DF90CF90BF90AF909F908F907F9079
:108FC0006F905F904F903F902F90EF910895FF9397
:108FD000EF93EFB7EF93E0918400EE50E13000F0B3
:108FE000E23000F0E33000F0E43000F0E53000F073
:108FF000E63000F0E73000F0E83000F0E93000F053
:1090000005D0EF91EFBFEF91FF9118950F921F924E
:10901000ECE8F7E80090000A000C1124E00DF11DC7
:1090200005901490F00109951F900F9008952898CD
:109030000E94A74AE5E1EA95F1F7E091010AEA9575
:10904000E093010A289A00000000089528980E94E1
:10905000D04A289A0000E1E0F6E019D02BD008951C
:1090600028980E94D04AE0EB0000EA95E9F700005A
:109070000000289AF6E0E2E00AD0089528980E94BD
:10908000D04A289A0000E3E0FDEF01D00895009057
:10909000010A0A9410905F0011FC0F2E0092010A41
:1090A0000090000A11FC0E2E0092000AE0E011FC74
:1090B000E1E00895E3E0E0938900EDE8E0938800C3
:1090C0000895E7E0E0938900EBE1E09388000895DC
:1090D000E0E6F4E0A0E4B1E06091080A7091090ACA
:1090E0006D937D933197E1F7112408950F931F93AA
:1090F00080E694E0A0E4B1E0E091060AF091070A6E
:1091000040E30091040A1091050A65917591649FEE
:109110009001749F300D200F311F2D933D930197C7
:10912000A1F711241F910F910895992777273327CD
:1091300020E5629F880F080E131EE091060AF09149
:10914000070AE00DF11D45915591A0E4B1E0A00D95
:10915000B11D20E3429FB001529F700D4091040A5F
:109160005091050A640F751F6D937C931124089527
:109170009927552728E2220F629F880F080E191E93
:10918000A0E4B1E0A00DB11D6091080A7091090A38
:1091900020E3429F600D711D6D937C93112408950F
:1091A0009927772728E2220F629F880F080E191E41
:1091B000A0E4B1E0A00DB11D6091040A7091050A10
:1091C00020E3429F600D711D529F700D6D937C9343
:1091D000112408958093060A9093070A08958093B6
:1091E000080A9093090A08958093040A9093050A47
:1091F00008958091020A089511241092020A089598
:10920000882329F480910A0A90910B0A089580918D
:109210000C0A90910D0A089580E891E08093610016
:1092200090936100089580E890E0809361009093AE
:109230006100089500000000000000000000000030
:10924000000000000000000000000000000000001E
:10925000000000000000000000000000000000000E
:1092600000000000000000000000000000000000FE
:1092700000000000000000000000000000000000EE
:1092800000000000000000000000000000000000DE
:1092900000000000000000000000000000000000CE
:1092A00000000000000000000000000000000000BE
:1092B00000000000000000000000000000000000AE
:1092C000000000000000000000000000000000009E
:1092D000000000000000000000000000000000008E
:1092E000000000000000000000000000000000007E
:1092F000000000000000000000000000000000006E
:1093000099277727833008F00895E0E0F0EA660FA8
:10931000771FE60FF71FA591B491E2E3FCE02AE086
:10932000289FE00DF11DA183B2831124089590912F
:10933000510C9170880F892B8093510C08959927B7
:109340007727E2E3FCE02AE0289FE00DF11D6E3F65
:1093500031F46091510C6E7F6093510C0BC06F3FE4
:1093600031F46091510C6E6F6093510C03C076E93B
:10937000760F75831124089599277727E2E3FCE09F
:109380002AE0289FE00DF11D6083112408952F939A
:109390003F934F935F936F937F938F939F93AF937D
:1093A000BF93789411240E945B470E94816E2F9294
:1093B0003F924F925F926F927F928F929F92AF9265
:1093C000BF92CF92DF92EF92FF920F931F93CF93B2
:1093D000DF9300902F0C002019F4A1E2BAE002C044
:1093E000A7E2BBE001E0002600922F0C02E0009310
:1093F000300C5091500C6091520C7091530C809134
:10940000540C2090330C3090340C4090360C50901B
:10941000370C6090350C1091320C70903D0C8090A0
:109420003E0C90903F0CA090400CB090410C2091CD
:109430003C0CC090470CD090480CE0904A0CF09047
:109440004B0C0091490C3091460C9FEF620C431C71
:10945000F2014491410300240008C12DD02D970C46
:10946000A81CF5014491420300240008C10DD01D41
:109470000C0DED1CF7014491430300240008C10DBD
:10948000D01D8A956AF44091510C842F8695062E42
:109490000694062600FA7695679576F940FF66F9F8
:1094A00040E860FD4FE7450300240008C10DD01DD2
:1094B0000024C038D0050CF0CFE70A94C038D0059E
:1094C0000CF4C0E8C058CD939A9509F0BFCF4091F5
:1094D000300C4A954093300C97E009F0B7CF60927A
:1094E000350C4092360C90923F0CA092400C0093A9
:1094F000490CE0924A0C6093520C7093530C809389
:10950000540CDF91CF911F910F91FF90EF90DF905E
:10951000CF90BF90AF909F908F907F906F905F9013
:109520004F903F902F9099278091000A7727609164
:10953000010A11240E94D16DBF91AF919F918F912B
:109540007F916F915F914F913F912F9108950C946E
:10955000A94A0C94AB4A0F931F932ABDE0912D0C9E
:10956000F0912E0C019100000093B3000CE0ED325D
:10957000F00710F40000000010F0E1E2FAE0E093E0
:109580002D0CF0932E0CC895C895C895C895C89514
:10959000C8950000000000002AB51F910F910895A2
:1095A0000000E091010AE0FFD6CFE1E1EA95F1F792
:1095B000000000000895000000000000000000000E
:1095C000000000000000000000000000000000009B
:1095D000000000000000000000000000000000008B
:1095E000000000000000000000000000000000007B
:1095F000000000000000000000000000000000006B
:10960000000306090C101316191C1F2225282B2EE7
:10961000313336393C3F414447494C4E51535558FC
:109620005A5C5E60626466686A6B6D6F70717374B9
:10963000757678797A7A7B7C7D7D7E7E7E7F7F7F72
:109640007F7F7F7F7E7E7E7D7D7C7B7A7A79787658
:1096500075747371706F6D6B6A68666462605E5C6E
:109660005A585553514E4C494744413F3C39363383
:10967000312E2B2825221F1C191613100C09060346
:1096800000FDFAF7F4F0EDEAE7E4E1DEDBD8D5D24D
:10969000CFCDCAC7C4C1BFBCB9B7B4B2AFADABA818
:1096A000A6A4A2A09E9C9A9896959391908F8D8C3B
:1096B0008B8A888786868584838382828281818162
:1096C0008181818182828283838485868687888A5C
:1096D0008B8C8D8F9091939596989A9C9EA0A2A426
:1096E000A6A8ABADAFB2B4B7B9BCBFC1C4C7CACDF1
:1096F000CFD2D5D8DBDEE1E4E7EAEDF0F4F7FAFD0E
:10970000808182838485868788898A8B8C8D8E8FE1
:10971000909192939495969798999A9B9C9D9E9FD1
:10972000A0A1A2A3A4A5A6A7A8A9AAABACADAEAFC1
:10973000B0B1B2B3B4B5B6B7B8B9BABBBCBDBEBFB1
:10974000C0C1C2C3C4C5C6C7C8C9CACBCCCDCECFA1
:10975000D0D1D2D3D4D5D6D7D8D9DADBDCDDDEDF91
:10976000E0E1E2E3E4E5E6E7E8E9EAEBECEDEEEF81
:10977000F0F1F2F3F4F5F6F7F8F9FAFBFCFDFEFF71
:10978000000102030405060708090A0B0C0D0E0F61
:10979000101112131415161718191A1B1C1D1E1F51
:1097A000202122232425262728292A2B2C2D2E2F41
:1097B000303132333435363738393A3B3C3D3E3F31
:1097C000404142434445464748494A4B4C4D4E4F21
:1097D000505152535455565758595A5B5C5D5E5F11
:1097E000606162636465666768696A6B6C6D6E6F01
:1097F000707172737475767778797A7B7C7D7E7FF1
:1098000000020406080A0C0E10121416181A1C1E68
:1098100020222426282A2C2E30323436383A3C3E58
:1098200040424446484A4C4E50525456585A5C5E48
:1098300060626466686A6C6E70727476787A7C7E38
:109840007F7D7B79777573716F6D6B696765636118
:109850005F5D5B59575553514F4D4B494745434108
:109860003F3D3B39373533312F2D2B2927252321F8
:109870001F1D1B19171513110F0D0B0907050301E8
:10988000FFFDFBF9F7F5F3F1EFEDEBE9E7E5E3E1D8
:10989000DFDDDBD9D7D5D3D1CFCDCBC9C7C5C3C1C8
:1098A000BFBDBBB9B7B5B3B1AFADABA9A7A5A3A1B8
:1098B0009F9D9B99979593918F8D8B8987858381A8
:1098C00080828486888A8C8E90929496989A9C9EA8
:1098D000A0A2A4A6A8AAACAEB0B2B4B6B8BABCBE98
:1098E000C0C2C4C6C8CACCCED0D2D4D6D8DADCDE88
:1098F000E0E2E4E6E8EAECEEF0F2F4F6F8FAFCFE78
:109900007F7F7F7F7F7F7F7F7F7F7F7F7F7F7F7F67
:109910007F7F7F7F7F7F7F7F7F7F7F7F7F7F7F7F57
:109920007F7F7F7F7F7F7F7F7F7F7F7F7F7F7F7F47
:109930007F7F7F7F7F7F7F7F7F7F7F7F7F7F7F7F37
:109C00000309131E28313A40464C5054585B5E619C
:109C1000636567696B6C6E6F70717273747576775C
:109C2000777879797A7A7B7B7C7C7C7D7D7D7E7E82
:109C30007E7E7F7F7F7F7F7F7F7F7F7F7F7F7F7F36
:109C40007F7F7F7F7F7F7F7F7F7F7F7F7F7E7E7E27
:109C50007E7D7D7D7C7C7C7B7B7A7A797978777759
:109C6000767574737271706F6E6C6B696765636122
:109C70005E5B5854504C46403A31281E130903008D
:109C8000C6CCD5DBDFE3E5E7E9EAEBECEDEEEFEFA1
:109C9000F0F0F0F1F1F1F1F2F2F2F2F2F2F2F2F3AD
:109CA000F3F3F3F3F3F3F3F3F3F3F3F3F3F3F3F384
:109CB000F3F3F3F3F3F3F3F3F3F3F3F3F3F3F3F374
:109CC000F3F3F3F3F3F3F3F3F3F3F3F3F3F3F3F364
:109CD000F3F3F3F3F3F3F3F3F3F3F3F3F3F3F3F354
:109CE000F2F2F2F2F2F2F2F2F1F1F1F1F0F0F0EF61
:109CF000EFEEEDECEBEAE9E7E5E3DFDBD5CCC60020
:109D000000283D42302D2C2B2C2D2E2F3032333578
:109D100037393B3D3F414345484A4C4E50535557D8
:109D2000595B5D5F61636567696B6C6E70717374BD
:109D3000757778797A7B7C7D7D7E7E7F7F7F7F7F64
:109D40007F7F7F7F7F7F7E7E7D7D7C7B7A7978774A
:109D500075747371706E6C6B69676563615F5D5B71
:109D600059575553504E4C4A484543413F3D3B3966
:109D700037353332302F2E2D2C2B2C2D30423D28D1
:109D800000E9E5FED4D7D7D7D6D4D2D0CECCCAC836
:109D9000C6C3C1BFBDBAB8B6B4B1AFADABA9A7A574
:109DA000A3A19F9E9C9A999795949391908F8D8C47
:109DB0008B8A898888878685858484848383838346
:109DC0008383838383848484858586878888898A3E
:109DD0008B8C8D8F909193949597999A9C9E9FA12F
:109DE000A3A5A7A9ABADAFB1B4B6B8BABDBFC1C347
:109DF000C6C8CACCCED0D2D4D6D7D7D7D4FEE5E900
:109E0000F9F8F9F5EBE1DDDEE0E2E4E5E6E5E4E2D0
:109E1000DED9D2CAC1B7ACA299918A8683818080EB
:109E20008182838586888A8C8D8F90929395969770
:109E300098999A9B9B9C9D9D9D9E9E9E9F9F9F9F58
:109E40009F9F9F9E9E9E9D9D9D9C9B9B9A99989750
:109E500096959392908F8D8C8A8886858382818057
:109E6000808183868A9199A2ACB7C1CAD2D9DEE239
:109E7000E4E5E6E5E4E2E0DEDDE1EBF5F9F8F90042
:109E80000708070B151F2322201E1C1B1A1B1C1E54
:109E900022272E363F49545E676F767A7E7F7F7F1A
:109EA0007F7E7D7B7A7876747371706E6D6B6A6974
:109EB000686766656564646363626262616161616B
:109EC0006161616262626363636465656667686954
:109ED0006A6B6D6E7071737476787A7B7D7E7F7F2E
:109EE0007F7F7E7A766F675E54493F362E27221E2B
:109EF0001C1B1A1B1C1E2022231F150B0708070002
:109F00001F313D444E5354565A5F64696E747679DE
:109F10007C7F7F7F7F7F7F7F7F7F7F7F7F7F7F7F54
:109F20007F7F7F7F7F7F7F7F7F7F7F7F7F7F7F7F41
:109F30007F7F7F7F7F7F7F7F7F7F7F7F7F7F7F7F31
:109F40007F7F7F7F7F7F7F7F7F7F7F7F7F7F7F7F21
:109F50007F7F7F7F7F7F7F7F7F7F7F7F7F7F7F7F11
:109F60007F7F7F7F7F7F7F7F7F7F7F7F7F7F7F7F01
:109F70007F7F7F7F7F7F7F7F7F7F7F7C7871684C53
:109F80002C1C120C0A0B0A05FDF3E9DFD4CAC0B77A
:109F9000AEA69E97918B868582808080808080800F
:109FA00080808080808080808080808080808080B1
:109FB00080808080808080808080808080808080A1
:109FC0008080808080808080808080808080808091
:109FD0008080808080808080808080808080808081
:109FE0008080808080808080808080808080808071
:109FF000808080808087919DACC4CBD4DDF2FAFA5A
:10A0000022002400260028002B002D003000330001
:10A01000360039003D004000440048004C0051002B
:10A0200056005B00600066006C00730079008100E0
:10A03000880090009900A200AC00B600C100CC00DE
:10A04000D800E500F30001011001210132014401B3
:10A0500057016C0181019801B001CA01E5010202BA
:10A060002102410264028802AE02D70203033003D8
:10A0700061039403CB03050442048304C704100561
:10A080005D05AF0505066106C206290796070908A2
:10A09000830805098E09200ABA0A5D0B0A0CC10C57
:10A0A000840D510E2B0F121007110A121D134014AC
:10A0B0007415BA1614188319071BA31C571E2420E5
:10A0C0000E22142439267F28E82A752D29300633DC
:10A0D0000F364539AD3C49401B442848734CFE506F
:10A0E000CF55EA5A51600C661D6C8B725A7992807A
:10A0F00037885090E598FDA19FABD3B5A3C0000071
:10A10000A0E0B0E0E6E8F0E50C943E74EC01A88035
:10A11000B980CA80DB80A114B104C104D10441F428
:10A1200084E2A82E89EDB82E8BE5C82E87E0D82EC4
:10A13000C601B5012DE133EF41E050E00E941B74F0
:10A1400027EA31E440E050E00E94FC737B018C017F
:10A15000C601B5012DE133EF41E050E00E941B74D0
:10A16000CA01B9012CEE34EF4FEF5FEF0E94FC7390
:10A170006E0D7F1D801F911F97FF04C061507040BE
:10A1800080409048688379838A839B839B013F77D3
:10A19000C901CDB7DEB7EAE00C945A740E94805032
:10A1A000089586E091E00E9480500895A0E0B0E01C
:10A1B0008093060190930701A0930801B0930901D1
:10A1C00008956091EA0F7091EB0F4091E40F509168
:10A1D000E50FCA01817090709695982F8827979502
:10A1E0008795840F951F20E030E08F3F910519F08F
:10A1F00014F021E030E0F901E80FF11DCF014396A2
:10A2000020E030E08F3F910519F014F021E030E0BC
:10A2100090709093E50F8093E40FCB018170907064
:10A220009695982F882797958795860F971F820F69
:10A23000931F20E030E08F3F910519F014F021E0EA
:10A2400030E0280F311D559547954F775070240FFA
:10A25000351F30703093EB0F2093EA0F08959C0167
:10A26000009779F486E190E0689FF001699FF00D16
:10A27000789FF00D1124E40FF51FE55AF34F10827B
:10A280003BC08130910581F486E190E0689FF00148
:10A29000699FF00D789FF00D1124E40FF51FE55A2A
:10A2A000F34F81E080833DC08230910589F486E1DF
:10A2B00090E0689FF001699FF00D789FF00D1124E8
:10A2C000E40FF51FE55AF34F8091DB0F80833CC00C
:10A2D0008330910589F486E190E0689FF001699FE1
:10A2E000F00D789FF00D1124E40FF51FE55AF34FA0
:10A2F0008091E60F80833BC02430310591F486E1E4
:10A3000090E0689FF001699FF00D789FF00D112497
:10A31000E40FF51FE55AF34F88E080838093EC0F3C
:10A3200039C02530310581F486E190E0689FF00165
:10A33000699FF00D789FF00D1124E40FF51FE55A89
:10A34000F34F85E0808338C02630310581F486E103
:10A3500090E0689FF001699FF00D789FF00D112447
:10A36000E40FF51FE55AF34F81E4808337C02730AF
:10A37000310581F486E190E0689FF001699FF00D5E
:10A38000789FF00D1124E40FF51FE55AF34F86E98D
:10A39000808337C02830310579F486E190E0689FEA
:10A3A000F001699FF00D789FF00D1124E40FF51F67
:10A3B000E55AF34F86E923C02930310579F486E167
:10A3C00090E0689FF001699FF00D789FF00D1124D7
:10A3D000E40FF51FE55AF34F89E411C02B35310521
:10A3E00081F486E190E0689FF001699FF00D789F0D
:10A3F000F00D1124E40FF51FE55AF34F8BE5808330
:10A4000008952C35310579F486E190E0689FF001DC
:10A41000699FF00D789FF00D1124E40FF51FE55AA8
:10A42000F34F8CE580830895DC019B01FA01E2592A
:10A43000F348E491225030408E2F90E0BD01A901F5
:10A440000E942F5108953F924F925F926F927F9298
:10A450008F929F92AF92BF92CF92DF92EF92FF9234
:10A460000F931F93CF93DF93782E662E342E502EAA
:10A47000EE24FF24A22EBB24862E9924C42FD0E0E4
:10A4800021976E01C00ED11C219612C08701080DC4
:10A49000191DC801BE01472D50E00E941452C80189
:10A4A000B601472D50E00E9414520894E11CF11CA3
:10A4B000EA14FB045CF3EE24FF24452C5524C62D3E
:10A4C000D0E0832C992421976E01CA0CDB1C2196C5
:10A4D00012C08701080D191DCE01B801472D50E0AB
:10A4E0000E941452C601B801472D50E00E94145238
:10A4F0000894E11CF11CE414F5045CF3DF91CF91A6
:10A500001F910F91FF90EF90DF90CF90BF90AF9091
:10A510009F908F907F906F905F904F903F900895A5
:10A520002F923F924F925F926F927F928F929F9263
:10A53000AF92BF92CF92DF92EF92FF920F931F9351
:10A54000DF93CF93CDB7DEB727970FB6F894DEBF72
:10A550000FBECDBF982E362E242E802EE982CC241D
:10A56000DD24622E7724A02EBB24462E5524E42E13
:10A57000FF249501215030403B832A830894E10851
:10A58000F108C7018A0D9B1D9D838C830894E11CF3
:10A59000F11C36C0EE81FF81309729F02A813B8182
:10A5A000E217F30739F46E817F816E0D7F1DC801BC
:10A5B000492D06C06E817F816E0D7F1DC8014981C6
:10A5C00050E00E9414528E819F8101969F838E835A
:10A5D000EE81FF81EA15FB05ECF28601040D151DE5
:10A5E000C801B701492D50E00E941452C8016C8186
:10A5F0007D81492D50E00E9414520894C11CD11C49
:10A60000C614D70434F41F821E828601040D151D62
:10A61000DFCFEE24FF24A32CBB24422C5524089426
:10A62000410851086201C80CD11C0894411C511CFE
:10A6300012C087010A0D1B1DC801B201492D50E04F
:10A640000E941452C801B601492D50E00E941452D4
:10A650000894E11CF11CE614F7045CF3EE24FF24DB
:10A66000482C5524232D30E0A22CBB24215030400F
:10A670006901C60CD71C2F5F3F4F3F832E8313C049
:10A6800087010A0D1B1D8E819F81B801492D50E065
:10A690000E941452C601B801492D50E00E94145284
:10A6A0000894E11CF11CE414F50454F327960FB64A
:10A6B000F894DEBF0FBECDBFCF91DF911F910F91F8
:10A6C000FF90EF90DF90CF90BF90AF909F908F90D2
:10A6D0007F906F905F904F903F902F900895BF9222
:10A6E000CF92DF92EF92FF920F931F93CF93DF935E
:10A6F000B82EF62E142FE02FF0E0EE0FFF1FCF0143
:10A7000082549348C1E0D0E0C22EDD24E255F348E4
:10A71000E490FC0104910BC08F2D90E0612F70E05C
:10A720004B2D50E00E941452FE0C100F2196CC16B7
:10A73000DD0694F7DF91CF911F910F91FF90EF907D
:10A74000DF90CF90BF900895EF92FF920F931F93E9
:10A75000CF93DF93982F915020E030E040E050E01D
:10A76000692F70E008C02F5F3F4F849131968F3F73
:10A77000D1F74F5F5F4F4617570724F4F901EF5D9C
:10A78000F749F1CF992311F02F5F3F4FF901EC5DAD
:10A79000F749E491E093E40F1092E50F1092EB0F6C
:10A7A0001092EA0FC901099620910501213031F478
:10A7B000FC01E05EF749E491E093F00F019622304E
:10A7C00031F4FC01E05EF749E491E093F00F01966B
:10A7D000233031F4FC01E05EF749E491E093F00F9F
:10A7E0000196243031F4FC01E05EF749E491E093F6
:10A7F000F00F0196253030F0FC01E05EF749E4915E
:10A80000E093F00F0196213041F4FC01E05EF7493E
:10A81000E491E0932401109225010196223041F445
:10A82000FC01E05EF749E491E093240110922501D8
:10A830000196233041F4FC01E05EF749E491E09396
:10A840002401109225010196243041F4FC01E05EC0
:10A85000F749E491E09324011092250101962530F7
:10A8600040F0FC01E05EF749E491E093240110928E
:10A87000250106969093E90F8093E80FEC0124964A
:10A88000D093EE0FC093ED0F83E08093E10F11E0C2
:10A8900049C01092CC0F3CC01093CD0F6091E40FD3
:10A8A0007091E50F8091EA0F9091EB0F0E94E150BB
:10A8B0009091EA0F4091CD0F2091ED0F3091EE0F66
:10A8C000205E3749A091E80FB091E90FA05EB7492B
:10A8D00060E070E0F9018491981710F4FD01449153
:10A8E0006F5F7F4F2F5F3F4F11966430710591F777
:10A8F0004093CD0F6091E10F8091CC0F90E070E01C
:10A9000050E00E9414528091CC0F8F5F8093CC0F47
:10A910008091CC0F883208F4BFCF8091E10F8F5F18
:10A920008093E10F8091E10F883108F4B2CF249633
:10A930009EC0382F3F733093CD0F829586958695B4
:10A940008370813011F1813038F0823009F441C0D8
:10A95000833009F08BC067C0CE010196FC01E05E38
:10A96000F74924912093CC0FEC012196FE01E05E83
:10A97000F749E491E093E10F822F90E06E2F70E0B1
:10A98000432F50E00E94145271C0CE010196FC0189
:10A99000E05EF74964916093CC0F0196FC01E05EA4
:10A9A000F74944914093E10F0196FC01E05EF749BD
:10A9B0002491EC012196FE01E05EF749E491832F9A
:10A9C00090E070E050E030E00E2F10E00E946F53F6
:10A9D0004DC0CE010196FC01E05EF74964916093A1
:10A9E000CC0F0196FC01E05EF74944914093E10FE2
:10A9F0000196FC01E05EF74924910196FC01E05EBE
:10AA0000F7490491EC012196FE01E05EF749E491DB
:10AA1000832F90E070E050E030E010E0EE2EFF2455
:10AA20000E94905223C0CE010196FC01E05EF749DE
:10AA300064916093CC0F0196FC01E05EF74944916C
:10AA40004093E10F0196FC01E05EF7492491EC018F
:10AA50002196FE01E05EF749E491832F90E070E0DB
:10AA600050E030E00E2F10E00E9423522196FE01AC
:10AA7000E05EF74984918F3F09F05BCF87E090E07B
:10AA800060E070E042E050E028E230E006E110E0F3
:10AA90000E942352DF91CF911F910F91FF90EF9071
:10AAA0000895282F80E090E031E009C03083769649
:10AAB000E417F507D9F701968631910539F0FC01C5
:10AAC000E55AF34FAC014553504FF0CF213041F4DC
:10AAD00082E08093DB0F83E08093E60F81E0CBC0C0
:10AAE000223041F484E68093DB0F85E68093E60F05
:10AAF00082E0C1C0233041F486E68093DB0F87E615
:10AB00008093E60F83E0B7C0243051F430932201E4
:10AB100088E68093DB0F89E68093E60F84E0ABC084
:10AB2000253069F43093220186E08093F00F8AE6A5
:10AB30008093DB0F8BE68093E60F85E09CC0263088
:10AB400041F48CE68093DB0F8DE68093E60F86E080
:10AB500092C0273041F48EE68093DB0F8FE680931E
:10AB6000E60F87E088C0283041F480E78093DB0F50
:10AB700081E78093E60F88E07EC0293041F482E7C8
:10AB80008093DB0F83E78093E60F89E074C02A305F
:10AB900041F484E78093DB0F85E78093E60F8AE03A
:10ABA0006AC02B3041F486E78093DB0F87E7809300
:10ABB000E60F8BE060C02C3081F486E990E0909342
:10ABC0002501809324012093F00F88E78093DB0F09
:10ABD00089E78093E60F8CE04EC02D3041F486E685
:10ABE0008093DB0F87E68093E60F8DE044C02E3024
:10ABF00041F488E68093DB0F89E68093E60F8EE0D0
:10AC00003AC02F3089F484E190E09093250180933D
:10AC100024018EE08093F00F8AE68093DB0F8BE6B1
:10AC20008093E60F8FE027C0203141F48CE68093BB
:10AC3000DB0F8DE68093E60F80E11DC0213141F4EA
:10AC40008EE68093DB0F8FE68093E60F81E113C0E1
:10AC5000223141F480E78093DB0F81E78093E60F98
:10AC600082E109C0233151F482E78093DB0F83E74F
:10AC70008093E60F83E10E94A4530895243149F4A0
:10AC800084E78093DB0F85E78093E60F84E10E94E1
:10AC9000A45308952FE63CE080E090E046E150E0C8
:10ACA0000BC01192E217F307E1F701969F012A5EAC
:10ACB0003F4F8832910551F0849FF001859FF00D40
:10ACC000949FF00D1124E55AF34FEBCF08950F93A5
:10ACD0001F938091D50F90E06091DD0F70E040915F
:10ACE000D20F2091E30FFC01E20FF11D9F0106E15D
:10ACF00010E0209FF001219FF00D309FF00D1124F6
:10AD0000E55AF34FE60FF71FE40FF11D319740812D
:10AD1000552747FD50952091E70F420F511D440FD5
:10AD2000551F440F551F880F660F771F0E94D0488C
:10AD30008091D50F90E06091DD0F70E04091D20FCF
:10AD40002091E30FFC01E20FF11D9F01209FF00114
:10AD5000219FF00D309FF00D1124E55AF34FE60FBF
:10AD6000F71FE40FF11D31974081552747FD50959E
:10AD70002091E70F420F511D440F551F440F551FDF
:10AD80004F5F5F4F880F991F8F5F660F771F0E947D
:10AD9000D0488091D50F90E04091DD0F50E0BA018E
:10ADA000660F771F6F5FA091D20F2091E30FFC0118
:10ADB000E20FF11D9F01209FF001219FF00D309FB8
:10ADC000F00D1124E55AF34FE40FF51FEA0FF11DC2
:10ADD00031974081552747FD50952091E70F420F4D
:10ADE000511D440F551F440F551F4E5F5F4F880F75
:10ADF0000E94D0488091D50F90E04091DD0F50E047
:10AE0000BA01660F771F6F5FA091D20F2091E30FF9
:10AE1000FC01E20FF11D9F01209FF001219FF00D29
:10AE2000309FF00D1124E55AF34FE40FF51FEA0FA0
:10AE3000F11D31974081552747FD50952091E70F2F
:10AE4000420F511D440F551F440F551F4D5F5F4F5B
:10AE5000880F991F8F5F0E94D0488091E70F8F5F06
:10AE60008093E70F873010F01092E70F1F910F913A
:10AE700008957F928F929F92AF92BF92CF92DF926E
:10AE8000EF92FF920F931F93CF93DF9301E010E0B7
:10AE900055E0C52E46E0A42E36E1E32EF12C21E349
:10AEA000722E99E3892E45C18091E30FAE01480FC0
:10AEB000511D8091D20F9801280F311D4E9DF00138
:10AEC0004F9DF00D5E9DF00D1124E20FF31FE55A2A
:10AED000F34F9080892D86598A3018F089E3982E97
:10AEE00007C080912201882311F4808201C0708202
:10AEF0004E9DF0014F9DF00D5E9DF00D1124E20F6F
:10AF0000F31FE55AF34F8081482F552747FD509591
:10AF10008091EC0F90E04817590709F075C08091B7
:10AF2000DF0F480F511D440F551F440F551F8D2D26
:10AF30006C2D0E94D0482091D20F8091E30FAE017A
:10AF4000480F511D4E9DF0014F9DF00D5E9DF00D7F
:10AF50001124E55AF34FE00FF11FE20FF11D40817C
:10AF6000552747FD50958091DF0F480F511D440F25
:10AF7000551F440F551F4F5F5F4F8B2D6C2D0E9447
:10AF8000D0482091D20F8091E30FAE01480F511DA0
:10AF90004E9DF0014F9DF00D5E9DF00D1124E55A80
:10AFA000F34FE00FF11FE20FF11D4081552747FDE0
:10AFB00050958091DF0F480F511D440F551F440FCE
:10AFC000551F4E5F5F4F8D2D6A2D0E94D0482091F6
:10AFD000D20F8091E30FAE01480F511D4E9DF0013D
:10AFE0004F9DF00D5E9DF00D1124E55AF34FE00FDB
:10AFF000F11FE20FF11D4081552747FD50958091CB
:10B00000DF0F480F511D64C0440F551F440F551FDB
:10B010008D2D6C2D0E94D0482091D20F8091E30F8E
:10B02000AE01480F511D4E9DF0014F9DF00D5E9DEC
:10B03000F00D1124E55AF34FE00FF11FE20FF11D5F
:10B040004081552747FD5095440F551F440F551F0C
:10B050004F5F5F4F8B2D6C2D0E94D0482091D20FF7
:10B060008091E30FAE01480F511D4E9DF0014F9DA1
:10B07000F00D5E9DF00D1124E55AF34FE00FF11F26
:10B08000E20FF11D4081552747FD5095440F551F94
:10B09000440F551F4E5F5F4F8D2D6A2D0E94D04883
:10B0A0002091D20F8091E30FAE01480F511D4E9DAC
:10B0B000F0014F9DF00D5E9DF00D1124E55AF34F08
:10B0C000E00FF11FE20FF11D4081552747FD50951C
:10B0D000440F551F440F551F4D5F5F4F8B2D6A2D39
:10B0E0000E94D04859E39516A9F02091D20F809183
:10B0F000E30FAE01480F511D4E9DF0014F9DF00D25
:10B100005E9DF00D1124E55AF34FE00FF11FE20FA1
:10B11000F11D9082219652E0D50EB50E88E2D81628
:10B1200009F0C2CE0F5F1F4FC50EA50E4BE1C4162E
:10B1300031F0C0E0D0E0DD24BB24B394B5CEDF9184
:10B14000CF911F910F91FF90EF90DF90CF90BF9024
:10B15000AF909F908F907F9008957F928F929F9253
:10B16000AF92BF92CF92DF92EF92FF920F931F9315
:10B17000CF93DF9301E010E063E0C62E54E0A52EEC
:10B1800046E1E42EF12C31E3732E29E3822E45C1F2
:10B190008091E30FAE01480F511D8091D20F9801AD
:10B1A000280F311D4E9DF0014F9DF00D5E9DF00D5D
:10B1B0001124E20FF31FE55AF34F9080892D865931
:10B1C0008A3018F099E3992E07C0809122018823D4
:10B1D00011F4808201C070824E9DF0014F9DF00DF0
:10B1E0005E9DF00D1124E20FF31FE55AF34F8081AD
:10B1F000482F552747FD50958091EC0F90E0481758
:10B20000590709F075C08091DF0F480F511D440F99
:10B21000551F440F551F8D2D6C2D0E94D048209135
:10B22000D20F8091E30FAE01480F511D4E9DF001EA
:10B230004F9DF00D5E9DF00D1124E55AF34FE00F88
:10B24000F11FE20FF11D4081552747FD5095809178
:10B25000DF0F480F511D440F551F440F551F4F5FFF
:10B260005F4F8B2D6C2D0E94D0482091D20F809182
:10B27000E30FAE01480F511D4E9DF0014F9DF00DA3
:10B280005E9DF00D1124E55AF34FE00FF11FE20F20
:10B29000F11D4081552747FD50958091DF0F480FE4
:10B2A000511D440F551F440F551F4E5F5F4F8D2D8D
:10B2B0006A2D0E94D0482091D20F8091E30FAE01F9
:10B2C000480F511D4E9DF0014F9DF00D5E9DF00DFC
:10B2D0001124E55AF34FE00FF11FE20FF11D4081F9
:10B2E000552747FD50958091DF0F480F511D64C0D1
:10B2F000440F551F440F551F8D2D6C2D0E94D048B3
:10B300002091D20F8091E30FAE01480F511D4E9D49
:10B31000F0014F9DF00D5E9DF00D1124E55AF34FA5
:10B32000E00FF11FE20FF11D4081552747FD5095B9
:10B33000440F551F440F551F4F5F5F4F8B2D6C2DD2
:10B340000E94D0482091D20F8091E30FAE01480FA8
:10B35000511D4E9DF0014F9DF00D5E9DF00D11248D
:10B36000E55AF34FE00FF11FE20FF11D4081552721
:10B3700047FD5095440F551F440F551F4E5F5F4FBB
:10B380008D2D6A2D0E94D0482091D20F8091E30F1D
:10B39000AE01480F511D4E9DF0014F9DF00D5E9D79
:10B3A000F00D1124E55AF34FE00FF11FE20FF11DEC
:10B3B0004081552747FD5095440F551F440F551F99
:10B3C0004D5F5F4F8B2D6A2D0E94D04859E3951633
:10B3D000A9F02091D20F8091E30FAE01480F511DCB
:10B3E0004E9DF0014F9DF00D5E9DF00D1124E55A2C
:10B3F000F34FE00FF11FE20FF11D9082219652E012
:10B40000D50EB50E88E2D81609F0C2CE0F5F1F4FD9
:10B41000C50EA50E49E1C41631F0C0E0D0E0DD2430
:10B42000BB24B394B5CEDF91CF911F910F91FF90C4
:10B43000EF90DF90CF90BF90AF909F908F907F90D4
:10B4400008957F928F929F92AF92BF92CF92DF9298
:10B45000EF92FF920F931F93CF93DF9300E010E0E2
:10B46000B2E0CB2EA3E0AA2EF6E1EF2EF12CE1E321
:10B470007E2E79E3872E45C18091E30FAE01480F00
:10B48000511D8091D20F9801280F311D4E9DF00162
:10B490004F9DF00D5E9DF00D1124E20FF31FE55A54
:10B4A000F34F9080892D86598A3018F069E3962EE3
:10B4B00007C080912201882311F4808201C070822C
:10B4C0004E9DF0014F9DF00D5E9DF00D1124E20F99
:10B4D000F31FE55AF34F8081482F552747FD5095BC
:10B4E0008091EC0F90E04817590709F075C08091E2
:10B4F000DF0F480F511D440F551F440F551F8D2D51
:10B500006C2D0E94D0482091D20F8091E30FAE01A4
:10B51000480F511D4E9DF0014F9DF00D5E9DF00DA9
:10B520001124E55AF34FE00FF11FE20FF11D4081A6
:10B53000552747FD50958091DF0F480F511D440F4F
:10B54000551F440F551F4F5F5F4F8B2D6C2D0E9471
:10B55000D0482091D20F8091E30FAE01480F511DCA
:10B560004E9DF0014F9DF00D5E9DF00D1124E55AAA
:10B57000F34FE00FF11FE20FF11D4081552747FD0A
:10B5800050958091DF0F480F511D440F551F440FF8
:10B59000551F4E5F5F4F8D2D6A2D0E94D048209120
:10B5A000D20F8091E30FAE01480F511D4E9DF00167
:10B5B0004F9DF00D5E9DF00D1124E55AF34FE00F05
:10B5C000F11FE20FF11D4081552747FD50958091F5
:10B5D000DF0F480F511D64C0440F551F440F551F06
:10B5E0008D2D6C2D0E94D0482091D20F8091E30FB9
:10B5F000AE01480F511D4E9DF0014F9DF00D5E9D17
:10B60000F00D1124E55AF34FE00FF11FE20FF11D89
:10B610004081552747FD5095440F551F440F551F36
:10B620004F5F5F4F8B2D6C2D0E94D0482091D20F21
:10B630008091E30FAE01480F511D4E9DF0014F9DCB
:10B64000F00D5E9DF00D1124E55AF34FE00FF11F50
:10B65000E20FF11D4081552747FD5095440F551FBE
:10B66000440F551F4E5F5F4F8D2D6A2D0E94D048AD
:10B670002091D20F8091E30FAE01480F511D4E9DD6
:10B68000F0014F9DF00D5E9DF00D1124E55AF34F32
:10B69000E00FF11FE20FF11D4081552747FD509546
:10B6A000440F551F440F551F4D5F5F4F8B2D6A2D63
:10B6B0000E94D04859E39516A9F02091D20F8091AD
:10B6C000E30FAE01480F511D4E9DF0014F9DF00D4F
:10B6D0005E9DF00D1124E55AF34FE00FF11FE20FCC
:10B6E000F11D9082219652E0D50EB50E87E2D81654
:10B6F00009F0C2CE0F5F1F4FC50EA50E4CE1C41658
:10B7000039F0C0E0D0E0DD24D39472E0B72EB4CE9F
:10B71000DF91CF911F910F91FF90EF90DF90CF902D
:10B72000BF90AF909F908F907F9008957F928F925F
:10B730009F92AF92BF92CF92DF92EF92FF920F93C0
:10B740001F93CF93DF9300E010E062E0E62E53E01A
:10B75000A52E46E1C42ED12C31E3832E29E3722E8F
:10B7600074C18091E30FAE01480F511D8091D20F3B
:10B770009801280F311D4C9DF0014D9DF00D5C9DF1
:10B78000F00D1124E20FF31FE55AF34F9080892D3D
:10B7900086598A3018F099E3992E07C080912201CA
:10B7A000882311F4708201C080824C9DF0014D9D70
:10B7B000F00D5C9DF00D1124E20FF31FE55AF34FDD
:10B7C0008081482F552747FD50958091EC0F90E0E0
:10B7D0004817590709F075C08091DF0F480F511DB8
:10B7E000440F551F440F551F8F2D6E2D0E94D048BA
:10B7F0002091D20F8091E30FAE01480F511D4C9D57
:10B80000F0014D9DF00D5C9DF00D1124E55AF34FB4
:10B81000E00FF11FE20FF11D4081552747FD5095C4
:10B820008091DF0F480F511D440F551F440F551FC6
:10B830004F5F5F4F8B2D6E2D0E94D0482091D20F0D
:10B840008091E30FAE01480F511D4C9DF0014D9DBD
:10B85000F00D5C9DF00D1124E55AF34FE00FF11F40
:10B86000E20FF11D4081552747FD50958091DF0F74
:10B87000480F511D440F551F440F551F4E5F5F4F1A
:10B880008F2D6A2D0E94D0482091D20F8091E30F16
:10B89000AE01480F511D4C9DF0014D9DF00D5C9D7A
:10B8A000F00D1124E55AF34FE00FF11FE20FF11DE7
:10B8B0004081552747FD50958091DF0F480F511D5E
:10B8C00093C08091D60F90E04817590749F54091F1
:10B8D000E60F50E0440F551F440F551F8F2D6E2D5E
:10B8E0000E94D0484091E60F50E0440F551F440F8E
:10B8F000551F4F5F5F4F8B2D6E2D0E94D04840919A
:10B90000E60F50E0440F551F440F551F4E5F5F4F29
:10B910008F2D6A2D0E94D0484091E60F50E064C000
:10B92000440F551F440F551F8F2D6E2D0E94D04878
:10B930002091D20F8091E30FAE01480F511D4C9D15
:10B94000F0014D9DF00D5C9DF00D1124E55AF34F73
:10B95000E00FF11FE20FF11D4081552747FD509583
:10B96000440F551F440F551F4F5F5F4F8B2D6E2D9A
:10B970000E94D0482091D20F8091E30FAE01480F72
:10B98000511D4C9DF0014D9DF00D5C9DF00D11245D
:10B99000E55AF34FE00FF11FE20FF11D40815527EB
:10B9A00047FD5095440F551F440F551F4E5F5F4F85
:10B9B0008F2D6A2D0E94D0482091D20F8091E30FE5
:10B9C000AE01480F511D4C9DF0014D9DF00D5C9D49
:10B9D000F00D1124E55AF34FE00FF11FE20FF11DB6
:10B9E0004081552747FD5095440F551F440F551F63
:10B9F0004D5F5F4F8B2D6A2D0E94D04859E39516FD
:10BA0000A9F02091D20F8091E30FAE01480F511D94
:10BA10004C9DF0014D9DF00D5C9DF00D1124E55AFB
:10BA2000F34FE00FF11FE20FF11D9082219652E0DB
:10BA3000F50EB50E87E2F81609F093CE0F5F1F4F93
:10BA4000E50EA50E4CE1E41639F0C1E0D0E0FF248C
:10BA5000F39482E0B82E85CEDF91CF911F910F91A4
:10BA6000FF90EF90DF90CF90BF90AF909F908F901E
:10BA70007F9008952091E30F8091D50F90E0821B75
:10BA8000910940973CF0243128F42F5F2093E30F75
:10BA90000E94215A2091E30F8091D50F90E0821BE4
:10BAA000910905973CF4222329F021502093E30FBC
:10BAB0000E94965B2091D20F8091DD0F90E0821B57
:10BAC000910909974CF0293038F40E94AD588091C3
:10BAD000D20F8F5F8093D20F2091D20F8091DD0F14
:10BAE00090E0821B910903974CF4222339F00E94C5
:10BAF00039578091D20F81508093D20F08957F9251
:10BB00008F929F92AF92BF92CF92DF92EF92FF926D
:10BB10000F931F93CF93DF9300E010E082E0E82EB5
:10BB2000B3E0AB2EA6E1CA2ED12CF1E37F2EE9E3E0
:10BB30008E2E88C18091E30FAE01480F511D809178
:10BB4000D20F9801280F311D4C9DF0014D9DF00D35
:10BB50005C9DF00D1124E20FF31FE55AF34F908026
:10BB6000892D86598A3018F079E3972E07C0809185
:10BB70002201882311F4808201C070824C9DF00163
:10BB80004D9DF00D5C9DF00D1124E20FF31FE55A61
:10BB9000F34FE0814E2F552747FD50958091EC0FD4
:10BBA00090E048175907A9F080915A0C90E0481787
:10BBB000590779F0E83169F0E03159F0E93249F09C
:10BBC000E13339F0E93329F0E13419F0E93409F0CF
:10BBD00075C08091DF0F480F511D440F551F440F52
:10BBE000551F8F2D6E2D0E94D0482091D20F80912D
:10BBF000E30FAE01480F511D4C9DF0014D9DF00D1E
:10BC00005C9DF00D1124E55AF34FE00FF11FE20F98
:10BC1000F11D4081552747FD50958091DF0F480F5A
:10BC2000511D440F551F440F551F4F5F5F4F8B2D04
:10BC30006E2D0E94D0482091D20F8091E30FAE016B
:10BC4000480F511D4C9DF0014D9DF00D5C9DF00D78
:10BC50001124E55AF34FE00FF11FE20FF11D40816F
:10BC6000552747FD50958091DF0F480F511D440F18
:10BC7000551F440F551F4E5F5F4F8F2D6A2D0E9439
:10BC8000D0482091D20F8091E30FAE01480F511D93
:10BC90004C9DF0014D9DF00D5C9DF00D1124E55A79
:10BCA000F34FE00FF11FE20FF11D4081552747FDD3
:10BCB00050958091DF0F480F511D93C08091D60F92
:10BCC00090E04817590749F54091E60F50E0440FBE
:10BCD000551F440F551F8F2D6E2D0E94D048409147
:10BCE000E60F50E0440F551F440F551F4F5F5F4F45
:10BCF0008B2D6E2D0E94D0484091E60F50E0440FEE
:10BD0000551F440F551F4E5F5F4F8F2D6A2D0E94A8
:10BD1000D0484091E60F50E064C0440F551F440FD7
:10BD2000551F8F2D6E2D0E94D0482091D20F8091EB
:10BD3000E30FAE01480F511D4C9DF0014D9DF00DDC
:10BD40005C9DF00D1124E55AF34FE00FF11FE20F57
:10BD5000F11D4081552747FD5095440F551F440F55
:10BD6000551F4F5F5F4F8B2D6E2D0E94D048209145
:10BD7000D20F8091E30FAE01480F511D4C9DF00191
:10BD80004D9DF00D5C9DF00D1124E55AF34FE00F31
:10BD9000F11FE20FF11D4081552747FD5095440FDB
:10BDA000551F440F551F4E5F5F4F8F2D6A2D0E9408
:10BDB000D0482091D20F8091E30FAE01480F511D62
:10BDC0004C9DF0014D9DF00D5C9DF00D1124E55A48
:10BDD000F34FE00FF11FE20FF11D4081552747FDA2
:10BDE0005095440F551F440F551F4D5F5F4F8B2DCE
:10BDF0006A2D0E94D04859E39516A9F02091D20FE0
:10BE00008091E30FAE01480F511D4C9DF0014D9DF7
:10BE1000F00D5C9DF00D1124E55AF34FE00FF11F7A
:10BE2000E20FF11D9082219652E0F50EB50E88E2E8
:10BE3000F81609F07FCE0F5F1F4FE50EA50E4CE1FF
:10BE4000E41631F0C0E0D0E0FF24BB24B39472CEFE
:10BE5000DF91CF911F910F91FF90EF90DF90CF90E6
:10BE6000BF90AF909F908F907F900895AF92BF92B8
:10BE7000CF92DF92EF92FF920F931F93CF93DF93B6
:10BE800085E06FEF41E00E94BE7080E79CE00E9479
:10BE9000F44800E00CC0802F612F40E050E00E9489
:10BEA000D0481F5F1C31B9F70F5F083211F012E064
:10BEB000F2CF84E690E02BEC32E0F9013197F1F714
:10BEC0000197D9F780EA9CE00E94F448C1E0D0E0F5
:10BED000E3E0DE2E76E1A72EB12C95C02091D20FA3
:10BEE0008091E30FAE01480F511D4A9DF0014B9D1B
:10BEF000F00D5A9DF00D1124E55AF34FEE0DFF1D84
:10BF0000E20FF11D4081552747FD5095440F551F05
:10BF1000440F551F8C2D602F0E94D0482091D20FC6
:10BF20008091E30FAE01480F511D4A9DF0014B9DDA
:10BF3000F00D5A9DF00D1124E55AF34FEE0DFF1D43
:10BF4000E20FF11D4081552747FD5095440F551FC5
:10BF5000440F551F4F5F5F4F8D2D602F0E94D048BB
:10BF6000102F1F5F2091D20F8091E30FAE01480F79
:10BF7000511D4A9DF0014B9DF00D5A9DF00D11246D
:10BF8000E55AF34FEE0DFF1DE20FF11D40815527DD
:10BF900047FD5095440F551F440F551F4E5F5F4F8F
:10BFA0008C2D612F0E94D0482091D20F8091E30FF9
:10BFB000AE01480F511D4A9DF0014B9DF00D5A9D59
:10BFC000F00D1124E55AF34FEE0DFF1DE20FF11DA8
:10BFD0004081552747FD5095440F551F440F551F6D
:10BFE0004D5F5F4F8D2D612F0E94D0480894E11C5A
:10BFF000F11C0E5F0A3109F071CF219652E0D50E87
:10C0000089E2D81639F0AE01440FC42EEE24FF2485
:10C0100002E064CFDF91CF911F910F91FF90EF90DD
:10C02000DF90CF90BF90AF900895FF920F931F9332
:10C03000CF93DF93F82EEB018A0185E06FEF41E0AB
:10C040000E94BE709E012150304086E190E0289F02
:10C05000F001299FF00D389FF00D1124E00FF11F22
:10C06000E55AF34F8081813009F0F082D8011196B2
:10C0700086E190E0289FF001299FF00D389FF00D98
:10C080001124EA0FFB1FE55AF34F8081813009F03C
:10C09000F082A8014150504086E190E0289FF001D5
:10C0A000299FF00D389FF00D1124E40FF51FE55A7C
:10C0B000F34F8081813009F0F08286E190E0C89FE3
:10C0C000F001C99FF00DD89FF00D1124E00FF11F72
:10C0D000E55AF34F8081813009F0F08286E190E0EB
:10C0E000C89FF001C99FF00DD89FF00D1124EA0FF1
:10C0F000FB1FE55AF34F8081813009F0F08286E121
:10C1000090E0C89FF001C99FF00DD89FF00D112459
:10C11000E40FF51FE55AF34F8081813009F0F0827A
:10C12000BE016F5F7F4F86E190E0689FF001699FDD
:10C13000F00D789FF00D1124E00FF11FE55AF34F39
:10C140008081813009F0F08286E190E0689FF00103
:10C15000699FF00D789FF00D1124EA0FFB1FE55A3F
:10C16000F34F8081813009F0F08286E190E0689F92
:10C17000F001699FF00D789FF00D1124E40FF51F79
:10C18000E55AF34F8081813009F0F082DF91CF9141
:10C190001F910F91FF9008959C01AB0181E290E007
:10C1A000B9010E94156008959C01AB0187E590E0FC
:10C1B000B9010E94156008959C01AB0183E590E0F0
:10C1C000B9010E9415600895CF93DF932091DD0F90
:10C1D0008091D50F90E0C6E1D0E08C9FF0018D9F5B
:10C1E000F00D9C9FF00D1124E20FF11DE55AF34F65
:10C1F0002081332727FD30958091EC0F90E02817A0
:10C200003907B9F5809120018F5F8093200120913B
:10C21000D70F3091D80F4091D90F5091DA0F2C5988
:10C220003F4F4F4F5F4F2093D70F3093D80F40931E
:10C23000D90F5093DA0F9091F00F8917A9F40E944B
:10C24000365F2091DE0F8091DC0F90E08C9FF00133
:10C250008D9FF00D9C9FF00D1124E20FF11DE55A0A
:10C26000F34F8BE5808305C081E06FEF41E00E94D2
:10C27000BE702091DD0F8091D50F90E0C6E1D0E037
:10C280008C9FF0018D9FF00D9C9FF00D1124E20F0B
:10C29000F11DE55AF34F2081332727FD309580911A
:10C2A000CE0F90E028173907B9F5809120018F5FF4
:10C2B000809320012091D70F3091D80F4091D90F52
:10C2C0005091DA0F2C593F4F4F4F5F4F2093D70FAC
:10C2D0003093D80F4093D90F5093DA0F9091F00F0D
:10C2E0008917A9F40E94365F2091DE0F8091DC0F40
:10C2F00090E08C9FF0018D9FF00D9C9FF00D11241C
:10C30000E20FF11DE55AF34F8BE5808305C081E014
:10C310006FEF41E00E94BE708091D50F482F50E032
:10C320008091DD0F682F70E086E190E0489FF0017A
:10C33000499FF00D589FF00D1124E60FF71FE55AA5
:10C34000F34F2081332727FD30958091D60F90E061
:10C350002817390729F410920101CA010E94CC6004
:10C360008091D50F482F50E08091DD0F682F70E04D
:10C3700086E190E0489FF001499FF00D589FF00D35
:10C380001124E60FF71FE55AF34F2081332727FDCD
:10C3900030958091CF0F90E02817390729F410923B
:10C3A0000101CA010E94CC608091D50F282F30E096
:10C3B0008091DD0F682F70E086E190E0289FF0010A
:10C3C000299FF00D389FF00D1124E60FF71FE55A55
:10C3D000F34FE081EB3519F481E08093E00FE659EB
:10C3E000E53068F41092010180912201882321F444
:10C3F000C9010E94CC6003C0C9010E94D460DF91D2
:10C40000CF91089580E090E061E070E046ED5CE758
:10C410000E94DB718BE090E061E070E040912001D0
:10C420000E944A7280E090E060E070E040EE5CE7DD
:10C430000E94DB71809124019091250168E070E0F9
:10C440000E94B373462F8BE090E060E070E00E94A2
:10C450004A728DE090E060E070E04BEF5CE70E9494
:10C46000DB7185E190E060E070E0409102010E94A4
:10C470004A728DE090E061E070E04DEE5CE70E9472
:10C48000DB7185E190E061E070E0409100010E9485
:10C490004A7287E190E060E070E044EF5CE70E9460
:10C4A000DB712091D70F3091D80F4091D90F509167
:10C4B000DA0F83E290E060E070E00E947572089508
:10C4C0006F927F928F929F92AF92BF92CF92DF92A4
:10C4D000EF92FF920F931F93CF93DF93CC24DD2431
:10C4E00026E1A22EB12C94E6692E712CB4C08F5F88
:10C4F0008B3F09F097C02091D20F8091E30FAE01DE
:10C50000480F511D4A9DF0014B9DF00D5A9DF00DB5
:10C510001124E55AF34FEE0DFF1DE20FF11D40818E
:10C52000552747FD5095440F551F440F551F882D23
:10C53000602F0E94D0482091D20F8091E30FAE016E
:10C54000480F511D4A9DF0014B9DF00D5A9DF00D75
:10C550001124E55AF34FEE0DFF1DE20FF11D40814E
:10C56000552747FD5095440F551F440F551F4F5FEA
:10C570005F4F812F602F0E94D048902E939420917E
:10C58000D20F8091E30FAE01480F511D4A9DF0017B
:10C590004B9DF00D5A9DF00D1124E55AF34FEE0D11
:10C5A000FF1DE20FF11D4081552747FD5095440FB7
:10C5B000551F440F551F4E5F5F4F882D692D0E94F8
:10C5C000D0482091D20F8091E30FAE01480F511D4A
:10C5D0004A9DF0014B9DF00D5A9DF00D1124E55A36
:10C5E000F34FEE0DFF1DE20FF11D4081552747FD72
:10C5F0005095440F551F440F551F4D5F5F4F812FBE
:10C60000692D0E94D0480E94D150869DA001879D2F
:10C61000500D969D500D112481E061E028EC0E94A0
:10C62000D56D80E00894E11CF11C0E5F0A3109F021
:10C630005ECF21961E5F193239F09E01220F822EA5
:10C64000EE24FF2402E053CF0894C11CD11C38EC27
:10C65000C316D10421F0C1E0D0E013E0EECFDF91AA
:10C66000CF911F910F91FF90EF90DF90CF90BF90EF
:10C67000AF909F908F907F906F900895EF92FF9270
:10C680000F931F93CF93DF93C0E0D0E034E6E32E07
:10C69000F12C27C08F5F873FB9F41230A0F0802FB4
:10C6A000612F44E050E00E94D0480E94D1508E9DFE
:10C6B000A0018F9D500D9E9D500D112481E061E0E1
:10C6C00028EC0E94D56D80E01F5F1C3119F70F5FC9
:10C6D000083211F010E0DECF219691E0C039D90781
:10C6E00011F000E0F7CFDF91CF911F910F91FF90F4
:10C6F000EF9008950F931F93CF93DF9380E00E94F4
:10C7000000499C011091D50FC12FD0E00091DD0FA1
:10C71000602F70E046E150E0C49FF001C59FF00D2E
:10C72000D49FF00D1124DF01A60FB71FA55AB34FF8
:10C7300080E28C9325FF99C01C92812F81508093B9
:10C74000D50F90E0849FF001859FF00D949FF00D30
:10C750001124E60FF71FE55AF34FE0812E2F332700
:10C7600027FD30958091E20F90E02817390741F0BE
:10C770008091EF0F90E02817390711F0E13419F498
:10C780001093D50F05C082E060E541E00E94BE70C5
:10C790008091D50F482F50E08091DD0F682F70E019
:10C7A000C6E1D0E04C9FF0014D9FF00D5C9FF00D75
:10C7B0001124E60FF71FE55AF34F2081332727FD99
:10C7C00030958091E60F90E028173907C1F5415068
:10C7D00050404C9FF0014D9FF00D5C9FF00D1124D7
:10C7E000E60FF71FE55AF34F8081882319F50E9461
:10C7F000D1509C0173E0880F991F7A95E1F7220FC1
:10C80000331F820F931F0997ACF02091DD0F8091A9
:10C81000D50F90E001978C9FF0018D9FF00D9C9FAC
:10C82000F00D1124E20FF11DE55AF34F8091E60F50
:10C83000808305C08091D50F8F5F8093D50F0E94B4
:10C84000E4604091DD0F8091D50F90E026E130E06B
:10C85000829FF001839FF00D929FF00D1124E40F51
:10C86000F11DE55AF34F80E19AC024FF9CC01C9251
:10C87000812F8F5F8093D50F90E0849FF001859F7B
:10C88000F00D949FF00D1124E60FF71FE55AF34FBA
:10C89000E0812E2F332727FD30958091E20F90E025
:10C8A0002817390741F08091EF0F90E028173907DA
:10C8B00011F0E13419F41093D50F05C082E060E562
:10C8C00041E00E94BE708091D50F482F50E08091CA
:10C8D000DD0F682F70E0C6E1D0E04C9FF0014D9F66
:10C8E000F00D5C9FF00D1124E60FF71FE55AF34F92
:10C8F0002081332727FD30958091E60F90E028179F
:10C900003907C1F54F5F5F4F4C9FF0014D9FF00D10
:10C910005C9FF00D1124E60FF71FE55AF34F80815D
:10C92000882319F50E94D1509C0153E0880F991F6C
:10C930005A95E1F7220F331F820F931F0897ACF02F
:10C940002091DD0F8091D50F90E001968C9FF00132
:10C950008D9FF00D9C9FF00D1124E20FF11DE55A03
:10C96000F34F8091E60F808305C08091D50F8150F1
:10C970008093D50F0E94E4604091DD0F8091D50F28
:10C9800090E026E130E0829FF001839FF00D929FBE
:10C99000F00D1124E40FF11DE55AF34F88E1808377
:10C9A0008093D40F51C027FF04C01C92802F815068
:10C9B00005C026FF42C01C92802F8F5F8093DD0F41
:10C9C000E80FF11DE55AF34FE0812E2F332727FDA5
:10C9D00030958091E20F90E02817390771F080912F
:10C9E000EF0F90E02817390741F08091E60F90E0B3
:10C9F0002817390711F0E13419F40093DD0F05C051
:10CA000082E060E541E00E94BE700E94E4604091D7
:10CA1000DD0F8091D50F90E026E130E0829FF0019C
:10CA2000839FF00D929FF00D1124E40FF11DE55A44
:10CA3000F34F8091D40F808307C030FF05C0CE0133
:10CA40000E94DC6010920101DF91CF911F910F9144
:10CA500008952F923F924F925F926F927F928F92A2
:10CA60009F92AF92BF92CF92DF92EF92FF920F937D
:10CA70001F93DF93CF93CDB7DEB727970FB6F89408
:10CA8000DEBF0FBECDBF0E947F5D1092D10F10920E
:10CA9000D00F10922301CC24DD2481E08A83AFEFF4
:10CAA000BFEFBC83AB8316E1612E712CD6C3FA2C89
:10CAB000809121018F5F80932101863010F01092C8
:10CAC00021018091D50F90E02091DD0F869DF0012E
:10CAD000879DF00D969DF00D1124E20FF11DE55A92
:10CAE000F34F40801082EE81FF81E0802E2D3327AE
:10CAF00027FD30958091CF0F90E02817390709F076
:10CB0000A7C08091D00F9091D10F01969093D10F33
:10CB10008093D00F46898091DB0F282F30E0842F3F
:10CB2000992787FD90958217930711F0442319F4F4
:10CB3000F1E0F0932301D8014C91842F992787FDD0
:10CB400090958217930711F0442319F4B1E0B09344
:10CB50002301F8014789842F992787FD9095821733
:10CB6000930711F0442319F4F1E0F0932301D80165
:10CB700055964C91842F992787FD9095821793079E
:10CB800011F0442319F4B1E0B09323010E94D15075
:10CB9000EAE08E9F502D1124852F81508230A8F419
:10CBA000AE81BF8156964C91242F332727FD3095B7
:10CBB0008091DB0F90E02817390711F0442329F406
:10CBC0008091CF0FEE81FF81868B852F835082303D
:10CBD00090F4D8014C91242F332727FD3095809174
:10CBE000DB0F90E02817390711F0442321F48091DE
:10CBF000CF0FF8018083852F8550823098F4D801BB
:10CC000057964C91242F332727FD30958091DB0FC9
:10CC100090E02817390711F0442321F48091CF0FB9
:10CC2000F801878B5750523098F4D80155964C91A3
:10CC3000242F332727FD30958091DB0F90E02817B4
:10CC4000390711F0442321F48091CF0FF801858B2F
:10CC5000F6E9EF1631F030E060E087E9E81611F50B
:10CC60000DC0D80157968C915797882389F1F80108
:10CC700080818823B1F580EA808306C0D8018C9139
:10CC8000882339F4E0EAEC93AE81BF811C923D81A8
:10CC90004EC0F8018589882319F481EA858B32C05A
:10CCA00083EA20C099E9E91609F5AE81BF8156965D
:10CCB0008C915697882331F4E2EA5696EC93569776
:10CCC0001C922EC0D80157968C915797882349F40F
:10CCD000E3EA5796EC93AE81BF811C92682D352D07
:10CCE00027C081EAEE81FF81808320C098E9E916A0
:10CCF000F9F4D80155968C915597882349F4E1EAC7
:10CD00005596EC93AE81BF811C92352D698110C080
:10CD1000EE81FF818689882329F482EA868B10823E
:10CD20003A8105C0E0EAAE81BF81EC93352D6F2DCD
:10CD30002091D50F4091DD0F822F90E0869DF0016C
:10CD4000879DF00D969DF00D1124E40FF11DE55A1D
:10CD5000F34F40823217B9F46417A9F480910101AE
:10CD6000813089F480912201882331F4832F90E06F
:10CD700070E00E94CC6005C0832F90E070E00E94BC
:10CD8000D46010920101AE81BF818C91833574F122
:10CD9000863509F41C92EE81FF818081853511F47E
:10CDA00086E58083AE81BF818C91843511F4E5E501
:10CDB000EC93AE81BF818C91833511F4E4E5EC9363
:10CDC000AE81BF818C91893519F48091EC0F8C93E1
:10CDD000EE81FF818081883511F489E58083AE8101
:10CDE000BF818C91873511F4E8E5EC93AE81BF816A
:10CDF0008C91833219F48091E60F8C93EE81FF8140
:10CE00008081823211F483E28083AE81BF818C9174
:10CE1000813211F4E2E2EC93AE81BF812C91332791
:10CE200027FD30958091E60F90E028173907C9F467
:10CE3000B401F8018789882319F41C9281E6878B55
:10CE4000D80157968C9186598A3058F480912201E6
:10CE5000882321F4C6010E94CC6003C0C6010E9451
:10CE6000D460EE81FF812081332727FD30958091AA
:10CE7000D60F90E02817390709F083C0F82CE92C69
:10CE8000D80157968C915797813419F558962C9163
:10CE9000222349F0332727FD30958091DB0F90E066
:10CEA00028173907B1F4C69CF001C79CF00DD69C39
:10CEB000F00D1124AE0EBF1E8BE59CE0A80EB91E2E
:10CEC000D5011C92E20DF31DE80FF91F8091EC0FC4
:10CED000A0C08091D50F90E02091DD0F869DF001DC
:10CEE000879DF00D969DF00D1124E20FF11DE55A7E
:10CEF000F34F4080B3E6B083F8018789882331F48B
:10CF0000AE81BF811C92B1E6B78B0AC08091E60F5B
:10CF1000EE81FF81808384E06FEF40E00E94BE706D
:10CF2000D80157968C91833639F4C6016F2D7E2D2A
:10CF30000E94DC6010920101F801878986598A30CD
:10CF400078F480912201882331F4C6016F2D7E2D63
:10CF50000E94CC6005C0C6016F2D7E2D0E94D4605A
:10CF60008091DD0F2091D50F30E0269DF001279DA7
:10CF7000F00D369DF00D1124E80FF11DE55AF34F29
:10CF800040824091EC0FAE81BF818C91992787FD43
:10CF90009095242F30E08217930739F4F8018789A0
:10CFA000882319F41C9282E6878BAE81BF812C9175
:10CFB000332727FD30958091CE0F90E02817390751
:10CFC00009F07FC0F82CE92CF8018789813419F524
:10CFD000208D222349F0332727FD30958091DB0FE8
:10CFE00090E028173907B9F4C69CF001C79CF00DF2
:10CFF000D69CF00D1124AE0EBF1E8BE59CE0A80E52
:10D00000B91ED5011C92E20DF31DE80FF91F8091A6
:10D01000E60F808315C18091D50F90E02091DD0F40
:10D02000869DF001879DF00D969DF00D1124E20F75
:10D03000F11DE55AF34F4080B3E6B083F8018789CC
:10D04000882331F4AE81BF811C92B2E6B78B08C051
:10D05000EE81FF81408383E06FEF40E00E94BE706D
:10D06000D80157968C91833639F4C6016F2D7E2DE9
:10D070000E94DC6010920101F801878986598A308C
:10D0800078F480912201882331F4C6016F2D7E2D22
:10D090000E94CC6005C0C6016F2D7E2D0E94D46019
:10D0A0008091DD0F2091D50F30E0269DF001279D66
:10D0B000F00D369DF00D1124E80FF11DE55AF34FE8
:10D0C0004082AE81BF818C91992787FD90952091F8
:10D0D000E60F30E08217930709F048C0F80180811D
:10D0E0008823F1F481818823D9F48789482F552733
:10D0F00047FD50958091EC0F90E04817590749F093
:10D100004217530731F08091EF0F90E0481759070D
:10D1100069F5AE81BF811C9281E6F801808326C04B
:10D12000AE81BF8156968C9156978823F9F4579615
:10D130008C918823D9F4F8018789482F552747FD1A
:10D1400050958091EC0F90E04817590749F042172D
:10D15000530731F08091EF0F90E04817590731F4F1
:10D16000AE81BF811C92E1E65696EC93AE81BF8101
:10D170008C91682F772767FD70958091EC0FE82FD1
:10D18000F0E06E177F0709F045C0D8018C91882325
:10D19000F1F411968C9111978823C9F457968C91CC
:10D1A000482F552747FD50954617570749F0421716
:10D1B000530731F08091EF0F90E04817590751F570
:10D1C000EE81FF811082E2E6D801EC9323C0AE81AC
:10D1D000BF8156968C9156978823E1F457968C918F
:10D1E0008823C1F4D80157968C91482F552747FDC5
:10D1F00050954E175F0749F04217530731F0809161
:10D20000EF0F90E04817590729F4EE81FF81108253
:10D2100082E6868B0894A11CB11CAE81BF81119659
:10D22000BF83AE830F5F1F4F0894811C911C08942D
:10D23000211C311CB981BF5FB983B53109F037CCEE
:10D240000894C11CD11CEA81EF5FEA838B819C8129
:10D2500001969C838B83E93219F15C2CC69CD0012A
:10D26000C79CB00DD69CB00D1124A55AB34FBF83F7
:10D27000AE83EB81FC81E69D8001E79D100DF69D5C
:10D28000100D1124055A134FAA24BB24B1E08B2E94
:10D29000912CA2E02A2E312CFFEFF983ED8307CCED
:10D2A00080912301882351F58091CF0F682F70E082
:10D2B0001091EC0F40E75CE020E030E0A6E1B0E048
:10D2C00013C08081992787FD90958617970709F4E9
:10D2D00010833196E417F507A1F72F5F3F4F4A5EA1
:10D2E0005F4F2832310551F02A9FF0012B9FF00D3E
:10D2F0003A9FF00D1124E55AF34FE3CF8091D00F00
:10D300009091D10F853691056CF08091CF0F682FE9
:10D3100070E01091E60F40E75CE020E030E0A6E12D
:10D32000B0E026C0B091CE0FA091D60F9091E60F3D
:10D3300040E75CE020E030E066E170E0F6E9EF2EE7
:10D34000E7E9FE2E08E919E945C08081992787FDA4
:10D3500090958617970709F410833196E417F5071F
:10D36000A1F72F5F3F4F4A5E5F4F28323105D1F260
:10D370002A9FF0012B9FF00D3A9FF00D1124E55AE2
:10D38000F34FE3CF8081823609F4B0838081813608
:10D3900009F4A0838081803A09F4E0828081813A97
:10D3A00009F4F0828081823A09F400838081833A13
:10D3B00009F410838081853209F490833196E41753
:10D3C000F50701F72F5F3F4FAF014A5E5F4F2832ED
:10D3D000310551F0269FF001279FF00D369FF00D8B
:10D3E0001124E55AF34FCECF27960FB6F894DEBF3F
:10D3F0000FBECDBFCF91DF911F910F91FF90EF90A6
:10D40000DF90CF90BF90AF909F908F907F906F9064
:10D410005F904F903F902F9008953F924F925F9270
:10D420006F927F928F929F92AF92BF92CF92DF9234
:10D43000EF92FF920F931F93CF93DF9384E080933B
:10D4400000018AE39CE00E943F6D81EC92E70E941C
:10D45000596DCC24DD24332433949924939464E1CE
:10D46000562E50E1452E46E1A42EB12C88248394FB
:10D470003BEC632E32E0732E84E0809300019092A7
:10D4800001010E94684880EA9CE00E94F44880E71D
:10D4900090E00E94EF4880E090E060E070E048E2B9
:10D4A00050E02CE130E001E010E00E94B67289E922
:10D4B0009EE60E94F4480E946848CBE1D0E7EE2443
:10D4C00020C0F394F801449150E0415050408E2D1B
:10D4D0006F2D0E94D04886E261E143E050E00E9457
:10D4E000D04887E261E143E050E00E94D048085D07
:10D4F0001F4FF1E1FF1629F7E394219688E2E81621
:10D5000019F08E01FF24DDCF909202019092050167
:10D5100024E0F22E03ED1BE880E00E940049EC01BC
:10D5200089E090E064E170E04BEF5CE70E94DB7122
:10D5300080E190E064E170E0409102010E944A7253
:10D5400085E190E064E170E046EE5CE70E94DB710B
:10D550008DE190E064E170E0409105010E944A7223
:10D560008EE090E067E170E041E05DE70E94DB71F2
:10D57000C5FF07C080910201823018F0855080936A
:10D580000201C4FF0FC0809102018B5F80930201F2
:10D59000813110F04092020180910201853110F03A
:10D5A00050920201C6FF07C080910501823018F039
:10D5B000815080930501C7FF09C0809105018F5FED
:10D5C00080930501853010F0F0920501D0FD17C061
:10D5D000C8010197F1F70894C11CD11CE6EECE16E4
:10D5E000E1E0DE060CF498CF81EC92E70E94876DB3
:10D5F00081EC92E70E94596DCC24DD248DCF80EA26
:10D600009CE00E94F4480E94876D80E090E060E01A
:10D6100070E048E250E02CE130E001E010E00E94D0
:10D62000B67288E08093EC0F85E08093CB0F9092E8
:10D63000E20F8093EF0F80E58093D60F81E5809312
:10D64000CE0F8BE580935A0C89E48093CF0F86E050
:10D650008093D50F8EE08093DD0F82E08093E30FFF
:10D660008AE08093D20F1092DF0F80E095E09093D4
:10D6700025018093240199E0F92E84E0E82E85C1EC
:10D680004092D40F809102010E9451558091240153
:10D690009091250103E0880F991F0A95E1F7909377
:10D6A0002501809324010E9402625092E30FF092C0
:10D6B000D20F809201011092E00F10922001C091D0
:10D6C0002401D09125011091DD0F0091D50F5091CB
:10D6D000DE0F6091DC0F20E030E021C08C918B35B3
:10D6E00019F4072F142F04C08C3511F4672F542F11
:10D6F000862F90E08A9DF0018B9DF00D9A9DF00D94
:10D700001124E50FF11DE55AF34F30824F5F11965A
:10D71000463121F72F5F3F4F2832310561F02A9DB6
:10D72000D0012B9DB00D3A9DB00D1124A55AB34FD9
:10D7300040E0722FD3CF1093DD0F0093D50F50939D
:10D74000DE0F6093DC0F0E94606200E010E00E9438
:10D7500029658091240190912501019790932501DD
:10D76000809324018091DF0F8F5F8093DF0F8730DC
:10D7700010F01092DF0F0E943A5D0F5F1F4F0E31C5
:10D78000110529F7D0932501C093240185E06FEF9F
:10D7900041E00E94BE700E9402620E947A630E9471
:10D7A00029652091DF0F2F5F2093DF0F80912401E7
:10D7B00090912501019790932501809324012730B2
:10D7C00010F01092DF0F0E943A5D809101018823D2
:10D7D00041F08091240190912501181619060CF44E
:10D7E0008EC08091000181508093000180910201E0
:10D7F000853021F08A3011F08F3079F48F5F80937B
:10D8000002018091240190912501181619062CF02F
:10D81000809100018F5F809300018091020184312B
:10D82000B9F480920201809124019091250118168B
:10D8300019062CF0809100018F5F80930001809188
:10D8400005018F5F80930501853010F0E09205019E
:10D85000809124019091250118161906DCF08EE0C4
:10D8600090E069E070E04BE050E023E030E001E060
:10D8700010E00E94B6728FE090E06AE070E047E14D
:10D880005DE70E94DB7188E893E1F3013197F1F7DE
:10D890000197D9F78091DD0F2091D50F30E02A9DB7
:10D8A000F0012B9DF00D3A9DF00D1124E80FF11DB4
:10D8B000E55AF34F108200E010E01092D50F10925D
:10D8C000DD0F80925B0C0E9429658091240190916C
:10D8D0002501019790932501809324018091DF0F0A
:10D8E0008F5F8093DF0F873010F01092DF0F0E9460
:10D8F0003A5D0F5F1F4F0A301105F9F644C0809161
:10D90000E00F813009F047CF30C044979093250154
:10D910008093240168E070E00E94B373462F485D55
:10D9200081E061E028EC0E94D56D8091D70F909145
:10D93000D80FA091D90FB091DA0F0A96A11DB11D91
:10D940008093D70F9093D80FA093D90FB093DA0F8D
:10D950000E9402620E9429658091DF0F8F5F809391
:10D96000DF0F873010F01092DF0F8091240190912B
:10D970002501823091054CF6809102018F5F8093E2
:10D980000201109220010E943E63809100018823D1
:10D9900009F076CE8EE090E069E070E04BE050E078
:10D9A00023E030E001E010E00E94B6728FE090E0EA
:10D9B0006AE070E04DE05DE70E94DB7188E893E18A
:10D9C000F3013197F1F70197D9F756CD90E025E1B2
:10D9D00030E0829FF001839FF00D929FF00D1124A3
:10D9E000ED50F04F618708956093510C089590E0D9
:10D9F00025E130E0829FF001839FF00D929FF00DB2
:10DA00001124ED50F04F12861182089590E025E127
:10DA100030E0829FF001839FF00D929FF00D112462
:10DA2000ED50F04F81E0828B089590E025E130E0E9
:10DA3000829FF001839FF00D929FF00D1124ED5015
:10DA4000F04F6087089590E025E130E0829FF0017B
:10DA5000839FF00D929FF00D1124ED50F04F6483E1
:10DA6000089590E025E130E0829FF001839FF00D62
:10DA7000929FF00D1124ED50F04F6583089590931F
:10DA80004A10809349108FE680934F101092200A1D
:10DA9000E3EFFFE021E09FEF88E120831782968388
:10DAA000138611828583759630E1E734F307A9F771
:10DAB00008951092F40F1092091010921E101092F7
:10DAC0003310019690935310809352109093F20F5D
:10DAD0008093F10F9093561080935510109251102F
:10DAE00010925010109248101092471010924B1044
:10DAF00081E08093200A10924E1010924D100895EC
:10DB00008091F10F9091F20F0E94596D08958091CC
:10DB1000FC0F87FD03C08AEF8093FC0F80911110EA
:10DB200087FD03C08AEF809311108091261087FD36
:10DB300003C08AEF8093261080913B1087FD03C0BD
:10DB40008AEF80933B101092200A089581E0809321
:10DB5000200A0895DC01ED91FC911197AF014F5F10
:10DB60005F4F11965C934E93E4912E2F30E0E7FFC8
:10DB700013C02F7730703695322F2227379527958F
:10DB8000FA014F5F5F4FE4918E2F8F77280F311D81
:10DB9000E7FDF1CF4D935C93C901089580934F1039
:10DBA000089508950E949F490895EF92FF920F9360
:10DBB0001F93CF93DF93182F062FF42EE22EC82F3A
:10DBC000D0E085E190E0C89FF001C99FF00DD89F9B
:10DBD000F00D1124ED50F04F8285882321F08181D2
:10DBE000882309F087C0EE2091F485E190E0C89F7A
:10DBF000F001C99FF00DD89FF00D1124ED50F04FAA
:10DC0000128A8185882309F075C0178273C013308A
:10DC100059F481E091E09093530C8093520C81E091
:10DC20008093510C0F2D08C0812F60E00E949F4906
:10DC3000812F6F2D0E9480490F3799F485E190E084
:10DC4000C89FF001C99FF00DD89FF00D1124ED5031
:10DC5000F04F80914C1086878DE490E1948B838BFC
:10DC600030C089E0089FC0011124E0914910F09173
:10DC70004A10E80FF91F339645915491411551050B
:10DC800071F485E190E0C89FF001C99FF00DD89F25
:10DC9000F00D1124ED50F04F148A138A12C0FA01CE
:10DCA000249185E190E0C89FF001C99FF00DD89FB5
:10DCB000F00D1124ED50F04F26874F5F5F4F548BCE
:10DCC000438B85E190E0C89FF001C99FF00DD89F7C
:10DCD000F00D1124ED50F04F178611860387118245
:10DCE0008FEF8087E782F282108A81E08287128A32
:10DCF000118A1482DF91CF911F910F91FF90EF90C5
:10DD00000895CF92DF92FF920F931F93CF93DF93EB
:10DD1000EBEFFFE08181282F332727FD30958081AD
:10DD2000280F311D2F3F310519F014F02FEF30E08F
:10DD3000C90137FF02C080E090E08083759640E122
:10DD4000EF34F40739F78091200A882309F01AC1CB
:10DD500036C1E0915210F09153109F012F5F3F4F59
:10DD6000309353102093521044914F3F69F5A9010D
:10DD70004F5F5F4F5093531040935210F9018491BD
:10DD80008F3219F41092200A0BC1863009F0EBC0D3
:10DD9000FA013196CF01019690935310809352105F
:10DDA000E491E33529F49093561080935510DBC02D
:10DDB000E53409F0D8C08091551090915610909399
:10DDC000531080935210CFC047FF02C040934B10B6
:10DDD000542F5F70842F90E0807F9070803B91057E
:10DDE00031F1803C910581F18039910509F043C002
:10DDF000C9010196F90144910196909353108093C3
:10DE000052100197FC012491852F90E08C9FF00126
:10DE10008D9FF00D9C9FF00D1124ED50F04F8081EF
:10DE2000882309F4A0C0220F852F638553C0C90140
:10DE30000196F901449101969093531080935210EA
:10DE40000197FC01249153C02F5F3F4F3093531033
:10DE50002093521021503040F9012491852F90E0F9
:10DE60008C9FF0018D9FF00D9C9FF00D1124ED50C3
:10DE7000F04F238778C080914B10582F5F7090E04F
:10DE8000807F9070803B910541F1803C910509F4C1
:10DE90005EC08039910509F066C02F5F3F4F309317
:10DEA00053102093521021503040F9012491852FB6
:10DEB00090E08C9FD0018D9FB00D9C9FB00D1124E0
:10DEC000AD50B04F8C91882309F44DC0220F852F9F
:10DED0001B966C910E94D56D46C02F5F3F4F3093CB
:10DEE00053102093521021503040F90124914730B3
:10DEF00071F4852F90E08C9FF0018D9FF00D9C9F19
:10DF0000F00D1124ED50F04F220F26832CC04C351C
:10DF100071F4852F90E08C9FF0018D9FF00D9C9FF8
:10DF2000F00D1124ED50F04F220F24831CC0443615
:10DF3000D1F4852F90E08C9FF0018D9FF00D9C9F78
:10DF4000F00D1124ED50F04F220F25830CC0852FCA
:10DF500090E08C9FF0018D9FF00D9C9FF00D11249F
:10DF6000ED50F04F438782E590E10E94AA6D9695AF
:10DF700087959093511080935010109248101092F2
:10DF8000471002C0C5E1D0E0609147107091481081
:10DF900080915010909151106817790709F4D9CEEB
:10DFA0006F5F7F4F709348106093471080914D10C2
:10DFB00090914E10019690934E1080934D1002E375
:10DFC0001CE0C4EFDFE0FF24BFEFCB2ED12C89890A
:10DFD000882309F05EC08A899B89892B09F456C081
:10DFE0009E858D85981708F04CC050C08A852A8977
:10DFF0003B898F37E9F4D9018D91BB8BAA8B8F3F79
:10E0000001F1F90161811196BB8BAA8BE82FF0E039
:10E01000EE0FFF1FEF5DF2480190F081E02D8F2D94
:10E020000995EA89FB8981918D87FB8BEA8B28C052
:10E03000A9014F5F5F4F5B8B4A8BF90184918F3F42
:10E0400021F418821B8A1A8A21C04F5F5F4F5B8BB5
:10E050004A8B41505040FA01649190E0880F991F1B
:10E060008F5D9248FC01259134918F2DF90109951E
:10E07000EA89FB893196FB8BEA8B3197E491ED8736
:10E080001E869E858D85981709F4B0CF8E858F5F8B
:10E090008E878985882319F420E030E05DC08F8564
:10E0A0008F3F11F08F5F8F879E81992309F44EC0B7
:10E0B0002F81222309F44AC08D81882309F446C0A8
:10E0C00040914F10442309F441C0899FC00111249D
:10E0D00080509F4F892F992730E0BC01629FC0017B
:10E0E000639F900D729F900D112480509F4F892F38
:10E0F0009927242F30E0FC01E29FC001E39F900D9F
:10E10000F29F900D112480509F4F292F33278B8130
:10E110008823F1F0EA81F0E0E050FA46E491E0581B
:10E12000E89FC001112480509F4F892F9927A60195
:10E13000481B590B429FC001439F900D529F900D69
:10E14000112480509F4F292F332702C020E030E058
:10E150008A819C81890F8A83F8012083F394065F6A
:10E160001F4F6596F4E0FF1609F031CFDF91CF9194
:10E170001F910F91FF90DF90CF9008951F93CF9341
:10E18000DF93582F89E0589FC00111242091491036
:10E1900030914A10280F391FC9010396FC01A5913F
:10E1A000B491F90184918150823010F413E01DC0C4
:10E1B000809109108823B1F080911410851711F413
:10E1C000442381F480911E10882371F080912910DE
:10E1D000851711F4442341F49091181080912D106B
:10E1E000891710F411E001C012E0212F30E0FD0189
:10E1F000449185E190E0289FE001299FD00D389F50
:10E20000D00D1124CD50D04F4E871196BC8BAB8BC7
:10E210001F8680E58A836F838FEF888719861A8A25
:10E22000188A21E02A87198A5C8729831C82133087
:10E2300049F481E091E09093530C8093520C209329
:10E24000510C08C0812F60E50E948049812F6989A7
:10E250000E949F49DF91CF911F910895FF920F93E4
:10E260001F93082FF62E0E94804910E085E190E070
:10E27000089FF001099FF00D189FF00D1124ED503B
:10E28000F04FF2821F910F91FF900895962F482F23
:10E2900050E025E130E0429FF001439FF00D529F96
:10E2A000F00D1124ED50F04F6281691B62830E94D2
:10E2B00080490895482F50E025E130E0429FF00169
:10E2C000439FF00D529FF00D1124ED50F04F9281BD
:10E2D000690F62830E94804908951F93CF93DF9353
:10E2E000FA01549131961491C52FD0E09F012F5F10
:10E2F0003F4F70E095E0660F771F9A95E1F7680F42
:10E30000711D40E00FC084918C9311961C9211975F
:10E310009F5F319612969517B0F34F5F2C0F3D1FFC
:10E32000605E7F4F411740F4DB01AA0FBB1FA05C6A
:10E33000BE4FF90190E0EFCFDF91CF911F9108958B
:10E340008F929F92AF92BF92CF92DF92EF92FF9205
:10E350000F931F93CF93DF93882E962E5A01690156
:10E36000F02E00E010E080EEF80E0CC0882D8C0F2F
:10E370006E2D4F2D0E94B8482196CA15DB05B4F3C7
:10E380000F5F1F4F0C151D052CF4C0E0D0E0E02EF0
:10E39000E90CF3CFDF91CF911F910F91FF90EF9098
:10E3A000DF90CF90BF90AF909F908F900895405294
:10E3B0000E94B8480895FF920F931F93CF93DF9365
:10E3C0008C01F62EEA01FE0144912196442349F086
:10E3D000802F0F5F1F4F4F7740526F2D0E94B8481C
:10E3E000F2CFDF91CF911F910F91FF900895FF928F
:10E3F0000F931F93182F062FF42E42954F704A301B
:10E4000010F4405F01C0495E812F602F0E94B84820
:10E410004F2D4F70812F8F5F4A3010F4405F01C045
:10E42000495E602F0E94B8481F910F91FF90089598
:10E43000FF920F931F93182F062FF42E452F0E9443
:10E44000F771812F8E5F602F4F2D0E94F7711F9102
:10E450000F91FF900895EF92FF920F931F93F62E66
:10E46000042F182F28E0E22EE80E07FF04C0812FAA
:10E470006F2D41E103C0812F6F2D40E10E94B8480C
:10E480001F5F1E1511F0000FF0CF1F910F91FF902D
:10E49000EF900895FF920F931F93CF93DF93F62E83
:10E4A000042FEC0110E0002311F4112349F4802F14
:10E4B0006AE00E94A773905F8C2F6F2D492F03C0D5
:10E4C0008C2F6F2D40E00E94B8481F5F21971330BA
:10E4D00031F0802F6AE00E94A773082FE4CFDF910C
:10E4E000CF911F910F91FF900895CF92DF92EF92FD
:10E4F000FF920F931F93CF93DF93C62E79018A016A
:10E50000EC01DD24E114F1040105110511F4DD2015
:10E5100069F4C801B7012AE030E040E050E00E9411
:10E52000C673462F405F8C2F6C2D03C08C2F6C2D33
:10E5300040E00E94B848D394219786E0D81669F04D
:10E54000C801B7012AE030E040E050E00E94C67305
:10E55000C901DA017C018D01D5CFDF91CF911F91E7
:10E560000F91FF90EF90DF90CF9008957F928F9260
:10E570009F92AF92BF92CF92DF92EF92FF920F9352
:10E580001F93CF93DF93782E862E5A01690178016D
:10E5900000E010E00CC0872D8C0F692DA7010E94B0
:10E5A000D0482196CA15DB05B4F30F5F1F4F0C1539
:10E5B0001D052CF4C0E0D0E0902E980CF3CFDF9135
:10E5C000CF911F910F91FF90EF90DF90CF90BF9070
:10E5D000AF909F908F907F9008957F928F929F929F
:10E5E000AF92BF92CF92DF92EF92FF920F931F9361
:10E5F000CF93DF93782E862EEA01FA01C590D4904E
:10E60000FA013296A590B49000E016C0FC01EE0D20
:10E61000FF1D3296EE0FFF1FEC0FFD1F4591549129
:10E62000812F870D692D0E94D0481F5F812F90E0B8
:10E630008C159D055CF30F5F802F90E08A159B057C
:10E640005CF48C9D70018D9DF00C9C9DF00C112450
:10E6500010E0902E980CEACFDF91CF911F910F918F
:10E66000FF90EF90DF90CF90BF90AF909F908F90F2
:10E670007F9008950F931F93CF93DF938C01C0E099
:10E68000D0E007C00E94F9488823E1F30E94FC48CB
:10E690002196C017D107B4F3DF91CF911F910F914D
:10E6A000089528E088E190E00FB6F894A89580934B
:10E6B00060000FBE209360000895EF92FF920F93C9
:10E6C0001F930AE716E8C8010E943F6D87EBE82E0A
:10E6D0008EE7F82EC7010E94F448C7010E94EF4858
:10E6E0000E9468488FE090E00E943A73C8010E943F
:10E6F0003F6D80E06FEF41E00E94BE7007E016E8DA
:10E7000082E16CE0A8010E94ED7283E090E00E943B
:10E710003A7382E16CE04BE356E80E94ED7282E0CE
:10E7200090E00E943A7382E16CE0A8010E94ED72D1
:10E730008EE190E00E943A730E94684884E190E084
:10E740000E943A731F910F91FF90EF900895991BCB
:10E7500079E004C0991F961708F0961B881F7A95D8
:10E76000C9F78095089597FB092E07260AD077FDF3
:10E7700004D02ED006D000201AF4709561957F4FFA
:10E780000895F6F7909581959F4F0895A1E21A2E6E
:10E79000AA1BBB1BFD010DC0AA1FBB1FEE1FFF1F45
:10E7A000A217B307E407F50720F0A21BB30BE40B95
:10E7B000F50B661F771F881F991F1A9469F76095DC
:10E7C0007095809590959B01AC01BD01CF01089596
:10E7D000AA1BBB1B51E107C0AA1FBB1FA617B70787
:10E7E00010F0A61BB70B881F991F5A95A9F78095A3
:10E7F0009095BC01CD010895629FD001739FF001F7
:10E80000829FE00DF11D649FE00DF11D929FF00DC0
:10E81000839FF00D749FF00D659FF00D9927729FF7
:10E82000B00DE11DF91F639FB00DE11DF91FBD0182
:10E83000CF011124089597FB092E05260ED057FD10
:10E8400004D0A4DF0AD0001C38F4509540953095D0
:10E8500021953F4F4F4F5F4F0895F6F79095809564
:10E86000709561957F4F8F4F9F4F08952F923F92E4
:10E870004F925F926F927F928F929F92AF92BF92D0
:10E88000CF92DF92EF92FF920F931F93CF93DF937C
:10E89000CDB7DEB7CA1BDB0B0FB6F894DEBF0FBED9
:10E8A000CDBF09942A88398848885F846E847D8426
:10E8B0008C849B84AA84B984C884DF80EE80FD8028
:10E8C0000C811B81AA81B981CE0FD11D0FB6F8949E
:0EE8D000DEBF0FBECDBFED010895F894FFCF5F
:0AE8DE000401010708010100000019
:00000001FF
